:020000040800F2
:10000000709C0020C1020008797D00087B7D0008FB
:100010008D7D00088F7D0008917D000800000000A4
:10002000000000000000000000000000D3020008F3
:10003000937D000800000000D7020008E155000889
:10004000DB0200086B5D0008DB0200089F4E000821
:10005000DB020008DB020008514C0008714C00086C
:10006000934C0008B34C0008D54C00084B460008E0
:100070008D460008CF4600081B470008314800089D
:1000800081480008D1480008DB020008DB020008B4
:10009000DB020008DB020008DB020008F54C000868
:1000A000DB020008DB020008DB020008DB020008BC
:1000B0002D5800084F58000871580008DB0200084E
:1000C000DB020008DB020008DB020008DB0200089C
:1000D000DB0200080B4100087B410008EB410008EF
:1000E000374D0008D74E0008DB020008DB0200088D
:1000F000DB020008DB020008DB020008DB0200086C
:10010000DB020008DB02000893580008DB0200084D
:100110005B420008CF420008B5580008D7580008D5
:10012000214900086F490008BF4900080B4A000830
:1001300000F002F800F0B0F80AA090E8000C824449
:100140008344AAF10107DA4501D100F0A5F8AFF226
:10015000090EBAE80F0013F0010F18BFFB1A43F0A5
:1001600001031847F0CA000010CB00000A444FF00A
:10017000000C10F8013B13F0070408BF10F8014B06
:100180001D1108BF10F8015B641E05D010F8016B4B
:10019000641E01F8016BF9D113F0080F1EBF10F8AF
:1001A000014BAD1C0C1B09D16D1E58BF01F801CBD2
:1001B000FAD505E014F8016B01F8016B6D1EF9D555
:1001C0009142D6D37047000000230024002500266A
:1001D000103A28BF78C1FBD8520728BF30C148BFAA
:1001E0000B6070476E2908F0FF80702908F0E581E8
:1001F00066290AF0E18565290AF0DE8567290AF09B
:10020000DB8561290AF0DA8503681B0A28BF41F003
:100210008001692908F0AC80642908F0A98075295B
:1002200008F0A6806F2908F07281782908F0B18162
:10023000E92908F0A584E42908F0A284F52908F04A
:100240009F84EF2908F06F81F82908F0B0810368D6
:10025000DB0928BF41F08001632908F05C84732921
:1002600008F06184E32908F07F84F32908F084848E
:10027000002070471FB509F0A1F9040000200021FB
:100280000AF0A2F8401C6060002000210AF0B2F8D9
:10029000E0601FBD10B510BD09F06BF91146FFF706
:1002A000E9FF00F0BEF809F04DFA03B4FFF7F2FFE2
:1002B00003BC03F0FAFC000080F3088870470000DC
:1002C0000948804709480047FEE7FEE7FEE7FEE7EA
:1002D000FEE7FEE7FEE7FEE7FEE7FEE70448054926
:1002E000054A064B704700009F7E00083101000858
:1002F000706C0020709C0020707C0020707C0020BE
:1003000070B50224E74D641E2878C00709D1E6A025
:1003100000F01FFF01F0A1FF03285ED0E4A003F06E
:10032000FBF82878C1071AD0800718D4E3A000F0A2
:1003300010FF1E2003F0B2F806461E21304602F0E0
:100340001CFA032851D0287820F00100287001F011
:10035000A5FF304603F0E0F8304603F0D9F82878DE
:10036000C10711D081070FD540070DD4D5A000F0EB
:10037000F0FE00F0A0FF03283CD0287820F0040015
:100380002870D4A003F0C8F82878C10711D08107DD
:100390000FD5C0060DD4D2A000F0DBFE00F048FF60
:1003A000032833D0287820F010002870D0A003F064
:1003B000B3F8002CA7DA2878C1072FD081072DD5F4
:1003C000C0062BD50324CD4802F0BFF9CB48401F0F
:1003D00001F0A9FE00F09CFE21E0287840F0010029
:1003E0002870C7A003F098F89BE7287840F0020037
:1003F0002870AEE7287840F004002870C3A142209E
:1004000000F073FFC7A003F087F8BDE7287840F03D
:1004100010002870C6A003F07FF8CCE70224204625
:1004200070BDFEB5C54800F075FD4FF4407005F095
:10043000A3FCC34800F074FCC24801F059F900F075
:1004400060FB05F097FAC0480068BC4C4FF4FA66B0
:1004500070B9BE48006858B9BDA000F07AFEBFA0D0
:1004600000F084FE304605F00BF931206070E0703A
:10047000E07830281AD0BC48D0F8301111B9D0F843
:100480002C0198B13027E770AC4800F033FD61785B
:10049000B64D302914D0312912D0A278B4A003F07F
:1004A0003BF86770A54800F025FDADE0B9A000F06D
:1004B00050FEBBA000F05AFE304605F0E1F8B5E072
:1004C00030296CD067709D4800F014FD05F052FA99
:1004D000FFF716FF022867D0B5A000F03AFEB7A1DB
:1004E000422000F002FF05F045FAA04800F036FB7C
:1004F000022865D0B9A000F02CFE281D02F054FEA1
:1005000002466862002867D0C2F3C72085F8280039
:10051000510502D0401C85F8280095F82830B3A179
:10052000422000F0E2FEBCA000F013FE4FF0FF30CE
:10053000029002A98D4800F049FB022852D00428FD
:1005400058D0B8A000F005FE95F82800BAA1CDE972
:100550000010002302221021184601F092FAB9A0DF
:100560000023009003221021184601F08AFA28681F
:1005700000F0A1FBB6A1422000F0B7FEBA480299F4
:100580004FF400620144286805F02AFB032864D078
:1005900000E004E0B5A1422000F0A7FE46E0A1780B
:1005A000BFA002F0B9FF2FE051A000F0DFFDA2785C
:1005B000C2A1422000F099FE304605F061F823E028
:1005C000C9A000F0D3FDA278CBA1422000F08DFE9F
:1005D000304605F055F817E0A278D2A1422000F08D
:1005E00084FE11E0DBA000F0C1FDDEA1422000F09E
:1005F0007CFE09E0E2A000F0B9FDE5A1422000F098
:1006000074FE304605F03CF8A07800F023FF044665
:1006100000F08EFA204600F06CFF286800F01AFF08
:10062000044600F085FA204600F063FFDF4C2046C8
:1006300000F010FF00F07CFA204600F05AFFDCA02A
:1006400000F087FDDDA000F091FD42F2107005F092
:1006500017F807F0C5FB0020FEBDDBA1422000F02B
:1006600044FE424800F0C9FA032811D095F8290049
:10067000DCA1CDE90010002303221021184601F06F
:1006800000FA286800F017FB304604F0F9FFCDE7C8
:10069000D8A00023009003221021184601F0F1F9A0
:1006A000BBE7000000000020CED5CAD6D6D03A0065
:1006B000CED5CAD6CAA7B0DC00000000C8EBCDF882
:1006C000D6D03A00C1ACBDD3544350B7FECEF1C62C
:1006D000F73A0000544350C1ACBDD3CAA7B0DC0008
:1006E000C1ACBDD3465450B7FECEF1C6F73A0000B8
:1006F000465450C1ACBDD3CAA7B0DC007C1000206A
:10070000CED5CAD6B3C9B9A6000000004465766943
:1007100063652074637020636F6E6E6574636564D7
:1007200021000000544350C1ACBDD3B3C9B9A600E9
:10073000465450C1ACBDD3B3C9B9A600640700206C
:10074000F4060020246503001C0122423C81224261
:10075000D6F7B6AFC9FDBCB63A000000BCB4BDAB1D
:10076000C9FDBCB600000000000021423407002093
:10077000496170466C61673D25632CB2BBBACFB747
:10078000A82CBCB4BDABD6B4D0D04150502563200A
:100790002E000000BBD6B8B4C4A3CABD3A00000006
:1007A000D6B4D0D0D3A6BCB1B3CCD0F200000000F8
:1007B000B2E9D5D2D0C2B9CCBCFE3A00465450B34F
:1007C000F5CABCBBAFB3C9B9A6A3ACBCB4BDABBF83
:1007D000AACABCC9FDBCB6A3A1000000BBF1C8A158
:1007E000B9CCBCFED0C5CFA23A000000D0C2B9CC73
:1007F000BCFEB0FCB4F3D0A12025642062797465FE
:1008000073203B20B2F0B7D6D7D3B0FCCAFDC4BF2B
:100810003A20256420A1A300B9CCBCFED0A3D1E925
:10082000D6D03A00D5FDD4DACFC2D4D8C7EBCEF0BB
:10083000B6CFB5E700000000D7DCD7D3B0FCCAFDC7
:100840003A256400CFC2D4D8D7D3B0FC3A310000E7
:10085000D7D3B0FCA3BA3120A1A3CFC2D4D8B3C997
:10086000B9A6A3A1000000001A130020D7D3B0FC42
:10087000A3BA3120A1A3D0B4C8EB464C415348CA17
:10088000A7B0DCA3A1C9E8B1B8BCB4BDABCCF8D764
:10089000AAB5BDD3A6BCB1B3CCD0F2A3A1000000D1
:1008A000CEDED0E8C9FDBCB62CBCB4BDABD6B4D04E
:1008B000D04150502563202E00000000465450B314
:1008C000F5CABCBBAFCAA7B0DCA3ACBCB4BDABCC53
:1008D000F8D7AA52756E4170704E756D3A2041502E
:1008E000502563A3A1000000B2E9D5D2B9CCBCFE6B
:1008F000CAA7B0DC00000000CEB4CBD1CBF7B5BDA9
:10090000D0C2B9CCBCFEA3ACBCB4BDABCCF8D7AAAA
:1009100052756E4170704E756D3A2041505025638E
:10092000A3A10000BBF1C8A1D0C2B9CCBCFEB4F3F6
:10093000D0A1CAA7B0DCA3ACBCB4BDABCCF8D7AADD
:1009400052756E4170704E756D3A2041505025635E
:10095000A3A10000B9CCBCFED0A3D1E9CAA7B0DCEA
:1009600000000000D0C2B9CCBCFED5BBB6A5B5D83E
:10097000D6B7D0A3D1E9CAA7B0DCA3A1000000007C
:10098000B9CCBCFED0A3D1E9B3ACCAB10000000021
:10099000D0C2B9CCBCFED5BBB6A5B5D8D6B7D0A30E
:1009A000D1E9B3ACCAB1A3A10000000000C00108A6
:1009B000C9E8B1B8B9CAD5CF3A000000C7EBC1AA9F
:1009C000CFB5B3A7BCD20000D7D3B0FCA3BA3120B7
:1009D000A1A3D0B4C8EB464C415348B3C9B9A6A3B0
:1009E000A1000000D7D3B0FC3A2564CFC2D4D8CA46
:1009F000A7B0DC00CFC2D4D8B3C9B9A6BCB4BDABD4
:100A0000D4CBD0D00000000070B505460C467B204A
:100A100005F08CFB012804D12246D2A1284607F01C
:100A2000B4FF7C2005F082FB012804D12246D0A12E
:100A3000284607F0AAFF7D2005F078FB012804D1A5
:100A40002246CEA1284607F0A0FF7E2005F06EFBCF
:100A5000012804D12246CDA1284607F096FF7C202C
:100A600005F064FB88B97D2005F060FB68B97E2045
:100A700005F05CFB48B97A2005F058FB012804D149
:100A80002246C6A1284607F080FFBDE8704005F069
:100A900074BC10B5C44807F0E1FBC44807F0DEFBA6
:100AA000C348044604F092F922460B21C1A007F086
:100AB000D5FBC548002242608260C2600B222146FD
:100AC000001D07F062FFC04800F014FAB848012189
:100AD000253804F084F9B64A1821253ABBA007F05E
:100AE000BDFBB3480B210C300446FFF78DFF2246B7
:100AF0000B21BBA007F0B2FBBDE81040AA4807F0ED
:100B0000ADBB10B504F078FD002002F0CFFF0F2040
:100B100004F026FBFFF7BDFF04F02CFF00F073FD8F
:100B200000F05EFD00F0C2FDBDE8104000F072BEB6
:100B300070B50324AF4D2978490704D5AEA002F063
:100B4000EBFC00F0AFFB2978C90605D5AEA002F09A
:100B5000E3FC00F083FB0446204670BD70B50446FC
:100B600002250121201D04F03AF9ACA1201D07F057
:100B70006AFE211DAB4802F002FB032813D01D21A1
:100B8000201D07F0DBFEA8A1201D07F05CFE211D43
:100B9000A94802F02BFF002803DB012084F8210084
:100BA0000325284670BD002084F821000325F8E7BE
:100BB0006FF30F00A149401804D0B0F5003F03D0F7
:100BC000002070479E4870479E48704770B50546A4
:100BD0000E460224A2020021281D02F005FB30600F
:100BE000002807DB98494058FFF7E2FF286010B162
:100BF000032400E00424204670BD7CB50446022096
:100C000084F8290047E091A1CDE9001000230322D8
:100C10001021184600F035FF00F0E7FC642004F0D6
:100C20002FFD4FF4006694F8290094F828108842AC
:100C300002D1A18CC1F30A06401EC1023246201D1A
:100C400002F0D2FA0546002D2DDB94F8292082A16E
:100C5000422000F04AFB94F829002168401E01EB75
:100C6000C02079493246091F294404F0B9FF0328FE
:100C700007D094F829207EA1422000F036FB042002
:100C80007CBD14F8292F87A1422000F02EFB20788C
:100C9000401C04F8290994F8290094F82810884287
:100CA000B1D903207CBD94F8292085A1422000F011
:100CB0001CFB02207CBD70B50546002406F02BFD10
:100CC0008B49681A8D4227D006DC312D24D0322D75
:100CD00009D0332D20D113E0B0F5003F03D0B0F59B
:100CE000802F19D10CE04025554E05E006EBC420BD
:100CF00006F04AFD641CE4B26D1EEDB2F6D20BE0C4
:100D00004025504E05E006EBC42006F03DFD641C76
:100D1000E4B26D1EEDB2F6D2BDE8704006F007BD3C
:100D2000002140F8191F41608160C160016141618B
:100D30001938192107F0E0BD10B504460B2204F163
:100D4000190007F022FE002084F8250010BD10B520
:100D500004460B2204F1250007F017FE002084F85A
:100D6000310010BDD6D8C9CFB5E7C6F4B6AF000084
:100D7000C8EDB8B4CEBBC6F4B6AF0000B6C0C1A2D1
:100D8000BFB4C3C5B9B7C6F4B6AF0000B4B0BFDADC
:100D9000BFB4C3C5B9B7C6F4B6AF0000D3B2B8B4D8
:100DA000CEBBC6F4B6AF000004C8000848C80008AF
:100DB000190700200D0A426F6F74B0E6B1BE203AE9
:100DC00020252E2A73000000640700200D0AC9E8C0
:100DD000B1B8B1E0BAC5203A20252E2A7300000030
:100DE0000D0AD6D8C6F4D4ADD2F2203A20252E2A48
:100DF0007300000000000020424F4F54B6CFBFAA3E
:100E0000544350C1ACBDD300424F4F54D7A2CFFA88
:100E1000465450B5C7C2BD21000000002E62696E65
:100E20000000000018010020436F6D6D6F6E41706F
:100E3000702E62696E0000009A1000200000FDF71D
:100E400000C0030800C005081E130020CFC2D4D87C
:100E5000D7D3B0FC3A256400D7D3B0FCA3BA25643D
:100E600020A1A3CFC2D4D8B3C9B9A6A3A1000000C2
:100E7000D7D3B0FCA3BA256420A1A3D0B4C8EB4655
:100E80004C415348CAA7B0DCA3A1C9E8B1B8BCB46F
:100E9000BDABCCF8D7AAB5BDD3A6BCB1B3CCD0F20C
:100EA000A3A10000D7D3B0FCA3BA256420A1A3D08E
:100EB000B4C8EB464C415348B3C9B9A6A3A100003E
:100EC000D7D3B0FCA3BA256420A1A3CFC2D4D8CA7B
:100ED000A7B0DCA3A1C9E8B1B8BCB4BDABCCF8D70E
:100EE000AAB5BDD3A6BCB1B3CCD0F2A3A10000007B
:100EF00000C001080146F822544804F0E0BD10B5D6
:100F0000F82107F0F9FCBDE81040F82250494F489D
:100F100004F032BD7CB504462046FFF7F0FF5B20AD
:100F200020706078FF2801D130206070A1783120D6
:100F3000FF2900D1A070E178FF2900D1E070207C6A
:100F400004F11005FF283DD02946424800F03AF947
:100F500094F8500004F15005FF283CD029463D4844
:100F600000F03EF994F8900004F19005FF283BD082
:100F70002946384800F041F994F8D00004F1D00532
:100F8000FF283BD02946334800F044F994F8E000AC
:100F9000FF283CD088B32E492F48E03100F06EF98D
:100FA00094F8F000FF283DD000283BD028492A487B
:100FB000F03100F070F95D2084F8F7002046BDE8BC
:100FC0007C4097E74021284607F096FC23A128465D
:100FD00007F0EBFBBCE74021284607F08DFC21A180
:100FE000284607F0E2FBBDE74021284607F084FCD5
:100FF0001DA1284607F0D9FBBEE708E010212846CE
:1010000007F07AFC1CA1284607F0CFFBBEE704F1ED
:10101000E0001021054607F06FFC17A1284607F0F5
:10102000C4FBBDE70020C4F8F000A4F8F400009071
:1010300001900A22694641F6583002F060FC694688
:1010400004F1F00007F0B1FBB5E7000000880108EB
:1010500064070020020000209A0100202F41424D29
:101060000000000041424D0053686F703334343744
:1010700039343734390000003132312E34312E37D3
:10108000392E38370000000008B5002300901A46BA
:101090001021184600F0F5FC08BD1CB504461021CF
:1010A000002200913EA31146104600F0BFFC3F49CC
:1010B0000022CDE90021002110232022084600F063
:1010C000ACFE0C2100220091234611461A2000F0AC
:1010D000ADFC1CBD1CB5044610210022009130A3BC
:1010E0001146402000F0A2FC304900224031CDE9F9
:1010F0000021102320220021402000F08EFE0C2130
:1011000000220091234611465A2000F08FFC1CBD9E
:1011100010B5102002F0C2F90446254B25A210217B
:10112000204607F0A7F82046FFF7D4FF10212046FD
:1011300007F0E2FB1E4B21A25B1D1021204607F0A9
:1011400099F82046FFF7A9FF2046BDE8104002F0BD
:10115000DFB908B50023009001221021184600F0E5
:1011600090FCBDE80840022000F080BC08B50023D8
:10117000009002221021012000F083FC08BD38B548
:101180000C460023009001221021184600F079FC43
:101190000023022210211846009400F072FC38BD92
:1011A000202020202020202000000000B0AE0008D9
:1011B0007710002025736D56000000004353512521
:1011C0007300000070B50C4600F58B708021054659
:1011D00007F092FB21462846BDE8704007F0E5BACB
:1011E00070B504460D468021601C07F085FB29463A
:1011F000601CBDE8704007F0D8BA70B50C4681306D
:101200008021054607F078FB21462846BDE870405E
:1012100007F0CBBA70B50C4600F582701021054678
:1012200007F06AFB21462846BDE8704007F0BDBACA
:1012300010B5114801F009FF03280ED10E4801F046
:1012400032FF032809D10C4801F04CFF032804D1D8
:10125000BDE81040084801F073BF10BD10B5064846
:1012600001F06BFF032805D103480078BDE810406A
:1012700001F091B910BD00000200002070B50446D5
:101280000D461021601C07F037FB2946601CBDE8A5
:10129000704007F08ABA10B50446084607F05CFAB9
:1012A000608210BD10B5002001F0D6FCBDE81040F2
:1012B000012001F070B910B501F0F8FB03280CD142
:1012C000444801F0CDFC04464249032C06D04A8A2A
:1012D000491C41A002F07AF9204610BD4A8A491CF7
:1012E00044A002F019F9204610BD0FB4F8B5064627
:1012F000022540F2492002F0D1F8044608AB0093E1
:101300002F02394604F12600079A06F08DFF0028C7
:1013100001DDB8420BDD82223DA142A002F056F968
:10132000204602F0F5F80220F8BC5DF814FB2822F4
:1013300022706670642290FBF2F13031A17090FB54
:10134000F2F102FB11010A2291FBF2F13031E1705E
:1013500090FBF2F102FB1100303020711D49891E13
:1013600008786071401CC0B20870392801D930205B
:101370000870042232A1A01D07F007FB012104F12F
:101380000A0003F02CFD3B2184F8221030220221B8
:1013900004F1230007F0A8FA262184F8251003227F
:1013A00029A1204607F0EFF929480078400708D521
:1013B000204607F029FA82B22146064801F065FC72
:1013C0000546204602F0A8F8204602F0A1F828467B
:1013D000AAE700009A01002054435020536572761A
:1013E0006572C1ACBDD3CAA7B0DC3A25733A256497
:1013F00020A3A10054435020536572766572C1AC9E
:10140000BDD3B3C9B9A63A25733A256420A3A10078
:10141000555345525F5443505C757365725F7463F6
:10142000702E630025732C25643A757044617461D5
:10143000427566207370696C6C6F766572A3A1004B
:101440004D41433A000000002458290D0A000000D5
:101450000000002070B50446002504F08BFA2E4EE3
:10146000A01BB44211D006DC312C0ED0322C1DD082
:10147000332C06D12BE0B0F5003F17D0B0F5802F0C
:1014800025D026A14220FFF730FF706840F6010109
:10149000B1EB104F05D12AA14220FFF726FF3546B8
:1014A00020E02DA14220FFF720FF1BE0304C6068B8
:1014B0002114B1EB104F05D12EA14220FFF715FFEB
:1014C00025460FE031A14220FFF70FFFDDE7354C45
:1014D00060682114B1EB104F06D133A14220FFF711
:1014E00004FF2546284670BD35A14220FFF7FDFECA
:1014F000CBE710B50168384A1140B1F1005F09D15E
:101500004168364C21600068FEF7D6FE2068BDE8D1
:101510001040004710BD000000C001084150504E6F
:10152000554DB2BBBACFB7A8A3A1BCB4BDABD6B41E
:10153000D0D0D3A6BCB1B3CCD0F2A3A100000000A0
:10154000BFAACABCD6B4D0D041505031D3C3BBA778
:10155000B4FAC2EB2100000041505031D3C3BBA705
:10156000B4FAC2EBD2D1CADCCBF0A3A100000000D8
:1015700000C00308BFAACABCD6B4D0D04150503274
:10158000D3C3BBA7B4FAC2EB2100000041505032D4
:10159000D3C3BBA7B4FAC2EBD2D1CADCCBF0A3A1B0
:1015A0000000000000C00508BFAACABCD6B4D0D055
:1015B00041505033D3C3BBA7B4FAC2EB21000000A3
:1015C00041505033D3C3BBA7B4FAC2EBD2D1CADC6B
:1015D000CBF0A3A1000000000000FE2FB00100200E
:1015E00010220921042003F091BA0921042003F0FC
:1015F000F3BA10B5FFF7F9FF4FF4C87004F040F8E4
:10160000BDE81040F1E738B506240C2348221946FE
:101610000020009403F096FA082348220B210020B2
:10162000009403F08FFA0823482209210220009435
:1016300003F088FA0823482207210220009403F0CF
:1016400081FA0823482206210220009403F07AFA46
:10165000082348220F210320009403F073FA082383
:1016600048220D210320009403F06CFA48220B213C
:10167000032003F04BFA48220821002003F046FA29
:1016800048220921022003F041FA482208210220C1
:1016900003F03CFA48220E21032003F037FABDE89C
:1016A000384048220C21032003F030BA10220A21CE
:1016B000042003F02BBA0A21042003F08DBA10B5E0
:1016C000FFF7F9FF4FF4C87003F0DAFFBDE81040F0
:1016D000F1E7000010B50A460146114801F0F9FF94
:1016E000002804D0BDE810400EA001F06FBF10BD6F
:1016F00010B504460A4801F0E3FF01230C222146FD
:10170000002002F0DDFAAFF23301BDE81040002006
:1017100002F0AABA0A460146002002F006BC000008
:101720005C080020735573625175657565D2E7B327
:10173000F6A3A1000320401EC0B2FCD27047F0B552
:101740000346002500260127F94C01290CD0002270
:10175000C4F89861C4F89061C4F894613AB118066D
:101760000DD5C4F89C610CE0C4F89871F2E7180636
:1017700002D5C4F89C7104E0C4F89C6101E0C4F88F
:101780009C71C4F89471FFF7D5FF5806030E6D1CC9
:10179000EDB2082DE0D3C4F89071C4F89871F0BD93
:1017A00010B50446B031C8B200221146FFF7C7FF9A
:1017B000A41CC4F30310002240F010001146FFF7F0
:1017C000BEFF04F00F000022BDE810401146B6E74E
:1017D00030B5002505F1B0000022C0B21146FFF778
:1017E000AEFF002211460220FFF7A9FF002211469A
:1017F0001020FFF7A4FF0024002201211046FFF76C
:101800009EFF641CE4B2802CF6D36D1CEDB2082D53
:10181000E0D330BD70B510220421002003F076F92A
:1018200010220521002003F071F91022062100206A
:1018300003F06CF910220721002003F067F9102251
:101840000521022003F062F9BA4C012525606420CD
:1018500003F016FF00202060642003F011FF2560D4
:1018600000221146AE20FFF76AFF00221146022037
:10187000FFF765FF002211461020FFF760FF0022EE
:1018800011464020FFF75BFF002211468120FFF741
:1018900056FF00221146FF20FFF751FF002211469C
:1018A000A120FFF74CFF00221146C820FFF747FF99
:1018B00000221146A620FFF742FF00221146A82071
:1018C000FFF73DFF002211463F20FFF738FF0022BF
:1018D0001146D320FFF733FF002211461046FFF7D1
:1018E0002EFF00221146D520FFF729FF00221146C6
:1018F0008020FFF724FF00221146D920FFF71FFFA9
:1019000000221146F120FFF71AFF00221146DA20CB
:10191000FFF715FF002211461220FFF710FF0022EB
:101920001146DB20FFF70BFF002211464020FFF796
:1019300006FF002211462020FFF701FF002211467A
:101940000220FFF7FCFE002211468D20FFF7F7FE74
:10195000002211461420FFF7F2FE00221146A420B7
:10196000FFF7EDFE00221146A620FFF7E8FE002259
:101970001146AF20FFF7E3FE00221146AF20FFF72C
:10198000DEFEFFF725FFBDE870400021084607E7AF
:101990002DE9F041804606980E461F460024203867
:1019A000C5B2B8F17F0F02D9A046B61CF6B20C2A18
:1019B00006D0102A19D0BDE8F0415FA001F006BEA4
:1019C000761CF1B24046FFF7EBFE604905EB45009F
:1019D00001EB40053A46285D0121FFF7B0FE641C8B
:1019E000E4B2062CF6D3BDE8F08131464046FFF75D
:1019F000D7FE574800EB05153A46285D0121FFF751
:101A00009EFE641CE4B2082CF6D3761CF1B240466C
:101A1000FFF7C6FE002428193A46007A0121FFF795
:101A20008EFE641CE4B2082CF5D3DCE72DE9F84304
:101A30000446DDF820800E4691461F46002510E042
:101A400000904B46424631462046FFF7A1FF04EB8B
:101A50005800C4B2782C02D90024761CF6B26D1C52
:101A6000EDB2785D0028EBD1BDE8F88308B5102110
:101A700040060091010E002236A31046FFF7D6FF64
:101A800008BD0FB42DE9FE4F0C46934600254FEAE2
:101A900054088020B0FBF8F64FEA4B07102C1BD0FF
:101AA000042002900DF14409CDF80490701C01F05F
:101AB000F5FC82464B46711C5046109A06F0B4FB6A
:101AC0008146B1450BD90AEB060010F8010C7F28BE
:101AD00005D9A6F1010905E064200290E2E7B145CD
:101AE00000D9B1460C98012802D002280AD105E09D
:101AF000A6EB0900400808FB00F503E0A6EB09008F
:101B000008FB00F5B9F1000F7DDD5846FFF7AEFF89
:101B10000026A8E01AF806107F2925D80091F9B20E
:101B2000E8B222460F9BFFF733FF05EB540599E01F
:101B300000002142940122424E6F2020434841522E
:101B4000484947485F65202E0000000048BD000856
:101B500070BF0008202020202020202020202020CE
:101B60002020202000000000002078E0102C02D06F
:101B70000C2C38D072E0C0EBC00202EB8203DA4AD0
:101B800003EB020898F82020914267D10AEB060285
:101B900098F8213052789A4260D1F9B2E8B2FFF752
:101BA000FFFD4FF0000B07E018F80B0001210F9A22
:101BB000FFF7C5FD0BF1010BA345F5D3781CC1B2AE
:101BC000E8B2FFF7EDFDA34607E018F80B0001218E
:101BD0000F9AFFF7B4FD0BF1010BBBEB440FF4D3ED
:101BE0002544761C3EE000EBC00202EB4203BE4AF5
:101BF0006C3A03EB020898F8182091422ED10AEBB8
:101C00000602527800E032E098F819309A4225D165
:101C1000F9B2E8B2FFF7C4FD4FF0000B07E018F887
:101C20000B0001210F9AFFF78AFD0BF1010BA34571
:101C3000F5D3781CC1B2E8B2FFF7B2FDA34607E0C6
:101C400018F80B0001210F9AFFF779FD0BF1010B3A
:101C5000BBEB440FF4D32544761C03E0401C029AEE
:101C6000904283D3761C4E45FFF454AF09E008D070
:101C7000B6229EA1A3A006F0F1FAAFF2341006F04E
:101C8000EDFA5046BDE8FE0F5DF814EB01F040BCE4
:101C900000B5002211468D20FFF751FD00221146AC
:101CA0001420FFF74CFD00221146AF205DF804EB35
:101CB00045E500B5002211468D20FFF740FD0022CA
:101CC00011461020FFF73BFD00221146AE205DF8C3
:101CD00004EB34E52DE9FF5F80460E9D8B461F46E1
:101CE000002459464046FFF75BFD0BF101090C2D1E
:101CF00008D0102D4FD0AFF2C01004B0BDE8F05F97
:101D000001F064BCDFF8E0A1AAF16C0A3CE06C22AF
:101D10001B2300203D1932E000EBC00606EB46060F
:101D20005644395D96F818C0614527D1697896F810
:101D300019C0614522D159464046FFF731FD0025C3
:101D40000121705D029AFFF7FAFC6D1CEDB20C2DBB
:101D5000F6D309F0FF014046FFF722FD0C250121D3
:101D6000705D029AFFF7EBFC6D1CEDB2182DF6D3F7
:101D700008F10C0808F0FF08641C04E0401C92FB0A
:101D8000F3F18142C8D8641C384606F03DFDA042FC
:101D9000BDD8BDE8FF9FDFF850A138E000203A5DD4
:101DA0003B19C0EBC00101EB810101EB0A0696F87B
:101DB00020108A4227D1597896F82150A94222D181
:101DC00059464046FFF7ECFC00250121705D029A60
:101DD000FFF7B5FC6D1CEDB2102DF6D309F0FF0135
:101DE0004046FFF7DDFC10250121705D029AFFF7E8
:101DF000A6FC6D1CEDB2202DF6D308F1100808F0FA
:101E0000FF08641C02E0401C6428CAD3641C3846E6
:101E100006F0FAFCA042C1D8BBE72DE9F04F81469D
:101E2000DDE909BA0E460025580705D0012000EB70
:101E3000D30702EB090815E0DF08FAE73146484608
:101E4000FFF7AEFC4C4609E028466D1C1AF800006E
:101E50005A460121FFF773FC641CE4B2A045F3D895
:101E6000761CF6B2BE42E9D3BDE8F08F10B586B05D
:101E70000121080304F04BFA04220621002002F09D
:101E800045FE18220521002002F040FE18220721FD
:101E9000002002F03BFE10220421002002F036FE5A
:101EA0000020ADF804004FF48271ADF80610ADF8D3
:101EB0000800ADF80A00ADF80C004FF40071ADF861
:101EC0000E100821ADF81010ADF812000720ADF883
:101ED0001400104C01A9204606F076F80121204696
:101EE00006F0F7F806B010BD9CAF00082E2E5C4837
:101EF000415244574152455C4F4C45445C6F6C65C0
:101F0000642E63004C6F674572723A2025732C254E
:101F10006400000000300140072813D2DFE800F021
:101F20000406080A0C0E1000E6A07047E7A07047F0
:101F3000E9A07047EBA07047EDA07047EFA0704795
:101F4000F1A07047F4A070474FF4A071F54806F077
:101F5000D3BC4FF4A071F44806F0CEBCF349002086
:101F600048604FF41061F24806F0C6BC70B50646F2
:101F70000D46EE4C207800280AD0ED4861682A46CC
:101F80000844314606F06BFC60682844606070BD10
:101F9000E8A1304601F02AFD002821DBE7A1304608
:101FA00001F024FD00280DDB2A463146E74801F008
:101FB00090FB0028EBD0BDE870408322E4A1EDA0A7
:101FC00001F004BB2A463146F14801F082FB0028AB
:101FD000DDD0BDE870408A22DDA1EEA001F0F6BAA6
:101FE000D04806F011FCC0F5A070A84205D93146D2
:101FF000BDE87040CB4806F026BC9622D4A1ECA0E8
:1020000001F0E4FAFFF7A0FF3146BDE870404FF45D
:10201000A072C44806F0B9BC0FB42DE9F84F82464F
:102020004FF00408C148CAEBCA01083000EB810434
:10203000667E60680B904FF4A165284601F02EFA89
:1020400083460CAB0093294658460B9A06F0ECF8F1
:1020500007464FF00009002F01DDAF423EDDC922E7
:10206000BBA1DAA001F0B2FA584601F051FA022001
:10207000BDE8F80F5DF814FBFFF766FF0025BAB264
:102080005946022001F051FF16E0642003F0F8FAEF
:10209000E168A44801F0AAFC20612069002802DB65
:1020A0004FF003081DE061699E4801F09FFC002885
:1020B00002DB4FF0020814E028466D1C2189EDB2C6
:1020C0008842E2D3607E801B00EBC00101EB001070
:1020D0004FF4FA7101EB800003F0D2FA761EF6B2EB
:1020E000CAD2584601F014FACDF80090B8F1050FA5
:1020F0000ED2DFE808F0030507090B00BAA408E0D8
:10210000BCA406E0BEA404E0BFA402E0C0A400E0BA
:10211000C1A45046FFF700FF01462246C1A001F0CE
:1021200029FA4046A4E770B50446002020602071DB
:1021300000210620FFF770FF0546032D09D12C2151
:10214000784806F056FB411C04230D22204601F07E
:1021500070FB284670BD70B505461521284606F06F
:10216000CBFB00210520FFF757FF0446032C09D1C4
:102170000D216C4806F0FDFA811C14230D2228461F
:1021800001F057FB204670BD10B500210220FFF77B
:1021900043FF032808D000210320FFF73DFF002163
:1021A000BDE81040022037E710BD0021012033E7D1
:1021B0009E4901200860704770B500240425FFF790
:1021C000F7FFFFF7C1FE4FF47A7610E0641CE4B22B
:1021D000304603F055FA96A1524801F007FC00285A
:1021E00005DB214693A001F0C5F9032501E0142C7D
:1021F000ECD3284670BD8D490020086040F6B83009
:1022000003F03EBA10B510220F21042002F07EFC2C
:10221000FFF7F1FF10220B21042002F077FC834925
:1022200000201039086010BD10B501230C224FF4B6
:10223000E131022001F044FDFFF786FEFFF789FE41
:10224000424801F03DFA524801F03AFAAFF2E32178
:10225000BDE81040022001F007BD70B5FFF7E4FFB4
:10226000FFF7D0FFFFF7A8FFFFF79FFFFFF78CFFF7
:1022700004462C483838FFF76EFF2A4A1421383AB2
:1022800072A001F049F9274823380546FFF74BFFB4
:10229000294673A001F040F9204670BD10B5002119
:1022A0000846FFF7B9FE0446032C02D072A001F0E5
:1022B0008DF94FF47A7003F0E3F9FFF79CFF2046A5
:1022C00010BD00005455524E4F46460048414E4402
:1022D0005348414B450000005155455259434F4E1C
:1022E00046494700434C4F534545434F00000000CB
:1022F00053415645434F4E464947000051554552BC
:102300005952454C455345005155455259564F4C2D
:102310005441474500000000CEDEB4CBC3FCC1EE03
:10232000000000009A100020DA110020B401002003
:102330001A1300202B51495552433A002B5149554D
:1023400052433A2022726563762200001A1C002054
:102350002E2E5C48415244574152455C4C54455CDA
:10236000454332305C656332306D6F64756C652E49
:102370006300000025732C25643A73546370517513
:10238000657565207370696C6C6F766572A3A100CA
:102390002024002025732C25643A735572635175EF
:1023A000657565207370696C6C6F766572A3A100AA
:1023B00025732C25643A656332304174427566207A
:1023C0007370696C6C6F7665722E200025732C25F6
:1023D000643A636D645061636B207370696C6C6FF9
:1023E000766572A3A1000000496E506172616D456F
:1023F000727200004F7574506172616D45727200A7
:1024000052554E455252000052554E4F4B0000005F
:1024100054494D454F555400CEB4D6AAB4EDCEF331
:10242000000000002573202573000000BC0123423A
:10243000524459004543323020537461727420571E
:1024400061697465643A2564205300004543323065
:1024500020C8EDBCFEB0E6B1BEA3BA252E2A73009B
:102460004543323020B9A9B5E7B5E7D1B9A3BA25BC
:1024700073206D56000000004543323020C8EDB98E
:10248000D8BBFACAA7B0DCA3ACBCB4BDABB6CFB561
:10249000E7B9D8BBFAA3A1000FB42DE9F84F8146E4
:1024A0000427F348C9EBC90100EB8104667E60682C
:1024B0000B90802000F0F2FF82460CAB009380214D
:1024C00050460B9A05F0B0FE8046B8F1000F02DDD1
:1024D000B8F1800F2FDD6522E6A1EEA001F076F8BD
:1024E00002272BE0FFF730FD00251FFA88F2514646
:1024F000022001F01AFD14E0642003F0C1F8E16845
:10250000EB4801F073FA20612069002801DB032702
:1025100014E06169E64801F069FA002801DB02274E
:102520000CE028466D1C2189EDB28842E4D34FF4BB
:102530007A7003F0A5F8761EF6B2D3D2504600F0BA
:10254000E7FF00200090052F0ED2DFE807F003051B
:1025500007090B00D7A408E0D9A406E0DBA404E037
:10256000DCA402E0DDA400E0DEA4484600F05AF955
:1025700001462246DEA000F0FDFF3846BDE8F80F18
:102580005DF814FB02460021DBA3072084E7024626
:102590000021082080E70246002109207CE72DE980
:1025A000F04104460F46224600210A20FFF774FF3F
:1025B0000646032E20D1AE4D012C20D0022C25D072
:1025C000032C2AD0CEA1BA4801F010FAC5F8280190
:1025D000D5F8280100280EDBD5F82811B44830348E
:1025E0000830085CA04206D1D5F82811B0480A305E
:1025F000085C312818D002263046BDE8F081C0A121
:10260000AB4801F0F3F9C5F82801E1E7BFA1A848FC
:1026100001F0ECF9C5F82801DAE7BFA1A44801F000
:10262000E5F9C5F82801D3E7D5F82811A04810230B
:102630000F3001442222384601F0FBF8DCE72DE997
:10264000F04104252D2400210120FFF725FF984E9D
:10265000874F09364FF4FA6815E0404603F010F84A
:1026600000210220FFF718FF0546032D0BD1B86C9F
:10267000002807DDB86C805D312807D0B86C805D1C
:10268000352803D00225641E601CE6D12846B4E735
:102690002DE9F04104251E2400210320FFF7FCFE54
:1026A000834E734F0A364FF4FA6818E0404602F042
:1026B000E7FF00210420FFF7EFFE0546032D0ED1B2
:1026C000D7F88000002809DDD7F88000805D312828
:1026D00008D0D7F88000805D352803D00225641E1D
:1026E000601CE3D1284688E770B5054619212846C5
:1026F00006F002F900210846FFF7CEFE0446032C3F
:1027000009D15B4801696A481923083001440D2248
:10271000284601F08EF8204670BD10B50021052036
:10272000FFF7BAFE032801D07EA010BD504C9C34A8
:1027300020685F4908440D2106F01BF80021017054
:1027400021685B480A30084410BD70B5054600207A
:10275000286000210620FFF79FFE0446032C0AD1C3
:102760004348D0F8B81052481923801D01442C2248
:10277000284601F05EF8204670BD2DE9F04105467F
:102780000E466D480446FFF7AFFF032809D06BA241
:102790003146284605F06EFD6BA000F017FF0220C1
:1027A0002BE7224619216CA000F0B6FEFFF747FF89
:1027B0000446032C09D06DA23146284605F05AFD87
:1027C0006DA000F003FF022017E7FFF761FFFFF79E
:1027D000A4FF01466EA000F09FFE5748001F074669
:1027E000FFF7B3FF3B466EA23146284605F042FD97
:1027F0003A4603216DA000F08FFE2046FDE670B53D
:1028000005460E462846FFF7BDFE2846FFF7BFFEE9
:102810000446032C03D131462846FFF7C0FE20466C
:1028200070BDB8E610B50B281DD2DFE800F0060831
:102830000A0C0E10121416181A0060A010BD62A027
:1028400010BD63A010BD64A010BD65A010BD66A042
:1028500010BD69A010BD6BA010BD6DA010BD6FA014
:1028600010BD72A010BD75A000F0B0FE79A010BD23
:10287000800200202E2E5C48415244574152455C54
:102880004C54455C454332305C656332306E657450
:102890002E63000025732C25643A636D64506163D8
:1028A0006B207370696C6C6F766572A3A100000079
:1028B0009A100020496E506172616D45727200007D
:1028C0004F7574506172616D4572720052554E457C
:1028D0005252000052554E4F4B00000054494D4596
:1028E0004F555400CEB4D6AAB4EDCEF3000000008C
:1028F0002573202573000000434D494F540000000C
:102900002B51494143543A20310000002B51494199
:1029100043543A20320000002B51494143543A209D
:1029200033000000BBF1C8A1CDF8C2E7D0C5CFA2EB
:10293000CAA7B0DC2100000080100020C7EBB2E580
:10294000C8EB53494DBFA800CEB4BCECB2E2B5BD54
:1029500053494DBFA800000053696DBFA8494343C8
:102960004944A3BA252E2A730000000053494DBFE5
:10297000A8C7B7B7D100000053494DC7B7B7D1CEEC
:10298000DEB7A8D7A2B2E1C9CFCDF8C2E7000000F8
:10299000CDF8C2E7D0C5CFA2A3BA257300000000CE
:1029A000D0C5BAC5D6CAC1BF3A2573004C5445201C
:1029B000435351A3BA252E2A7300000051554552A6
:1029C00059494343494400005345544353000000D0
:1029D000515545525943530053455450530000003C
:1029E000515545525950530051554552594E455431
:1029F000494E464F0000000051554552594353512E
:102A000000000000434F46434F4E544558540000C9
:102A1000414354434F4E54455854000044454143AC
:102A200054434F4E544558540000000051554552F0
:102A300059434F4E5445585400000000454332302E
:102A400020CEDED0A7654E6574436D644E756D2152
:102A500000000000CEDEB4CBC3FCC1EE00000000DD
:102A600005280ED2DFE800F0030507090B00D7A008
:102A70007047D9A07047DBA07047DCA07047DDA08D
:102A80007047DEA0704705280ED2DFE800F003058E
:102A900007090B00DCA07047DEA07047E0A070477C
:102AA000E2A07047E4A07047E6A0704770B5102020
:102AB00000F0F4FC054629460120FFF770FD0328CD
:102AC00007D029460120FFF79AFE0446032C02D0C6
:102AD00005E0032070BD2946DDA000F01DFD28465D
:102AE00000F016FD204670BD0FB42DE9F84F814669
:102AF0004FF00408DA48C9EBC90100EB8104667E97
:102B000060680B90802000F0C9FC82460CAB0093FB
:102B1000802150460B9A05F087FB0746002F01DD08
:102B2000802F2FDDCFA000F051FD4FF002082CE0E8
:102B3000FFF70AFA0025BAB25146022001F0F5F972
:102B400016E0642002F09CFDE168D24800F04EFFE0
:102B500020612069002802DB4FF0030815E061695D
:102B6000CC4800F043FF002802DB4FF002080CE0E5
:102B700028466D1C2189EDB28842E2D34FF47A7069
:102B800002F07EFD761EF6B2D2D2504600F0C0FCB6
:102B90004046FFF765FF04464846FFF774FF0146CD
:102BA0002246BDA000F0E6FC4046BDE8F80F5DF807
:102BB00014FB7CB5024600210220FFF795FF064674
:102BC000032E2BD1002000900190162000F066FC0F
:102BD0000446A34DA96CAF480A30085C2070A96C6C
:102BE000AC481023133001442C22601C00F021FE5D
:102BF000601C05F009FEA96C1430A64A0523114497
:102C000001442C22684600F014FE21786B46621CB9
:102C1000A3A000F0AFFC204600F07AFC30467CBD5B
:102C20001CB50446CDE900230B4600212246084688
:102C3000FFF75AFF03280ED189490B69954A3034B2
:102C400009329A5CA24205D10A6992490B31515C62
:102C5000302900D002201CBD02460021012043E79C
:102C600070B504462078FFF7F7FF03280CD1A38A3C
:102C7000628A2078611CFFF7D3FF0546032D02D13D
:102C80002078FFF796FF284670BD2DE9F84F0646DD
:102C90008A469146B9F1000F0DD00025A8460024C0
:102CA0000427FFF751F932786D4EB16D4B46022083
:102CB00001F084F90DE00320BDE8F88F142002F044
:102CC000DFFC3E21734805F054FD10B14FF00108C0
:102CD00004E028466D1CEDB24628EFD3B8F1010F91
:102CE00010D03846FFF7BCFE04460320FFF7CBFEAA
:102CF00001466848009077A3224679A000F066FC60
:102D00003846D9E74A465146022001F00EF930E034
:102D1000642002F0B5FCF16F5E4800F067FEC6F873
:102D20008000D6F8800000280DDB03273846FFF727
:102D300097FE04460420FFF7A6FE0146224656A051
:102D400000F018FCDCE7D6F88410524800F04EFE84
:102D500000280EDB02273846FFF782FE04460420D7
:102D6000FFF791FE01464B4B224660A000F02EFC7F
:102D7000C6E72046641CB6F87810A4B28842C7D3D0
:102D8000BEE770B5054605245BA1284600F02EFE7F
:102D9000002801DD002416E05CA1284600F026FE94
:102DA000002801DD04240EE05DA1284600F01EFE8F
:102DB000002801DD022406E05EA1284600F016FE90
:102DC000002800DD0324204670BD0000496E5061DC
:102DD00072616D45727200004F7574506172616D61
:102DE0004572720052554E455252000052554E4F98
:102DF0004B00000054494D454F555400CEB4D6AA5F
:102E0000B4EDCEF3000000004F50454E534F434BFE
:102E100045540000434C4F5345534F434B455400DA
:102E20005155455259534F434B4554005443505309
:102E3000454E44434D44000054435053454E444294
:102E400055460000CEDEB4CBC3FCC1EE000000004E
:102E5000544350B1BEB5D84950A3BA257300000001
:102E6000B403002054637020636D645061636B2071
:102E7000D2E7B3F6A3A12D2DD4F6BCD35443505FB3
:102E8000434D445041434B5F4C454ECAFDD6B5A11E
:102E9000A30000009A100020257320257300000075
:102EA000544350204368616E6E616CA3BA25632061
:102EB000A1A320B7FECEF1C6F74950A3BA2573A14E
:102EC000A320B7FECEF1C6F7B6CBBFDAA3BA2573FF
:102ED00000000000CEB4CAD5B5BD223E22000000DD
:102EE0002573202573202573202573002573202545
:102EF00073202573000000002B51495552433A209E
:102F000022636C6F73656422000000002B514955E9
:102F100052433A2022706470646561637422000039
:102F20002B51495552433A2022696E636F6D696E89
:102F3000672200002B51495552433A2022696E63A3
:102F40006F6D696E672066756C6C22000FB42DE999
:102F5000F84F81460427DF48C9EBC90100EB810423
:102F6000667E60680B90BD01284600F097FA8246A5
:102F70005FEA0A0010D00CAB009329460B9A05F0CB
:102F800053F98046B8F1000F01DDA84538DDD2A025
:102F900000F01CFB022736E0DBA000F017FB5046D8
:102FA00000F0B6FA0220BDE8F80F5DF814FBFEF75A
:102FB000CBFF00251FFA88F25146022000F0B5FF32
:102FC00014E0642002F05CFBE168D74800F00EFDDD
:102FD00020612069002801DB032714E06169D248E1
:102FE00000F004FD002801DB02270CE028466D1CE0
:102FF0002189EDB28842E4D34FF47A7002F040FBAD
:10300000761EF6B2D3D2504600F082FA002000902D
:10301000052F0ED2DFE807F0030507090B00C3A454
:1030200008E0C5A406E0C7A404E0C8A402E0C9A45F
:1030300000E0CAA4484600F020F90146BA4B2246F7
:10304000C9A000F097FA3846ADE770B504460021F4
:1030500022780846FFF77AFF032810D104F1810394
:103060001E46621C00210120FFF770FF0546324614
:10307000611CC0A000F050FA032D01D0284670BD9D
:1030800004F20114002122780220FFF75FFF62782A
:1030900000210320FFF75AFFA27800210420FFF748
:1030A00055FF284670BD70B50446102000F0F6F9B3
:1030B000054620782946FFF772FA032807D02078C2
:1030C0002946FFF79CFB0446032C02D005E00320B1
:1030D00070BD2946B1A000F01FFA284600F018FA8A
:1030E000204670BD2DE9F041B0F8143100F5827230
:1030F00000210520FFF72AFF03281CD10A248A4E4D
:10310000744D4FF4FA670D3612E0384602F0B8FA03
:1031100000210620FFF71AFF032809D1D5F8B810BF
:10312000002904DDD5F8B810895D312903D00220CB
:10313000641E611CE9D1BDE8F08100210E2005E785
:1031400070B500F58B72154600210720FFF7FEFED3
:10315000032813D100210820FFF7F8FE0446032CB2
:103160000BD15C48D0F8F000002805DD29466E48F8
:1031700000F03CFC002800DC0224204670BD10B5A5
:103180000C46024600210920FFF7E0FE032801D08B
:10319000022010BD2146644800F028FC002801DD13
:1031A000032010BD042010BD1CB500210091019129
:1031B00002460A20FFF7CAFE032801D000201CBDEA
:1031C0004448D0F82811584806230D3001440D22F8
:1031D000684600F02EFB684605F0BEFA1CBD0B46A3
:1031E000024600210D20B1E62DE9F84F83468A46BC
:1031F00017464FF0FF3844460025DFF8B091012014
:1032000089F80000FEF7AAFE324E0097D6F8381172
:1032100053465A46022000F0D1FE21E0C82002F0B9
:103220002FFA63A1644800F0E1FB00F10904D6F82D
:103230004011614A3819104400F0D8FBC6F8440127
:10324000D6F8440140B1D6F848115B4800F0CEFBF7
:10325000002805DB44460AE0002C08DA444606E074
:1032600028466D1CB6F83C11EDB28842D6D300203A
:1032700089F800002046BDE8F88F0F2827D2DFE844
:1032800000F0080A0C0E10121416181A1C1E202228
:1032900024004AA070474DA070474FA0704751A02E
:1032A000704754A0704757A0704759A070475CA062
:1032B00070475FA0704762A0704765A0704767A025
:1032C000704769A070476CA070476EA0704770A0EF
:1032D000704700004004002046545020636D645045
:1032E00061636B20D2E7B3F6A3A12D2DD4F6BCD336
:1032F0004654505F434D445041434B5F4C454ECA8A
:10330000FDD6B5A1A30000004543323020467470BD
:10331000436D645061636B20C4DAB4E6B7D6C5E48C
:10332000CAA7B0DC210000009A100020496E50614D
:1033300072616D45727200004F7574506172616DFB
:103340004572720052554E455252000052554E4F32
:103350004B00000054494D454F555400CEB4D6AAF9
:10336000B4EDCEF30000000025732025730D0A5B39
:1033700025735D00C5E4D6C3465450B7FECEF1C6F2
:10338000F7557365726E616D653A25732C20506137
:103390007373776F72643A2573202E00465450B1D0
:1033A000BEB5D84950A3BA2573000000B40100206F
:1033B000434F4E4E454354001A1300205345544387
:1033C0004F4E544558544944000000005345544161
:1033D00043434F554E54000053455446494C4554C1
:1033E000595045005345545452414E534D4F444556
:1033F00000000000534554525354494D454F555415
:10340000000000004654504C4F47494E0000000059
:103410004745544C4F47494E5354415445000000D2
:103420005345544449524543544F525900000000FB
:103430004745544449524543544F525900000000F7
:103440004C49535446494C454E414D4500000000FF
:1034500047455446494C4553495A4500444F574EF9
:1034600046494C4500000000474554484153444FED
:10347000574E53495A45000052454E414D45464925
:103480004C4500004654504C4F474F5554000000E7
:10349000CEDEB4CBC3FCC1EE0000000070B5064622
:1034A0003146002000F0AEFB0446002000F017FB80
:1034B00005464B2D08D918225AA161A004F0CEFE72
:1034C000294663A004F0CAFE24B13146204605F027
:1034D00013FA1BE0202253A159A004F0BFFE294695
:1034E00063A004F0BBFE002000F0E0FA31460020AB
:1034F00000F088FB04464CB925224AA150A004F0F4
:10350000ADFE68A004F0AAFE04F06AFC204670BD7F
:103510000146002000F06DBB0FB4F8B507AD009573
:103520004FF480742046FFF7B9FF06465EA221469D
:10353000304604F09FFE0446C4F5807130192B46D6
:10354000069A04F071FE002806DD204482B231465E
:10355000002000F0EAFC07E0502232A138A004F07D
:103560007DFE50A004F07AFE3046FFF7D1FFF8BC94
:103570005DF814FB0FB4F8B507AD00954FF48074F7
:103580002046FFF78BFF064649A22146304604F04D
:1035900071FE0446C4F5807130192B46069A04F07A
:1035A00043FE002806DD204482B23146002000F0B0
:1035B000BCFC07E06E221BA121A004F04FFE39A045
:1035C00004F04CFE3046FFF7A3FFD0E70FB4F8B588
:1035D00007AD00954FF480742046FFF75FFF064665
:1035E00035A22146304604F045FE0446C4F58071FC
:1035F00030192B46069A04F017FE002806DD2044F9
:1036000082B23146002000F090FC07E08B2205A139
:103610000BA004F023FE23A004F020FE3046FFF7A9
:1036200077FFA4E72E2E5C53595354454D5C5359F4
:1036300053504F52545C737973706F72742E6300E1
:103640004C6F674572723A2025732C256400000088
:103650000D0AB6AFCCACC4DAB4E6D5BCD3C3D2D174
:10366000B3ACB9FDA3BA25642525A3A10D0A0000BA
:103670000D0AC4DAB4E6D5BCD3C3A3BA25642525A4
:103680002D2DB6AFCCACC4DAB4E6D2E7B3F6A3A125
:10369000B3F5CABCBBAFB6AFCCACC4DAB4E6BFD5E9
:1036A000BCE4A3A1000000004C6F674170703A00B9
:1036B0004C6F674465623A004C6F674572723A001E
:1036C00000210180418081804FF40061801D05F060
:1036D00013B92DE9F0418388161D33444FF4006778
:1036E000BB4202D30120BDE8F08145881223841D2E
:1036F0002B5543885B1CC3F30A034380458834235E
:103700002B5543885B1CC3F30A03438000230BE063
:1037100011F8015BB0F802C00CF8045045886D1C2C
:10372000C5F30A0545805B1C9342F1DB42885621B4
:1037300011554188491CC1F30A0141804288782112
:1037400011554188491CC1F30A01418081883144E7
:1037500081808188B94209D3FFF7B2FF4322BFA11C
:10376000C5A004F07BFDC8A004F078FD0020BAE7F6
:1037700070B58388002B08D003889B1CC3F30A0311
:10378000038000231380831D21E0022070BD148874
:10379000641C14800488E45C01F8014B0488641CF8
:1037A000C4F30A04048014888588AC4203D20488D8
:1037B000B4F5006F0BD3FFF783FF6622A7A1AEA07D
:1037C00004F04CFDB0A004F049FD022070BD048857
:1037D000E45C562CDBD10488641CC4F30A04044462
:1037E000A479782CD3D10188891CC1F30A01018006
:1037F00081881288891A091F8180002070BD2DE9F7
:10380000F04105460C461746284604F0FDFF0646E3
:10381000384604F0F9FF3118A14204DB00212A19CF
:10382000101A00F8011C39462846BDE8F04105F0A1
:103830000AB830B5054600205B1E04E02C549842BF
:1038400004DA401C80B20C5C9442F7D130BD70B5F4
:103850000446084611461D46049E04F08AFF0246AF
:10386000012006E0231803F8011CB04204D8401CD4
:1038700080B2115CA942F5D170BD30B5002311446E
:10388000491E18E00C7824090A2C01D2302500E0EA
:1038900037252C4400F813400C7804F00F040A2C50
:1038A00001D2302500E037252C4400EB43056C7035
:1038B0005B1C9BB2491E9342E4D330BD30B500235C
:1038C0001AE0CD5C2C0905F00F053034392C03D9F2
:1038D000E41D00F8134001E000F813403035ECB26D
:1038E000392C04D900EB4305E41D6C7002E000EBB9
:1038F00043056C705B1C9BB29342E2D330BDF0B5C4
:1039000003460025084600260A2A01D00670F0BDAD
:10391000002B1DD005DA4FF02D0200F8012BC3F16A
:10392000000342F210724FF00A0793FBF2F454EADC
:10393000050C06D004F1300500F8015B04FB1233DE
:10394000012592FBF7F2002AEFDC06700846F0BD75
:103950003022027046700846F0BDF0B505460023DF
:10396000002042F210720A26B5FBF2F4E4B254EAE7
:10397000000704D030340746401CC0B2CC55B5FB1C
:10398000F2F402FB1455B2FBF6F25B1CDBB2052B22
:10399000EAD308B9302008700846F0BD2DE9F0419F
:1039A00005460C46284604F02FFF80B2002100B1E6
:1039B00021700122002312E0AE5CEF5CBE420CD10C
:1039C000521C92B25B1C9BB2AE5CEF5CBE4201D05B
:1039D000A35404E0E65CA65401E01BB1E35C824220
:1039E000EAD380E6521C92B2A154F8E72DE9F047E1
:1039F00082468946504604F007FF87B2484604F0E5
:103A000003FF86B2002500243046FFF747FD8046BD
:103A100041464846FFF7C2FF0DE01AF8050019F8C5
:103A20000410884204D16D1CADB2641CA4B202E043
:103A30006CB118F80440BD4201D2B442EDD3404607
:103A4000FFF766FDB44205D3A81BBDE8F0876D1CE7
:103A5000ADB2F0E74FF0FF30F7E700002E2E5C53D9
:103A6000595354454D5C5359534C49425C737973D7
:103A70006C69622E630000004C6F674572723A20D9
:103A800025732C25640000000000000003E011F8FD
:103A9000013B00F8013B521E531CF8D1704701E076
:103AA00000F8011B521E531CFAD1704770B5044632
:103AB0006B486C4E002150F8240006EB8405420050
:103AC0002869FFF7ECFF66480021103050F82420E9
:103AD000A868FFF7E4FF01203119087670BD10B522
:103AE000002200215E4B5F4C53F8203004EB800035
:103AF00005E0046934F8114004B1521C491C8B42A2
:103B0000F7D864204243B2FBF3F0C0B210BD2DE9F8
:103B1000F04105460F460024DFF8488108EB050018
:103B2000007E002803D1D8F80010284688474FF0BF
:103B3000FF32FFB14A4E083656F82500B7FBF0F3C6
:103B4000B7FBF0F100FB117000B15B1C444850F86A
:103B50002510491E002921DB08EB8507386930F85C
:103B600011C0BCF1000F08D000249C4213D10022E8
:103B700098B20AE01046BDE8F081641CF5E73C69A4
:103B800001EB020C24F81C00521C9A42F7D356F8A1
:103B900025004843EFE7491E0029E0DA1046EAE72E
:103BA00070B5304A13181B7E002B13D02C4B1033EA
:103BB00053F820308B421AD9294B083353F8203060
:103BC000B1FBF3F102EB8002106930F811300020F4
:103BD000002408E011688847012070BD15690E189F
:103BE00025F81640401C9842F8DB002070BD0220EA
:103BF00070BD002905D01B4A02EB80029268891A29
:103C0000CEE7704710B504462046FFF780FF411C01
:103C100005D0144901EB84018968084410BD0020D7
:103C200010BD2DE9F0410646884617463946304614
:103C3000FFF76DFF0446601C0FD00A483A4600EBC0
:103C400086054146A8682044FFF720FF41463046DC
:103C5000FFF7CFFFA86820448DE700208BE7000026
:103C600060C50008E405002010B50C46F24A52F881
:103C70002030002B09D05222F0A1F6A004F0EEFA79
:103C8000F8A004F0EBFA204610BD42F82040FAE715
:103C900030B40C46E84951F82030002B03D02046C0
:103CA00030BC1146184730BC704770477047F44924
:103CB000C2B20B689A8009680A885206FCD5704720
:103CC0002DE9F04387B004460D461646984601217B
:103CD000084602F01CFBEA4818220F38015D401F1D
:103CE000005D00F013FFE6480422401F015D401F05
:103CF000005D00F00BFFE348002C7CD050F824005E
:103D0000012102F00FFB02950025ADF80C50ADF833
:103D10000E50ADF81050ADF81450ADF81260D84EFA
:103D200002A956F8240002F091FB56F824004FF443
:103D3000587102F0DBFCBDF8120006F1140900070F
:103D400022D5042C20D056F824000122802102F034
:103D50001FFCCC4F00950195183F59F82410385D91
:103D60001023002200F02BFC06F12400002150F863
:103D70002420385D00F01CFBAF480121303850F89A
:103D80002420385D00F014FBBDF81200400759D51F
:103D9000BC481038005D8DF818008DF819808DF83A
:103DA0001A5001208DF81B0006A801F0EAFF56F812
:103DB0002400012240F2244102F0CFFB042C3BD02E
:103DC00056F824000122402102F0E2FBCDE9005820
:103DD000AC4859F824101430A0F1280550F82420DC
:103DE000285D002300F0EBFB05F10A00A64F30F838
:103DF0001410285D00E01AE057F8200003F080FF5F
:103E00008D480021203850F82420285D00F0D0FA99
:103E100089480121103850F82420285D00F0C8FAA4
:103E2000285D012157F8200003F053FF0AE00068E5
:103E3000012102F06CFA66E7012240F22551306957
:103E400002F08BFB56F82400012102F07AFB07B048
:103E5000BDE8F0831CB5044689480122802150F852
:103E6000240002F095FB06200021CDE900108448D3
:103E700010231430002250F8241082481838005DB6
:103E800000F09DFB1CBD7CB504467D48012240210D
:103E900050F8240002F07CFB06200021CDE9001040
:103EA0007848784D1430143D50F82420744800238D
:103EB000143050F82410285D00F081FB05F10A0051
:103EC000714E30F81410285D56F8200003F018FFEA
:103ED000285D012156F82000BDE87C4003F0F9BEC2
:103EE0002DE9F0410446674D674E143D0021285DE1
:103EF00056F8200003F0EDFE05F10A0705F1280051
:103F000037F8141050F8240004F0F6FC285D37F858
:103F1000141056F8200003F0F3FE285D012156F836
:103F20002000BDE8F04103F0D4BE2DE9F04704467F
:103F300088461646B8F1000F25D0002E23D0042C59
:103F400023D0504FDFF84091183F0021385D59F8D9
:103F5000200003F0BEFE4A4D0020183D2855385D74
:103F600059F82000C0F80C80385D314659F820001F
:103F700003F0C6FE385D012159F8200003F0A9FEC8
:103F8000285D0028FCD0BDE8F08700253C4F40218B
:103F9000386902F0A4FB0EE018F8051057F8240069
:103FA00002F030FB57F82400402102F098FB002873
:103FB000F8D06D1CADB2B542EED3E4E70FB470B5E6
:103FC00086B004460CA801902D4E10E05C2916D056
:103FD00025295BD0401C0B9056F8240002F012FB00
:103FE00056F82400402102F07AFB0028F8D00B9804
:103FF00001780029EAD106B070BC5DF814FB401CC2
:104000000B9001786E290DD0722902D0401C0B90C4
:10401000E6E756F824000D2102F0F4FA0B98401C54
:104020000B90DDE756F824000A2102F0EBFA0B981A
:10403000401C0B90D4E70000305B00202E2E5C5318
:10404000595354454D5C55534152545C75736172DC
:10405000742E63004C6F674572723A2025732C25CD
:1040600064000000556172742043616C6C6261638E
:104070006B207265706561742072656721000000B5
:104080001C06002090C5000854060020401C0B9020
:10409000017864291BD0732902D0401C0B909FE744
:1040A000019820C801900BE056F8240002F0AAFA0B
:1040B00056F82400402102F012FB0028F8D06D1CB5
:1040C00029780029F0D10B98401C0B9088E70198C3
:1040D00001990068091D01910A2202A9FFF70FFC4E
:1040E00002AD0BE056F8240002F08CFA56F82400DA
:1040F000402102F0F4FA0028F8D06D1C297800293C
:10410000F0D10B98401C0B906AE770B59C4C40F2C4
:104110002441204602F0EEFAA0B19A4D0021286910
:1041200003F0D7FD2088201D0088286903F0EAFDF0
:10413000C0F5807082B294490020FFF7A9FD0020ED
:10414000FFF7CEFE40F225552946204602F0D2FA6E
:1041500018B12946204602F0EDFA40F227752946AB
:10416000204602F0C7FA002806D029462046BDE8BE
:104170007040002202F0F1B970BD70B5834C40F27E
:104180002441204602F0B6FAA0B17E4D00216869B4
:1041900003F09FFD2088201D0088686903F0B2FDB0
:1041A000C0F5807082B27A490120FFF771FD0120CD
:1041B000FFF796FE40F225552946204602F09AFA6E
:1041C00018B12946204602F0B5FA40F22775294673
:1041D000204602F08FFA002806D029462046BDE886
:1041E0007040002202F0B9B970BD70B5694C40F260
:1041F0002441204602F07EFAA0B1624D0021A86859
:1042000003F067FD2088201D0088A86803F07AFD70
:10421000C0F5406082B260490220FFF739FD0220FC
:10422000FFF75EFE40F225552946204602F062FA6D
:1042300018B12946204602F07DFA40F2277529463A
:10424000204602F057FA002806D029462046BDE84D
:104250007040002202F081B970BD70B54F4C40F241
:104260002441204602F046FAA0B1464D0021686A7A
:1042700003F02FFD2088201D0088686A03F042FDAE
:10428000C0F5807082B246490320FFF701FD03208C
:10429000FFF726FE40F225552946204602F02AFA6D
:1042A00018B12946204602F045FA40F22775294602
:1042B000204602F01FFA20B100222946204602F0D3
:1042C0004CF92046BDE87040402102F00FBA2DE9BC
:1042D000F041344D40F22551284602F00BFA324CA1
:1042E000002658B1AA882168481C20602F484254F3
:1042F000216846542068FF2800DB266040F22447EE
:104300003946284602F0F6F988B12888A88820683E
:10431000264982B20420FFF7BBFC4FF4807123488A
:1043200004F00CFB26603946284602F003FA40F2FE
:1043300027742146284602F0DDF9002806D02146E0
:104340002846BDE8F041002202F007B9BDE8F0813F
:1043500015490120091D0870704713490120091DE6
:104360004870704710490120091D887070470E4938
:104370000120091DC870704770477047704770472B
:104380000038014054060020445B002000440040F7
:10439000445C002000480040445D0020004C004088
:1043A000446900200050004000060020446A0020BC
:1043B00010B5144600290BD0012919D04E22E9A1CD
:1043C000EDA003F04BFFF0A003F048FF204610BD26
:1043D000F64951F8202042B14322E2A1E6A003F0C1
:1043E0003DFFF3A003F03AFFF0E741F82040EDE78E
:1043F000EE49303151F8202042B14A22D9A1DEA045
:1044000003F02CFFF1A003F029FFDFE741F8204083
:10441000DCE730B4E549B0F1007F01F1300271D042
:1044200036DCB0F5005F6ED018DC80287AD00ADC6C
:1044300002286DD0082870D0202868D1486800284C
:1044400065D030BC0047B0F5007F71D0B0F5006F8B
:104450005DD1906800285AD030BC0047B0F5002FDD
:1044600077D00ADCB0F5004F6ED0B0F5003F4ED1EA
:10447000086900284BD030BC0047B0F5001F6DD054
:10448000B0F5000F43D15069002840D030BC004740
:10449000D54C031BA0427CD01ADCD44CA0EB040307
:1044A000A0426CD00BDCB0F1006F61D0A0F1805065
:1044B000801E2CD1C86900287FD030BC0047182B43
:1044C00062D0782B79D1106A002876D030BC0047B2
:1044D000B3F5FC4F67D00ADCB3F5C06F5ED0B3F51F
:1044E000F05F6AD1886A002867D030BC0047B3F516
:1044F000FF3F5DD0BE48C3425FD1D06A00285CD088
:1045000030BC00472FE018E00CE001E005E054E08B
:104510000868002851D030BC0047106800284CD0F3
:1045200030BC00475068002847D030BC0047FFE748
:104530008868002841D030BC0047C86800283CD0BB
:1045400030BC004705E0FFE7D068002835D030BC1C
:1045500000471069002830D030BC00474869002867
:104560002BD030BC00478869002826D030BC0047DB
:104570009069002821D030BC00470AE0FFE7D069ED
:1045800000281AD030BC0047086A002815D030BC7B
:104590000047486A002810D030BC0047506A002805
:1045A0000BD030BC0047906A002806D030BC0047D2
:1045B000C86A002801D030BC004730BC70472DE9E4
:1045C000F0478CB00446DDE914980D4617469A462C
:1045D000072C04D20121084601F08EFE03E00121E0
:1045E000022001F089FE834E56F8240003F0D0FA31
:1045F00001950297CDF80CA0002504950595802023
:10460000069007950895CDF8249040010A900B95E7
:1046100056F8240001A903F032FB774810F8240073
:104620008DF800008DF801808DF8025001208DF882
:104630000300684601F0A5FB56F824000122022180
:1046400003F054FB0CB0BDE8F08710B5022003F076
:104650005CFB012805D1022003F07FFB0220FFF75D
:10466000D8FE082003F051FB01280ED1082003F0EA
:1046700074FBD5223BA140A003F0F0FD5FA003F046
:10468000EDFDBDE810400820C3E610BD10B52020A8
:1046900003F03BFB012805D1202003F05EFB202026
:1046A000FFF7B7FE802003F030FB01280ED18020F9
:1046B00003F053FBEB222BA12FA003F0CFFD52A060
:1046C00003F0CCFDBDE810408020A2E610BD10B57F
:1046D0004FF40074204603F018FB012805D1204652
:1046E00003F03BFB2046FFF794FE4FF400642046A6
:1046F00003F00BFB01280FD1204603F02EFB40F204
:10470000011218A11CA003F0A9FD42A003F0A6FD10
:104710002046BDE810407CE610BD10B54FF40054B3
:10472000204603F0F2FA012805D1204603F015FBDC
:104730002046FFF76EFE4FF40044204603F0E5FAF2
:10474000012874D1204603F008FB40F2171205A19E
:1047500009A003F083FD32A003F080FD2046BDE8F0
:10476000104056E62E2E5C53595354454D5C444D33
:10477000415C646D612E63004C6F674572723A2034
:1047800025732C2564000000446D6154652043614D
:104790006C6C6261636B202265497271547970653B
:1047A00022206572726F722100000000446B0020AD
:1047B000446D6154632043616C6C6261636B207271
:1047C000657065617420726567210000446D6154F5
:1047D000652043616C6C6261636B2072657065611A
:1047E00074207265672100000002001008000010AC
:1047F0000002F8FF54060020B4C50008444D4131C2
:104800005F54453121000000444D41315F54453231
:1048100021000000444D41315F5445332100000028
:10482000444D41315F54453421000000FFE710BD85
:1048300010B54FF40034204603F067FA012805D183
:10484000204603F08AFA2046FFF7E3FD4FF40024E8
:10485000204603F05AFA012811D1204603F07DFAD0
:1048600040F22D12AFF20411AFF2F40003F0F6FCA7
:104870008AA003F0F3FC2046BDE81040C9E510BD56
:1048800010B54FF40014204603F03FFA012805D17B
:10489000204603F062FA2046FFF7BBFD4FF4000408
:1048A000204603F032FA012811D1204603F055FAD0
:1048B00040F24312AFF25411AFF2441003F0CEFCB9
:1048C00079A003F0CBFC2046BDE81040A1E510BD67
:1048D00010B54FF00074204603F017FA012805D1F7
:1048E000204603F03AFA2046FFF793FD4FF00064AC
:1048F000204603F00AFA012811D1204603F02DFAD0
:1049000040F25912AFF2A411AFF2941003F0A6FCDA
:1049100068A003F0A3FC2046BDE8104079E510BD77
:1049200010B5674C204603F0F0F9012805D1204668
:1049300003F013FA2046FFF76CFD614CA41D2046DE
:1049400003F0E3F9012811D1204603F006FA40F202
:104950006F12AFF2F011AFF2E01003F07FFC59A03C
:1049600003F07CFC2046BDE8104052E510BD10B5B8
:10497000534C1E34204603F0C8F9012805D12046C7
:1049800003F0EBF92046FFF744FD4D4C7E34204602
:1049900003F0BBF9012811D1204603F0DEF940F203
:1049A0008512AFF24021AFF2302003F057FC45A052
:1049B00003F054FC2046BDE810402AE510BD10B5B8
:1049C000434C204603F0A1F9012805D1204603F00D
:1049D000C4F92046FFF71DFD3E4C204603F095F933
:1049E000012811D1204603F0B8F940F29B12AFF232
:1049F0008C21AFF27C2003F031FC37A003F02EFCB9
:104A00002046BDE8104004E510BD10B5354C2046E9
:104A100003F07BF9012805D1204603F09EF92046DA
:104A2000FFF7F7FC304C204603F06FF9012810D156
:104A3000204603F092F940F2B112AFF2D821AFF262
:104A4000C82003F00BFC29A003F008FC2046FFF768
:104A5000E0FC294C204603F058F9012805D12046F6
:104A600003F07BF92046FFF7D4FC244C204603F0EA
:104A70004CF9012811D1204603F06FF94FF4DF7291
:104A8000AFF22031AFF2103003F0E8FB1CA003F0CE
:104A9000E5FB2046BDE81040BBE410BD444D41316C
:104AA0005F54453521000000444D41315F54453687
:104AB00021000000444D41315F5445372100000082
:104AC00002000010444D41325F5445322100000085
:104AD0000002001000080010444D41325F5445337D
:104AE000210000000020001000800010444D4132E1
:104AF0005F5445342100000000000210000008103F
:104B0000444D41325F54453521000000F8B504465C
:104B10000D4616469848012150F8240001F0F7FB95
:104B200095481C3030F81500ADF800008DF8036092
:104B300003208DF802009148694650F8240001F0E6
:104B4000E0F9F8BD2DE9FE430646DDF828900C4655
:104B5000154698462A4621463046FFF7D7FF282DAE
:104B600001D0482D36D10121084601F0D0FB824FFB
:104B70008C37385D8DF800008DF8019000258DF898
:104B800002508DF80350684601F0FBF8A7F1500081
:104B9000015D4438805D01F070FAA7F1400656F8D7
:104BA000240001908DF808508DF8098001258DF8BA
:104BB0000A5001A801F04AFE56F8240001F0A5FEB3
:104BC000385700F01F018D404009800000F1E020BF
:104BD000C0F80051BDE8FE83684A52F82000C26860
:104BE000654B1C3333F811104A40C260704710B552
:104BF0000C46634A52F82030002B09D0952261A15F
:104C000065A003F02BFB68A003F028FB204610BD35
:104C100042F82040FAE770B5064600204FF0804188
:104C200005F024FA04460D46304605F0BDFE05F0B9
:104C30001DFA22462B4605F0AFFC05F041FE504917
:104C400051F82000002802D0BDE87040004770BD38
:104C500010B5012001F03EFE28B1012001F043FE15
:104C60000120FFF7D8FFBDE81040012001F04DBE44
:104C700010B5022001F02EFE012805D1022001F01E
:104C800032FE0220FFF7C7FFBDE81040022001F00E
:104C90003CBE10B5042001F01DFE28B1042001F037
:104CA00022FE0420FFF7B7FFBDE81040042001F00A
:104CB0002CBE10B5082001F00DFE012805D10820FA
:104CC00001F011FE0820FFF7A6FFBDE81040082004
:104CD00001F01BBE10B5102001F0FCFD28B1102022
:104CE00001F001FE1020FFF796FFBDE810401020F4
:104CF00001F00BBE30B591B005241F4D4C3555F871
:104D0000240001F0F4FD88B155F8240001F0EBFD1A
:104D1000402101A803F012FE234629A2402101A848
:104D200003F0A8FA55F82400FFF775FF641C092C5E
:104D3000E5DD11B030BD30B591B00A240E4D4C35D3
:104D400055F8240001F0D3FD88B155F8240001F096
:104D5000CAFD402101A803F0F1FD234618A240211D
:104D600001A803F087FA55F82400FFF754FF641CEC
:104D70000F2CE5DDDDE70000ECC50008840600200F
:104D8000A46B00202E2E5C53595354454D5C494F63
:104D90005C696F2E630000004C6F674572723A20A9
:104DA00025732C2564000000494F2043616C6C6220
:104DB00061636B20726570656174207265672100A4
:104DC0004558544925642049525121000021016071
:104DD0004160018181720B2210A103F0D6BD0EB596
:104DE000114A12680092104A121D126801920E4A6E
:104DF00008321268029200290BD0012904D00C223B
:104E00006946FEF75BFD0EBD0C226946FEF756FDB6
:104E10000EBD0C22694603F0B8FD0EBD4A616E203E
:104E20003231203230323100E8F7FF1F10B50C4626
:104E3000F54901280BD0022816D03D22F3A1F8A095
:104E400003F00CFAFAA003F009FA204610BD4868F6
:104E500040B13222EDA1F2A003F000FAFBA003F072
:104E6000FDF9F2E74C60F0E7886840B13922E7A12C
:104E7000EBA003F0F3F9FDA003F0F0F9E5E78C6097
:104E8000E3E7E149012805D0022807D18868002816
:104E900004D000474868002800D00047704710B58C
:104EA000012001F0F2FD38B1012001F0FCFD01F01C
:104EB000CDFD0120FFF7E5FF022001F0E6FD00280F
:104EC00008D0022001F0EFFD01F0C0FDBDE8104068
:104ED0000220D6E710BD10B5022001F0D6FD002853
:104EE0000CD04FF4003001F010FD022001F0DBFD8A
:104EF00001F0ACFDBDE810400220C2E710BD30B5A6
:104F00006423B0FBF3F4E4B2B0FBF3F503FB15004C
:104F1000132C01D96430C0B200EB90030724B3FB1B
:104F2000F4F504FB1533D94D1A440D4415F8015C12
:104F30002A4492B2800703D1032901D2521E92B2B1
:104F4000B2FBF4F004FB102030BD810701D000203B
:104F500070476421B0FBF1F201FB120109B101209D
:104F600070474FF4C871B0FBF1F201FB120008B1B9
:104F700000207047012070472DE9F04788B00446B3
:104F800001F06AFD01F039FD0646DFF80483B6FB47
:104F9000F8F39D480A270188994279D0038040F2AE
:104FA000B2754FF4B7794FF4B67A0FE02846FFF7A1
:104FB000CCFF38B14B4502D3A3F5B77304E06D1CA9
:104FC000ADB205E0A3F26D136D1CADB25345EDD843
:104FD0000195BDF804104FF47A70B1FBF0F1303157
:104FE0002170BDF80410B1FBF0F200FB1212642135
:104FF000B2FBF1F230326270BDF80420B2FBF0F582
:1050000000FB1520B0FBF1F201FB1200B0FBF7F042
:105010003030A070BDF80400B0FBF7F107FB1100C1
:105020003030E0700025DFF8649209F10C090DE0E2
:10503000BDF80400FFF789FF08B1012D7AD019F8F7
:105040000500984204D81B1A6D1CADB21C2BEFD280
:105050006D1C04955B1C03939DF81000B0FBF7F0EA
:10506000303060719DF81000B0FBF7F107FB1100C4
:105070003030A0719DF80C00B0FBF7F0303020729A
:105080009DF80C00B0FBF7F107FB110030306072A7
:10509000B6FBF8F008FB10604FF46161B0FBF1F271
:1050A0000792B0FBF1F201FB12033C22B3FBF2F3D7
:1050B0000693B0FBF1F301FB1300B0FBF2F102FB2E
:1050C000110005909DF81C00B0FBF7F03030E07245
:1050D0009DF81C00B0FBF7F107FB11003030207386
:1050E0009DF81800B0FBF7F03030A0739DF8180061
:1050F000B0FBF7F107FB11003030E0739DF81400AE
:10510000B0FBF7F0303060749DF81400B0FBF7F19D
:1051100007FB11003030A0749DF80C209DF8101092
:10512000BDF80400FFF7EBFE029008B00320BDE8D5
:10513000F087FFE71D2B8BD31D3B85E755481BE709
:1051400008B503218DF800108DF8010000208DF8BE
:10515000020001208DF80300684600F012FE08BD31
:105160002DE9F041074600244A48202181722D2173
:10517000C17101713A210174417301214FF0C05096
:1051800001F0D0F80121084601F0C1F8012001F03A
:10519000D1FB042001F028FB45F25006B04232D08A
:1051A00001F0F8FA012001F03CF801F018FC01F0E0
:1051B0004DFC6FF07F4500E0641C412000F0B6FF1D
:1051C00008B9AC42F8D3DFF8D080444505D24FF49B
:1051D000807001F03BF8012466E00024012001F01A
:1051E00032F800E0641C612000F0A0FF08B9AC4276
:1051F000F8D3444570D24FF4007001F027F8CA226A
:1052000002A107A04AE079E0A00600202E2E5C5300
:10521000595354454D5C5254435C7274632E630081
:105220004C6F674572723A2025732C25640000008C
:105230005274635F526567486F6F6B43616C6C6259
:1052400061636B204661696C656421005274632060
:1052500053656354692043616C6C6261636B2072B7
:105260006570656174207265672100005274632067
:10527000416C7254692043616C6C6261636B207293
:1052800065706561742072656721000088C600083A
:1052900080510100E46B0020F0FFFF0002F0DEFF10
:1052A000C9A002F0DBFF0024012000F0D4FF01F0D0
:1052B000CDFBF4B147F6FF7001F0AFFB01F0C6FB88
:1052C00001F0C4FB01F092FB01F0C0FB3146042069
:1052D00001F082FA18E0FFE7CF22AFF2D001AFF27F
:1052E000C00002F0BBFFB8A002F0B8FF0220BDE88A
:1052F000F08149F6404001F090FBDFE701F0A6FBAA
:105300000121084601F060FB01F0A0FB01210846E5
:1053100001F05AFB01F09AFB0121022001F054FB3D
:1053200001F094FB002001F005FB3846FFF708FF71
:10533000A648FFF721FEAFF2FB110120FFF776FD33
:105340000320D4E72DE9F05F00230178C2783039DB
:1053500001EB4104C4EBC11102EBC10442786421AA
:10536000303A4A438178303901EB810102EB410147
:10537000214430398DB241798279303901EB810491
:105380006FF02F0101EB44042244D7B2027A447A31
:10539000303A02EB820201EB42022244D6B2C27AD8
:1053A000047B303A02EB820201EB4202224402F01B
:1053B000FF08827BC47B303A02EB820201EB42029F
:1053C000224402F0FF09827C407C303800EB8000F0
:1053D00001EB4000104400F0FF0AA5F2B2708228F1
:1053E00002D30220BDE8F09F40F2B274DFF8E0B1D2
:1053F00009E02046FFF7A9FD08B15B4401E07548CC
:105400000344641CA4B2AC42F3D37F1EFFB2002459
:10541000DFF8C4B110E01BF8040040F2A3214843B8
:1054200003EBC0132846FFF790FD18B1012C01D102
:105430006A480344641CA4B2BC42ECD3761E40F21A
:10544000A320464303EBC610C8EB4811C1EB08216B
:1054500000EB0110C9EB091100EB810000EB0A041D
:10546000012001F067FA01F0BAFA01F0EFFA2046E4
:1054700001F0CCFA01F0EAFA01F0B8FA01F0E6FA2C
:105480000320AFE72DE9F05F00230178C2783039BF
:1054900001EB4104C4EBC11102EBC1044278642169
:1054A000303A4A438178303901EB810102EB410106
:1054B000214430398DB241798279303901EB810450
:1054C0006FF02F0101EB44042244D7B2027A447AF0
:1054D000303A02EB820201EB42022244D6B2C27A97
:1054E000047B303A02EB820201EB4202224402F0DA
:1054F000FF08827BC47B303A02EB820201EB42025E
:10550000224402F0FF09827C407C303800EB8000AE
:1055100001EB4000104400F0FF0AA5F2B2708228AF
:1055200001D302205EE740F2B274DFF8A4B009E0D4
:105530002046FFF70AFD08B15B4401E0254803441B
:10554000641CA4B2AC42F3D37F1EFFB20024DFF888
:1055500088B010E01BF8040040F2A321484303EB9D
:10556000C0132846FFF7F1FC18B1012C01D11B48EC
:105570000344641CA4B2BC42ECD3761E40F2A320C8
:10558000464303EBC610C8EB4811C1EB082100EB02
:105590000110C9EB091100EB810000EB0A040120A6
:1055A00001F0C8F901F01BFA01F050FA204601F0B1
:1055B0003CFA01F04BFA01F019FA01F047FA002029
:1055C00001F0B8F903200DE700000000E46B0020B3
:1055D0000085E2018033E10194C60008805101009A
:1055E000354840683221B0FBF1F201FB120000287F
:1055F00001D1FBF7FABF704710B5042000F004FC9E
:105600002E482F492C4A0068B0FBF1F31370B0FB11
:10561000F1F142F2107041430A2050804FF0E02037
:10562000026942F0020202614161016941F0010137
:10563000016110BD70B505462248854208D905466E
:10564000502221A127A002F009FE2AA002F006FEA6
:1056500000214FF0E0267469174800784543B3698C
:10566000B2699A42FCD003D2A3EB0200014403E0EA
:10567000A4EB0200184401441346A942F0D370BDC4
:1056800070B5054600244FF47A7605E03046FFF702
:10569000D1FF00F06FF9641CAC42F7D370BD70B558
:1056A000054600244FF47A7603E03046FFF7C2FF48
:1056B000641CAC42F9D370BDAC060020E0060020AB
:1056C00040420F00E3388E032E2E5C53595354454D
:1056D0004D5C5359535449434B5C737973746963FC
:1056E0006B2E63004C6F674572723A2025732C2530
:1056F000640000000000000010B50C467E4A52F81D
:105700002030002B09D034227CA182A002F0A6FD1B
:1057100084A002F0A3FD204610BD42F82040FAE725
:10572000754951F82000002800D0004770472DE946
:10573000FF410446884615461F4641F699108045AC
:1057400008D980465E226DA172A002F087FD75A087
:1057500002F084FD7448012150F8240000F0E2FDBD
:10576000714E083E305D8DF80C008DF80D5000250F
:105770008DF80E508DF80F5003A800F002FB41F693
:105780001F40ADF80000ADF80650ADF8025040469D
:1057900005F00AF9654A664B04F0FEFE0022654BEF
:1057A00005F020FA05F0BCF8ADF804008DF80850BB
:1057B000614D694655F8240001F066FA012255F85A
:1057C0002400114601F04BFD55F82400394601F044
:1057D0002CFD55F82400012101F080FF30570121F4
:1057E00000F01F0291404009800000F1E020C0F865
:1057F0000011BDE8FF81504951F82000002101F05F
:1058000035BF70B504464C4D002155F8240001F019
:105810002DFF55F82400BDE87040012101F005BDC1
:10582000454951F82000002101F0FFBC10B50121CD
:105830008C07204601F046FF012807D101212046B0
:1058400001F04CFFBDE81040002069E710BD10B525
:105850003A4C0121204601F035FF012807D10121F2
:10586000204601F03BFFBDE81040012058E710BD85
:1058700010B5334C0121204601F024FF012807D147
:105880000121204601F02AFFBDE81040022047E731
:1058900010BD10B52B4C0121204601F013FF01284B
:1058A00007D10121204601F019FFBDE81040032077
:1058B00036E710BD10B5244C0121204601F002FF4F
:1058C000012807D10121204601F008FFBDE8104062
:1058D000042025E710BD10B51C4C0121204601F025
:1058E000F1FE012807D10121204601F0F7FEBDE8B5
:1058F0001040052014E710BDF86B00202E2E5C53DD
:10590000595354454D5C54494D45525C74696D651D
:10591000722E63004C6F674572723A2025732C25F6
:105920006400000000000000A8C600089A99999938
:105930009999B93F0000F03FB406002000040040F0
:1059400000080040000C004000100040001400401F
:1059500010B545F2555000F0FFFE062000F0FFFEA6
:1059600040F20D3000F0FEFE00F0FFFEBDE81040FA
:1059700000F000BF00F0F9BE03E010F8013B01F8B1
:10598000013B521E92B2F8D270472DE9F041054614
:105990000E461746002407E0284601F0C3FF26F80C
:1059A0001400AD1C641CA4B2BC42F5D3BDE8F08168
:1059B0002DE9F0410E4617460546002409E036F869
:1059C0001410284601F0B0FF0428EFD1AD1C641C70
:1059D000A4B2BC42F3D3E9E72DE9F04FADF6040DD4
:1059E00082460F461546AAF10064B4F1005F04D365
:1059F00000200DF6040DBDE8F08F212000F096FB8D
:105A0000012809D06B22A3A1A8A002F027FCABA01B
:105A100002F024FC0220ECE701F07DFE4FEAD428DE
:105A2000C4F34906C6F58064A54200D82C460DF1A2
:105A3000040B37E032183BF812208A4203D1401C95
:105A400080B2A042F6D3A04214D2484601F09CFE98
:105A5000002006E0821937F810102BF81210401CB5
:105A600080B2A042F6D348464FF4806201A9FFF706
:105A70009FFF04E0224639465046FFF799FFA542B2
:105A800003D101F054FE0320B3E708F1010800261A
:105A900007EB4407A244281B85B24FF48064A5425B
:105AA00000D82C464FF0006000EBC829421401A931
:105AB0004846FFF76AFF00204FF6FF71C1E72DE966
:105AC000F04107460E46002402F0010000EB5205AB
:105AD000212000F02BFB012809D0A8226DA173A082
:105AE00002F0BCFB75A002F0B9FB02205EE701F0FA
:105AF00012FEA7F10060B0F5002F01D278050BD09F
:105B0000AE2264A169A002F0A9FB6CA002F0A6FB82
:105B100001F00DFE022049E7B5F5006F0BD9B42264
:105B20005CA162A002F09AFB64A002F097FB01F076
:105B3000FEFD02203AE7352002F011F8384601F068
:105B400023FE04281BD0BB2252A158A002F086FBE2
:105B50005AA002F083FB12E00A20FFF791FD0A2C05
:105B60000BD9C2224BA151A002F078FB53A002F046
:105B700075FB01F0D0FD022018E7641CA4B20120DF
:105B800001F0DEFF0128E7D023E0202001F0E7FF4D
:105B900030787178B61C40EA0121384601F0C4FE25
:105BA000002410E00A20FFF76BFD1E2C09D9D32238
:105BB00038A13EA002F052FB40A002F04FFB0220B1
:105BC000F4E6641CA4B2202001F0BAFF0128E9D158
:105BD000BF1C6D1EADB2D8D201F0A9FD0320E5E6D1
:105BE0002DE9F0478146884600260024002702F070
:105BF000010000EB5205212000F098FA01280AD09C
:105C0000F12224A129A002F029FB2CA002F026FBFE
:105C10000220BDE8F08701F07EFD352001F09FFFF6
:105C200012E00A20FFF72CFD0A2C0BD9FB2219A148
:105C30001EA002F013FB21A002F010FB01F06BFD8F
:105C40000220E6E7641CA4B2012001F079FF0128DC
:105C5000E7D018E0202001F082FF701C18F8061031
:105C600080B2421C18F8000096B241EA002A09EB03
:105C70000704600502D1204601F086FD204651460A
:105C800001F052FEBF1C6D1EADB2E3D201F04FFD1C
:105C90000320BEE72E2E5C53595354454D5C464CB1
:105CA0004153485C666C6173682E63004C6F6745B6
:105CB00072723A2025732C25640000000000000059
:105CC000FEB505460E460121084600F020FB4FF4C4
:105CD0008037019700248DF808408DF80950012580
:105CE0008DF80A5001A800F0B1FD384600F00DFE15
:105CF0008DF800508DF801608DF802408DF803405A
:105D0000684600F03EF81B4902200860C02000F001
:105D100017FE012000F011FEFEBD3EB5012108076F
:105D200000F000FB01248DF808408DF809400025A3
:105D30008DF80A508DF80B4002A800F022F8684652
:105D400000F0BBFD200400908DF8045008208DF871
:105D500005008DF80640684600F078FDC02000F090
:105D6000EFFD012000F0E9FD3EBD4FF4803000F072
:105D7000CCBD000000E100E02A4908432A49086040
:105D8000704770B50F23C27801260178002A1ED013
:105D9000254A126802F4E062C2F5E062120AC2F11A
:105DA0000404D3404578A54082781A402A43120162
:105DB00001F1E02181F80024007800F01F018E40FD
:105DC0004009800000F1E020C0F8006170BD01F0E2
:105DD0001F0086404809800000F1E020C0F8806183
:105DE00070BD124A114001430F48001F0160704707
:105DF0000D4A121D002903D011680143116070473C
:105E000011688143116070474FF0E021042804D0ED
:105E1000086920F0040008617047086940F0040038
:105E2000086170470000FA050CED00E080FFFF1FDD
:105E300010B59C49884209D10121042000F07DFA67
:105E40000021BDE81040042000F077BA964988424E
:105E500009D10121082000F070FA0021BDE81040AE
:105E6000082000F06ABA9149884209D10121102026
:105E700000F063FA0021BDE81040102000F05DBA88
:105E80008B49884209D10121202000F056FA0021D7
:105E9000BDE81040202000F050BA8649884209D160
:105EA0000121402000F049FA0021BDE810404020C7
:105EB00000F043BA8049884209D10121802000F0D6
:105EC0003CFA0021BDE81040802000F036BA7B4942
:105ED00088420AD184150121204600F02EFA20467E
:105EE000BDE81040002100F028BA10BD10B5012116
:105EF000084600F022FA0021BDE81040012000F021
:105F00001CBA2DE9F0410022CC7804F00F03E4061E
:105F100001D58C7823430C784FF00F0714F0FF0F56
:105F20004FF0010C1CD005680CFA02F40E882640D4
:105F3000A64211D1960007FA06F825EA080503FAE9
:105F400006F848EA0505CE78282E02D0482E02D061
:105F500002E0446100E00461521C082AE4D30560B9
:105F60000A88FF2A1ED94568002202F108060CFAA9
:105F700006F40E882640A64210D1960007FA06F8CD
:105F800025EA080503FA06F848EA0505CE78282E22
:105F900000D14461CE78482E00D10461521C082AF9
:105FA000E3D34560BDE8F0814FF6FF710180022127
:105FB00081700421C17070470246002092680A4235
:105FC00000D001207047806880B2704702460020F0
:105FD000D2680A4200D001207047C06880B2704782
:105FE0000161704741617047002A01D0016170472B
:105FF00041617047C160704741F4803282618161C4
:10600000826181698069704710B52D4B1A684FF61F
:106010008074224042EA00100843186010BD2949EC
:10602000C8617047F0B5264C002801DAE36900E04A
:106030006368C0F30346420D120185B2C0F30157F5
:106040009540032F07D0C2020CD50322B2409343E0
:1060500043F0706209E023F07062636823F07063BC
:10606000636002E0AB4343F0706201B12A43002851
:1060700001DAE261F0BD6260F0BD10B58A07120F6F
:106080000F23934021F003040D4921448C689C4365
:106090008C608B68904003438B6010BD0949DC31F4
:1060A0000860704700080140000C014000100140EA
:1060B0000014014000180140001C01400020014074
:1060C0000000014000002042B448016841F0010195
:1060D00001604168B24A114041600168B14A114013
:1060E0000160016821F480210160416821F4FE0112
:1060F00041604FF41F0181607047A8490A6822F48B
:1061000080320A600A6822F480220A60B0F5803F7B
:1061100007D0B0F5802F03D1086840F4A0200860B4
:106120007047086840F480300860704703460020DC
:1061300059099A4A01290AD002290AD0516A03F062
:106140001F02012393400B4200D0012070471168C9
:10615000F5E7116AF3E718B5002000904FF4A0644A
:106160003120FFF7E3FF0099491C00910099A142FB
:1061700001D00028F4D03120FFF7D8FF08B101206A
:1061800018BD002018BD854A116821F0F80141EAC8
:10619000C000106070478449086070477F4B5A68A0
:1061A00022F47C1208431043586070477E49086609
:1061B00070477A4A516821F00301014351607047EA
:1061C0007648406800F00C007047744A516821F02E
:1061D000F001014351607047704A516821F4E06159
:1061E0000143516070476D4A516821F4605141EAA2
:1061F000C00050607047694A002903D0517A0143BA
:1062000051727047517A8143517270476649D83153
:1062100008607047614A516821F440410143516070
:1062200070475E49002220310A7001F820290128B8
:1062300005D0042802D1052081F8200070470120F4
:1062400081F82000704759490860704753490A6A2D
:1062500002430A627047554944390860704710B5D7
:106260004E4A516801F00C01514B002927D00429F6
:1062700027D0082927D00360516801F0F0010909EF
:106280004C4B5C5C0168E1404160546804F4E0649C
:10629000240A1C5D21FA04F48460546804F46054F8
:1062A000E40A1B5DD940C160526802F44042920B7F
:1062B000404B1B1F9A5CB1FBF2F1016110BD036002
:1062C000DAE70360D8E7516801F47011536803F40A
:1062D0008033022404EB914133B153689B0307D50B
:1062E000354B59430160C7E7334B59430160C3E75E
:1062F0002F4B59430160BFE7284A002903D0516959
:106300000143516170475169814351617047234A8C
:10631000002903D0916901439161704791698143DC
:10632000916170471D4A002903D0D1690143D161B1
:106330007047D1698143D1617047184A002903D061
:10634000D1680143D1607047D1688143D160704703
:10635000124A002903D01169014311617047116984
:1063600081431161704711494039086070470E49F7
:10637000C86470470949C87170470848416A41F0CC
:1063800080714162704701460020044A92680A42C7
:1063900000D0012070470149887270470010024008
:1063A0000000FFF8FFFFF6FE000042428004424278
:1063B00000127A00D006002000093D0010B5E14926
:1063C00088420AD101218C032046FFF7B6FF204600
:1063D000BDE810400021FFF7B0BFDB4988420AD179
:1063E00001214C042046FFF7B3FF2046BDE81040D2
:1063F0000021FFF7ADBFD54988420AD101218C04A5
:106400002046FFF7A5FF2046BDE810400021FFF71A
:106410009FBFCF4988420AD10121CC042046FFF713
:1064200097FF2046BDE810400021FFF791BFC94902
:1064300088420AD101210C052046FFF789FF20463A
:10644000BDE810400021FFF783BF10BD30B585B017
:1064500004460D46208A4CF6FF710840E988014346
:106460002182A0894EF6F3110840A9882A89114398
:106470006A8902431143A181A08A4FF6FF41084077
:10648000A9890143A1826846FFF7E9FEAD4884422D
:1064900001D1039800E00298A189090408D500EB16
:1064A000C00101EB001029684900B0FBF1F007E0E2
:1064B00000EBC00101EB001029688900B0FBF1F08E
:1064C0006422B0FBF2F109010B096FF018056B4370
:1064D00000EB8300A3891D044FF0320307D503EBC3
:1064E000C000B0FBF2F000F00700084306E003EB49
:1064F0000010B0FBF2F000F00F000843208105B05F
:1065000030BD4FF41651016000218180C1800181AE
:106510000C2242818181704710B5038A4FF2FF023D
:1065200013400A884C8822438C88C9880C43224334
:106530001A43028210BD0021018041808180C18008
:106540007047002904D0818941F40051818170474E
:10655000818921F400518181704710B540F66A139A
:10656000C1F3421301F01F040121A140012B07D008
:10657000022B07D014303AB102680A43026010BD02
:106580000C30F8E71030F6E702688A43026010BD6D
:10659000002A03D0828A0A4382827047828A8A4311
:1065A00082827047028A22F00F020282028A0A4324
:1065B00002827047828922F40062828182890A43C2
:1065C00082817047002904D0818941F002018181D4
:1065D0007047818921F0020181817047028A22F08F
:1065E00020020282028A0A4302827047002904D0F4
:1065F000018A41F4804101827047018A21F480417F
:1066000001827047C1F30801818070478088C0F320
:1066100008007047818941F0010181817047028B38
:10662000D2B20283028B42EA012101837047028BBE
:1066300002F47F420283028B0A43028370470029DF
:1066400004D0818A41F0200181827047818A21F043
:10665000200181827047002904D0818A41F0100115
:1066600081827047818A21F0100181827047002960
:1066700004D0818A41F0080181827047818A21F02B
:10668000080181827047002904D0818941F40041CA
:10669000818170478189C1F30E0181817047002992
:1066A00004D0818A41F4006181827047818A21F49B
:1066B000006181827047828A22F004028282828A8B
:1066C0000A4382827047002904D0818A41F0020186
:1066D00081827047818A21F00201818270470246DF
:1066E000002012880A4200D0012070478A05C94361
:1066F0000180704770B5002440F66A12C1F342135E
:1067000001F01F05012606FA05F2012B0CD0022B21
:106710000DD0838A1340090A8E40008830400BB1A7
:1067200000B10124204670BD83891340F3E7038A3A
:106730001340F0E740F66A120A0A01219140C9436A
:10674000018070470038014000440040004800408C
:10675000004C0040005000400D49086070470C4953
:10676000486070470A498860704709494AF6AA207C
:106770000860704706494CF6CC40086070470146F7
:106780000020034AD2680A4200D00120704700006E
:106790000030004010B50120FFF7E5FDBDE81040D6
:1067A0000020FFF7E0BD2049086070471E49091F1F
:1067B000086070471C498431086070471B4A118883
:1067C00021F46071014311807047184A118821F04B
:1067D0007F0101431180704708B5144A2C3A1044D8
:1067E00000900098016008BD08B510492C39084494
:1067F00000900098008808BD0B489C300068C0B22B
:1068000070470A480830018841F001010180704753
:106810000548A0300068C0B27047044808300188BD
:1068200041F002010180704704860D422C6C00404B
:10683000384900200860091D0860091D0860091D0D
:1068400008603449344814310860704730B5314A23
:1068500083790168002B2AD013688B431360111DC4
:106860000B680468A3430B60017911440B6804684A
:1068700023430B60274C0834216803689943216047
:10688000231D19680568A94319604179102905D0AD
:1068900011440A68006802430A6030BD216802683A
:1068A00011432160196800680143196030BD007907
:1068B000104402688A43026030BD0021016001710A
:1068C0000C22427181717047124910310A680243EB
:1068D0000A607047014600200E4A143212680A42CC
:1068E00000D0012070470B49143108607047014601
:1068F0000020084A12680A40064B14331B680B42FA
:1069000002D0002A00D001207047024914310860EB
:106910007047000000040140FFFF0F0010B5012187
:106920000C072046FFF714FD2046BDE8104000216B
:10693000FFF70EBD21490862704720490861704782
:106940001F4A116821F0E0010143116070471B49A3
:10695000A031086070471A4B1A6822F00302024304
:106960001A601848026842F004020260012905D04A
:1069700020BF016821F004010160704730BFF8E7D3
:106980000F48016841F004010160016841F0020113
:1069900001600C48016841F00401016030BF70479C
:1069A00001460020064A52680A4200D00120704782
:1069B00003490A6842EA80000860704700000E42FE
:1069C0000070004010ED00E03A4A002903D0118821
:1069D0000143118070471188814311807047354809
:1069E000001D018841F01001018070473148001DF1
:1069F000018821F01001018070472E481C3000886A
:106A00002C491831098840EA01407047294A010C95
:106A100018321180111D08807047264AC0F30341C7
:106A200008321180111D0880E0E7224A010C203253
:106A30001180111D088070471E4810300088000723
:106A4000010B1C4814300088084370471948001D8A
:106A500001888906FCD570471648001D018821F081
:106A60000801018001880907FCD570470146002014
:106A7000104A121D12880A4200D0012070470D49A9
:106A8000091D0A8882430A8070470A49091D09883E
:106A9000C2B21140074A1288024202D009B1012055
:106AA0007047002070470349091D0A8882430A8005
:106AB000704700000028004010B5FE4988420AD106
:106AC000C41401212046FFF738FC2046BDE81040E1
:106AD0000021FFF732BCB0F1804F0CD0F64988425C
:106AE00013D101210220FFF733FC0021BDE8104043
:106AF0000220FFF72DBC01210846FFF729FC0021E9
:106B0000BDE810400120FFF723BCEC49884209D1C1
:106B100001210420FFF71CFC0021BDE810400420E7
:106B2000FFF716BCE649884209D101210820FFF78A
:106B30000FFC0021BDE810400820FFF709BCE14927
:106B4000884209D101211020FFF702FC0021BDE895
:106B500010401020FFF7FCBBDB49884209D101211E
:106B60002020FFF7F5FB0021BDE810402020FFF7B3
:106B7000EFBBD64988420AD1441401212046FFF7D1
:106B8000DCFB2046BDE810400021FFF7D6BBD04912
:106B900088420AD10121CC042046FFF7CEFB2046D3
:106BA000BDE810400021FFF7C8BBCA4988420AD19E
:106BB00001210C052046FFF7C0FB2046BDE8104030
:106BC0000021FFF7BABBC44988420AD101214C0514
:106BD0002046FFF7B2FB2046BDE810400021FFF73A
:106BE000ACBBBE49884209D101214020FFF7B0FB70
:106BF0000021BDE810404020FFF7AABBB8498842F9
:106C000009D101218020FFF7A3FB0021BDE810403E
:106C10008020FFF79DBBB34988420AD1841501212A
:106C20002046FFF795FB2046BDE810400021FFF706
:106C30008FBBAD4988420AD101210C042046FFF7E1
:106C40007CFB2046BDE810400021FFF776BBA7493A
:106C500088420AD101214C042046FFF76EFB2046F2
:106C6000BDE810400021FFF768BBA14988420AD166
:106C700001218C042046FFF760FB2046BDE8104050
:106C80000021FFF75ABB10BD30B50288894C8F4DEB
:106C9000A0420DD0A8420BD0B0F1804F08D0864B57
:106CA000984205D0854B984202D0854B984203D13B
:106CB00022F070034A881A43824B984206D0824BD6
:106CC000984203D022F44073CA881A4302808A880B
:106CD00082850A880285A0420AD0A84208D0824A4A
:106CE000904205D0814A904202D0814A904201D11F
:106CF000097A01860121818230BD30B5028C22F0F3
:106D000001020284028C8388048B24F0700424F036
:106D100003050C882C4322F002020D8915434A8892
:106D20002A43644DA8420BD0684DA84208D06E4D4E
:106D3000A84205D06D4DA84202D06D4DA8420FD19A
:106D400022F008054A892A4322F004058A882A434A
:106D500023F4807323F400738D891D43CB892B4367
:106D600083800483C9888186028430BD70B5028C1B
:106D700022F010020284028C8388048B24F4E04405
:106D800024F440760D884FF6FF7404EA0525354358
:106D900022F020020E8904EA061616434A8804EA05
:106DA00002123243434EB04202D0484EB04217D195
:106DB00022F080024E8904EA0616164326F04006A9
:106DC0008A8804EA0212324323F4806323F40063C6
:106DD0008E8904EA86061E43CB8904EA8303334383
:106DE00083800583C9880187028470BD70B5028CD9
:106DF00022F480720284028C8388848B24F07004D5
:106E000024F003040D88254322F400720E894FF606
:106E1000FF7404EA062616434A8804EA0222324333
:106E2000244EB04202D0294EB04217D122F400665F
:106E30004A8904EA0222324322F480668A8804EAFC
:106E40000222324323F4805323F400538E8904EA50
:106E500006161E43CB8904EA0313334383808583DC
:106E6000C9888187028470BD70B5028C22F480527B
:106E70000284058C8288838B23F4E04323F44076DC
:106E80000C884FF6FF7303EA0424344325F40055BD
:106E90000E8903EA06362E434D8803EA053535434D
:106EA000044EB04202D0094EB04226D122F48046B0
:106EB0008A891FE0002C01400004004000080040C7
:106EC000000C00400010004000140040003401405D
:106ED000004C0140005001400054014000180040A7
:106EE000001C0040002000400040014000440140E0
:106EF0000048014003EA8212324382808483C988B9
:106F0000A0F84010058470BD828B22F44062828319
:106F1000828B4FF6FF7303EA01210A438283704795
:106F2000F0B5048C24F480540484868B048C4FF6D2
:106F3000FF7505EA013726F4734605EA022232435B
:106F400005EA03331343F74A90420ED0F64A9042C3
:106F50000BD0B0F1804F08D0F44A904205D0F44AEB
:106F6000904202D0F34A904205D124F400513943B3
:106F700041F4805104E024F402420A4342F4805177
:106F800083830184F0BD828B22F00C028283828B8A
:106F90000A4382837047F0B5048C24F4807404841F
:106FA000858B048C4FF6FF7707EA012625F0F30561
:106FB00007EA031313432B43DA4A90420ED0DA4A0E
:106FC00090420BD0B0F1804F08D0D84A904205D003
:106FD000D74A904202D0D74A904205D124F400719A
:106FE000314341F4807104E024F420620A4342F406
:106FF000807183830184F0BD028B22F4406202839E
:10700000028B4FF6FF7303EA01210A4302837047A4
:10701000F0B5048C24F010040484068B048C4FF625
:10702000FF7505EA011726F4734605EA0333334377
:1070300005EA02221A43BB4B98420ED0BA4B984243
:107040000BD0B0F1804F08D0B84B984205D0B84B68
:10705000984202D0B74B984205D124F02001394321
:1070600041F0100104E024F0A0030B4343F01001B1
:1070700002830184F0BD028B22F00C020283028B9A
:107080000A430283704770B5048C24F00104048421
:10709000058B048C25F0F3054FF6FF7606EA031303
:1070A00013432B439F4A90420ED09F4A90420BD0ED
:1070B000B0F1804F08D09D4A904205D09C4A904242
:1070C00002D09C4A904205D124F002020A4342F0C9
:1070D000010104E024F00A020A4342F001010383A3
:1070E000018470BD70B505460C468E48854209D0B6
:1070F0008D48854206D0B5F1804F03D08B4885423C
:1071000000D08B4820886188A288238958B1042840
:1071100011D0082817D02846FFF702FFE18828463B
:10712000BDE87040F0E62846FFF7ADFFE18828464D
:10713000BDE870409FE72846FFF76AFFE1882846D0
:10714000BDE8704058E72846FFF725FFE18828464C
:10715000BDE8704017E72DE9F04107460C460025D1
:1071600001266188002900D10225A288012A00D1C8
:1071700002262088238988B13846FFF749FFE18835
:107180003846FFF739FF2389324629463846FFF74C
:107190007AFFE1883846BDE8F0416CE73846FFF7F2
:1071A00072FFE1883846FFF766FF23893246294699
:1071B0003846FFF72DFFE1883846BDE8F0411BE770
:1071C00010B50A884B88CC881A438B8823431A430E
:1071D0000B891A434B8989891A430A43A0F8442032
:1071E00010BD4FF6FF71818000210180C180418078
:1071F000017270470021018041808180C18001813E
:1072000041818181C181704700210180418001223B
:107210008280C1800181704700210180418081808E
:10722000C1800181418181817047002904D001889A
:1072300041F0010101807047018821F001010180C6
:107240007047002905D030F8441F41F40041018007
:10725000704730F8441FC1F30E0101807047002AC7
:1072600003D082890A438281704782898A4382815E
:107270007047818270471143A0F848107047002A78
:1072800003D082890A438281704782898A4382813E
:107290007047018921F0070101817047028922F0BE
:1072A00070020A430281704700B503461846FFF793
:1072B000F5FF188940F00700188100BD70B50D4634
:1072C00004461146602D0CD001222046FFF7DBFE5C
:1072D00029462046FFF7E2FF208940F00700208181
:1072E00070BD01222046FFF793FEF1E730B5048917
:1072F000E4B24FF6FF7505EA032313430B43234320
:10730000038130BD10B504462046FFF7EFFF20890A
:1073100020F0070040F0070020F0700040F07000FF
:10732000208110BD002C01400034014000040040C9
:1073300000080040000C004010B504462046FFF74E
:10734000D5FF208940F480402081EAE701858282D0
:107350007047028822F070020A430280704770B5BD
:107360000589048B068C25F007050D434FF6FC417B
:107370000C4040F201110C4326F022064FF6FF713B
:1073800001EA03111143314305810483018470BD77
:10739000028B22F070020A4302837047028B22F4B0
:1073A000E0424FF6FF7303EA012111430183704766
:1073B000828B22F070020A4382837047828B22F410
:1073C000E0424FF6FF7303EA0121114381837047C6
:1073D000002904D0018841F08001018070470188B4
:1073E00021F0800101807047002904D0818841F09C
:1073F000040181807047818821F0040181807047F9
:10740000002904D0818841F008018180704781887B
:1074100021F0080181807047002904D0818841F063
:10742000010181807047818821F0010181807047CE
:10743000028B22F008020A4302837047028B22F477
:1074400000624FF6FF7303EA012111430183704785
:10745000828B22F008020A4382837047828B22F4D7
:1074600000624FF6FF7303EA0121114381837047E5
:10747000028B22F004020A4302837047028B22F43B
:1074800080624FF6FF7303EA0121114301837047C5
:10749000828B22F004020A4382837047828B22F49B
:1074A00080624FF6FF7303EA012111438183704725
:1074B000028B22F080020A4302837047028BC2F3E0
:1074C0000E024FF6FF7303EA012111430183704757
:1074D000828B22F080020A4382837047828BC2F340
:1074E0000E024FF6FF7303EA0121114381837047B7
:1074F000028C22F002020A4302847047028C22F0BE
:1075000008020A4302847047028C22F020024FF6E0
:10751000FF7303EA0111114301847047028C22F0CA
:1075200080024FF6FF7303EA011111430184704793
:10753000028C22F400724FF6FF7303EA012111431B
:1075400001847047028C22F400624FF6FF7303EA55
:107550000121114301847047028C22F400524FF63E
:10756000FF7303EA013111430184704710B5012311
:107570008B40048C9C430484038C8A401343038413
:10758000CFE610B504238B40048C9C430484038C09
:107590008A4013430384C4E630B500F11803012484
:1075A0008C40058CA5430584002911D008290FD0F3
:1075B000091FC1F34E001844016821F4E041016045
:1075C00001684FF6FF7303EA02221143016030BDE8
:1075D00003EB5100016821F0700101600168114363
:1075E000016030BD002904D0018841F00201018012
:1075F0007047018821F0020101807047002904D002
:10760000018841F0040101807047018821F00401E4
:1076100001807047002904D0818841F08001818079
:107620007047818821F0800181807047028822F0B4
:107630000802028002880A4302807047828822F092
:107640007002828082880A4382807047028922F019
:107650000702028102890A4302817047028922F0EF
:107660008002028102890A43028170478184704747
:107670008185704781867047018770478187704791
:10768000A0F840107047028822F4407202800288FD
:107690000A4302807047808E7047008F7047808F4A
:1076A0007047B0F840007047808C7047008D70477D
:1076B00002460020128A0A4200D001207047C943C6
:1076C0000182704702460020138A0B4092890A40CB
:1076D000002B02D0002A00D001207047C94301824C
:1076E00070470000FE4A116801F038010143116043
:1076F0007047FB490A6822F008020A600A680243E0
:107700000A607047F6490A6822F010020A600A68A7
:1077100002430A607047F248F2494160F249416011
:107720007047EF48EF494160EF4941607047EC48CE
:10773000016941F0800101617047E948016941F048
:107740008001016170470420E549CA68D20701D071
:1077500001207047CA68520701D502207047C968E6
:10776000C906FBD50320704700B50346FFF7EBFFC2
:1077700002E0FFF7E8FF5B1E012801D1002BF8D1E2
:10778000002B00D1052000BD70B505464FF4302612
:107790003046FFF7E9FF042811D1D14C206940F0B1
:1077A000020020616561206940F0400020613046A0
:1077B000FFF7DAFF216941F6FD721140216170BDCA
:1077C00030B54FF430252846FFF7CEFF042810D1FE
:1077D000C34C206940F004002061206940F0400063
:1077E00020612846FFF7C0FF216941F6FB72114076
:1077F000216130BD00B50346FFF7A5FF02E0FFF7AA
:10780000A2FF5B1E012801D1002BF8D1002B00D173
:10781000052000BD30B54FF430252846FFF7EAFFBC
:10782000042810D1AE4C206940F00400206120698A
:1078300040F0400020612846FFF7DCFF216941F657
:10784000FB721140216130BD0020A549C96989073B
:1078500000D50120704770B5A525FFF7F5FF00B1F1
:1078600000254FF430263046FFF77EFF042818D15C
:107870009B4C9C48A0609C48A060206940F0200080
:107880002061206940F0400020613046FFF76CFF26
:1078900041F6EF76042805D0052802D02169314051
:1078A000216170BD206941F6DF71084020612069C7
:1078B00040F0100020618D4805804FF40050FFF724
:1078C00053FF0528EDD021693140216170BD2DE9BC
:1078D000F84105460E46002000904FF40057384608
:1078E000FFF742FF04280FD17D4C206940F00100D2
:1078F00020612E80B8464046FFF736FFBF1E0428A1
:1079000004D0216939402161BDE8F881AD1C0095A2
:107910000099300C08804046FFF726FF2169394066
:107920002161F1E700887047F0B506460D464FF437
:1079300000573846FFF718FF04280CD1684C20691F
:1079400040F00100206135803846FFF70DFF2169C6
:10795000BA1E11402161F0BDF0B505460E464FF448
:1079600000573846FFF700FF042813D15C4C5D48F0
:10797000A0605D48A060206940F0100020612E806A
:107980003846FFF7F1FE052804D0216941F6EF7271
:1079900011402161F0BD2DE9F043C043C4B2C0F3F2
:1079A0000725C0F30746070E4FF400594846FFF776
:1079B000DBFE04283CD1DFF828814A49C8F80810CA
:1079C0004949C8F80810D8F8101041F01001C8F85B
:1079D0001010FF2C05D04548083004804846FFF7BA
:1079E000C3FE042807D1FF2D05D040480A3005808A
:1079F0004846FFF7B9FE042807D1FF2E05D03B48C3
:107A00000C3006804846FFF7AFFE042807D1FF2F51
:107A100005D036480E3007804846FFF7A5FE0528FA
:107A200006D0D8F8101041F6EF721140C8F81010C7
:107A3000BDE8F08370B505464FF430263046FFF7B9
:107A400093FE042818D1264C2648A0602648A06042
:107A5000206940F020002061206940F04000206152
:107A60003046FFF781FE41F6DF71042805D0052876
:107A700002D022690A40226170BD2069084020615D
:107A8000206940F010002061184815B100210180E4
:107A900001E0A52101803046FFF766FE0528EBD006
:107AA000216941F6EF721140216170BD2DE9F0416D
:107AB00006460D4617460A4C0A48A0600A48A060D0
:107AC0004FF400584046FFF74FFE04281DD12069AF
:107AD00040F0100020613D43354345F0F80007E0D9
:107AE0000020024023016745AB89EFCD00F8FF1F5E
:107AF0002549891C08804046FFF736FE052804D03A
:107B0000216941F6EF7211402161BDE8F0811F4803
:107B1000C069800870471D48006A704700201B49F3
:107B20000968890600D501207047184A002903D04A
:107B300011690143116170471169814311617047F7
:107B400001460020114A012904D0D2680A4200D01F
:107B500001207047D169C907FBD0012070470B494C
:107B6000C860704704200949CA68D20701D00120C3
:107B70007047CA68520701D502207047C968C90614
:107B8000FBD503207047000000F8FF1F00200240D3
:107B900001684FF6FE7211400160002101604160F2
:107BA0008160C1607249724A0839904204D14868C4
:107BB00040F00F00486070476D4A1432904204D183
:107BC000486840F0F00048607047694A28329042A7
:107BD00004D1486840F4706048607047644A3C32A1
:107BE000904204D1486840F4704048607047604A51
:107BF0005032904204D1486840F470204860704789
:107C00005B4A6432904204D1486840F47000486096
:107C10007047574A7832904204D1486840F070600B
:107C200048607047534A111F904204D1086840F0E1
:107C30000F00086070474F4A1432904204D1086820
:107C400040F0F000086070474A4A2832904204D160
:107C5000086840F4706008607047464A3C329042C1
:107C600004D1086840F4704008607047414A5032BF
:107C70009042FAD1086840F470200860704730B52F
:107C8000026847F6F0739A430C6A8B682343D1E984
:107C900004452C4323438C692343CC6923434C6A1A
:107CA00023438C6A234313430360CA6842600A6813
:107CB00082604968C16030BD00210160416081601F
:107CC000C160016141618161C161016241628162A2
:107CD0007047002904D0016841F00101016070473C
:107CE00001684FF6FE72114001607047002A03D010
:107CF00002680A430260704702688A430260704764
:107D000041607047406880B2704702460020D10051
:107D100003D518490839096802E015490839096886
:107D2000114200D001207047C10003D51149091F3D
:107D3000086070470E4908394860704702460020C5
:107D4000D10003D50B490839096802E00849083910
:107D50000968114200D001207047C10003D50549D0
:107D6000091F0860704702490839486070470000E1
:107D700008000240080402407047162205A10FA027
:107D800000F06CFA11A000F069FAFEE7FEE7FEE7EA
:107D9000FEE770472E2E5C53544D33324631307817
:107DA0005F46574C69625C7372635C73746D333207
:107DB000663130785F69742E630000004C6F674550
:107DC00072723A2025732C256400000048617264A9
:107DD0004661756C745F48616E646C657221000069
:107DE00071B65A4801685A4A01F4E06111430160D2
:107DF000BFF34F8FFEE70CB5002201920092554869
:107E0000016841F4803101604FF4A063016801F41E
:107E1000003100910199491C0191009911B9019912
:107E20009942F3D10168890302D50121009100E054
:107E300000920099012930D147490A6842F01002A6
:107E40000A600A6822F003020A600A6842F002022D
:107E50000A604168416041684160416841F4806165
:107E60004160416821F47C114160416841F4E811AE
:107E70004160016841F08071016001688901FCD5B1
:107E8000416821F003014160416841F00201416015
:107E90004168C1F381010229FAD10CBDABE710B5ED
:107EA0002C48016841F00101016041682B4A1140F2
:107EB000416001682A4A11400160016821F4802173
:107EC0000160416821F4FE0141604FF41F018160AF
:107ED000FFF7E4FF1D494FF00060091F086010BD67
:107EE00010B51C4A506800F00C011E4B1E480029BA
:107EF0000ED004290ED008290ED0036051681A4A0A
:107F0000C1F30311121D515C0268CA40026010BD2A
:107F10000360F3E70360F1E7516801F470115368FF
:107F200003F48033022404EB914133B153689B0383
:107F300007D50E4B59430160E0E70C4B59430160F4
:107F4000DCE7084B59430160D8E700000CED00E086
:107F50000400FA0500100240002002400000FFF873
:107F6000FFFFF6FE00127A00E006002000093D0047
:107F700010B5A94988420AD1841401212046FEF790
:107F8000DCF92046BDE810400021FEF7D6B9A34930
:107F900088420AD1041401212046FEF7D9F920466F
:107FA000BDE810400021FEF7D3B99D4988420AD1AF
:107FB000C41301212046FEF7CBF92046BDE810404E
:107FC0000021FEF7C5B910BD30B5028802F4415357
:107FD0000A884C88CD8822438C882C4322430C8904
:107FE00022434C8922438C892243CC8922431A4361
:107FF0000280828B22F400628283098A018230BD72
:10800000F0B585B005460C46022000210126AA8B5A
:108010004FF240031A40AA8302222A84AF8BA2683F
:10802000022A21D0A08800B102266846FEF717F97F
:108030000098E188B1F5007F2CD07101B0FBF1F020
:1080400000EB8000A1684000B0FBF1F0401D80B261
:108050000A21B0FBF1F000F00101401AC0F34F001B
:108060004FF6FF7202EA0121821EFE2A01D302208E
:108070000021E288084302432A8420886188A2897B
:108080000843A18811430843384340F40060A883A3
:1080900005B0F0BD000A00EB8000A1684000B0FB15
:1080A000F1F0401D80B2D3E7002101804180818042
:1080B000C180018141818181C18107210182704795
:1080C0000021018041808180C18002228260818103
:1080D0007047002904D0018841F0400101807047B9
:1080E000018821F0400101807047002904D0818B74
:1080F00041F4806181837047818B21F480618183A9
:108100007047090901238B4099B2002A03D0828865
:108110000A438280704782888A4382807047002A9F
:1081200003D082880A438280704782888A43828093
:1081300070478181704780897047A1F57E42FF3A80
:1081400004D0018841F4807101807047018821F4D6
:10815000807101807047002904D0818841F00401BA
:1081600081807047818821F00401818070470288F6
:1081700022F40062028002880A430280704701886C
:1081800041F4805101807047002904D0018841F4F6
:10819000005101807047018821F40051018070472F
:1081A000012901D0008B7047808A7047008A704790
:1081B000B1F5804F04D0018821F4804101807047DF
:1081C000018841F4804101807047024600201289F5
:1081D0000A4200D001207047C9430181704730B581
:1081E0000246002001F00F03012505FA03F4A3B2B3
:1081F000090905FA01F4A4B29188214012891A42B2
:1082000002D0002900D0012030BD01F00F02012171
:108210009140C9430181704700300140003800405F
:10822000003C0040704700007CB51D4616460C001F
:10823000009001D02044401E074B7B442A466946EB
:108240000190304600F03DFC05461CB10020694617
:1082500000F04AFC28467CBDB50800000FB4044974
:1082600010B503AA029800F063FC10BC5DF814FB83
:10827000500600200FB47CB50C0009AA009001D074
:108280002044401E084B7B4469460190089800F04A
:1082900018FC05461CB10020694600F025FC284664
:1082A0007CBC5DF814FB00006908000070B5044652
:1082B00085690068C10601D5302600E02026C00788
:1082C00007D070BDD4E9012130469047206A401C98
:1082D00020626D1EF6D570BD70B5044685690078C4
:1082E000C00707D170BDD4E9012120209047206A42
:1082F000401C20626D1EF6D570BD09684A0501D587
:1083000040B27047C905FCD500B2704709684A05FC
:1083100001D5C0B27047C905FCD580B2704770B5B1
:108320000C460546012A05D02878800600D5EA6962
:10833000002302E0012305E05B1C934202D2E05CD3
:108340000028F9D1A869E618C01AA861286A18445B
:1083500028622846FFF7AAFF04E0D5E9012114F8B6
:10836000010B9047B442F8D32846FFF7B5FF70BD24
:108370002DE9F0410646002410687529314616A5FE
:1083800010D0FFF7BAFF002802DA404213A507E039
:1083900031688A0701D512A502E0490704D511A565
:1083A000012401E0FFF7B2FF00210A2206F12407B1
:1083B00009E0B0FBF2FCB0FBF2F302FB1C00303032
:1083C00078541846491C0028F3D123462A463046E3
:1083D000BDE8F04100F017BB000000002D000000D8
:1083E0002B0000002000000011680268006A53059D
:1083F00001D508700AE0D30501D5088006E0130610
:1084000003D5C217C1E9000200E0086001207047EF
:108410002DE9FF5F15468A460446DFF8AC80F84434
:108420000027D8E900103E46CDE9001010E03AF8E8
:1084300016106A4602A800F019FC411C07D02178EA
:10844000890603D5E269391891420DD80744761C94
:108450002078800602D5E069B84205DDAE42E6DB51
:108460003AF816000028E2D1A069C01BA06120469E
:10847000FFF71CFFD8E90010CDE90010002017E03D
:108480003AF818106A4602A800F0F0FBB0F1FF3F7E
:1084900081460BD000250DF1080B05E0D4E9012140
:1084A0001BF8050090476D1C4D45F7D308F10100FE
:1084B000B0428046E4DB206A384420622046FFF761
:1084C0000BFFBDE8FF9F00009E42000030B400217A
:1084D00000F1240408E002F00705D208303542EA32
:1084E0004372DB086554491C52EA0305F3D1046862
:1084F000002310A2250707D5A40600D421B1C46922
:1085000001230DA2641EC46130BC00F07CBA10B51A
:10851000044621461068FFF7F9FE02462046BDE8F2
:1085200010400023D2E7D21D22F00701D1E9002339
:10853000CCE700000000000030000000F0B40D4661
:108540000188090502D5214C7C4402E01F4C7C4483
:108550000E34002100F1240608E002F00F07120992
:10856000E75D42EA03721B097754491C52EA03078C
:10857000F3D102780023120704D5702D06D009B17B
:10858000022311342246F0BC00F03DBA012310341E
:10859000F8E770B504460D4621461068FFF7B6FEB1
:1085A000024629462046BDE870400023C6E7D21D9A
:1085B00022F00703D3E90023C0E70368126843F001
:1085C000200303600823C3610023B7E77C41000058
:1085D0002DE9F05F894604464FF0000ADFF874B1D8
:1085E000FB44C0F820A02046E1688847002874D0EA
:1085F000252806D0D4E901219047206A401C20623A
:10860000F1E700265F462046E168884720280546B6
:1086100007DB312D05D2781910F8200C08B106437C
:10862000F1E7B00701D526F00406C4F81CA0002726
:10863000C4F818A02A2D09D0284601F010FD38B33F
:1086400004EB8708303DC8F8185019E059F8041BAE
:10865000204604EB87029161E1688847012F0546B7
:1086600018D1E069002820DA26F020061DE0D8F8AD
:10867000180000EB800005EB40003038C8F8180007
:108680002046E1688847054601F0E9FC0028EED164
:10869000012F0AD02E2D08D12046E16888477F1C83
:1086A0000546022F46F02006C4DBA069002803DA45
:1086B000404246F00106A061F00701D026F0100606
:1086C0006C2D0BD0682D09D04C2D39D06A2D35D0AA
:1086D000742D35D07A2D33D016E038E0E1682F467E
:1086E00020468847B842054609D16C2F26D04FF462
:1086F0008060E168064320468847054604E06C2F09
:108700001AD04FF4807006430DB3A5F1410019282B
:1087100002D8203546F400664A462946204626609F
:108720004E46F7F75FFD80B101280BD0F61D26F00D
:10873000070000F1080956E74020E4E78020D8E769
:108740000020D6E706F104094DE7284652E7206AE3
:10875000BDE8F09F0C41000070B5064600F044F9FA
:108760000468054630460A22002100F047FA2C60D2
:1087700070BD401ECAB210F8011F8A4202D0002903
:10878000F9D10020704710B5431E13F8014F002C9B
:10879000FBD105E011F8014B002C03F8014B03D08D
:1087A000521EF7D20021197010BD40EA01030246A3
:1087B00030B59B0710D14FF0013400E008C208C962
:1087C0001D1B9D4315EAC41FF8D013F0FF0102F8EA
:1087D000011B0DD01B0AF8E711F8013B002B02F832
:1087E000013B05D011F8013B002B02F8013BF3D10E
:1087F00030BD0022CBB210F8011B994200D1421EBD
:108800000029F8D11046704710B5431C02E010F85B
:10881000011B71B18107FAD14FF0013202C88C1AE5
:108820008C4314EAC211F9D0C01A0A0603D0C01E44
:1088300010BDC01A10BD0A0401D0801E10BD09026F
:10884000FCD0401E10BD421E12F8013F002BFBD190
:1088500011F8013B002B02F8013BF9D17047032AC4
:1088600040F2308010F0030C00F0158011F8013B4D
:10887000BCF1020F624498BF11F801CB00F8013B34
:1088800038BF11F8013BA2F1040298BF00F801CBF8
:1088900038BF00F8013B11F0030300F00782083AEB
:1088A000C0F0088051F8043B083A51F804CBA0E826
:1088B0000810F5E7121D5CBF51F8043B40F8043B7B
:1088C000AFF30080D20724BF11F8013B11F801CBB0
:1088D00048BF11F8012B24BF00F8013B00F801CB81
:1088E00048BF00F8012B704702F0FF0343EA032260
:1088F00042EA024200F002B84FF000020429C0F040
:10890000128010F0030C00F01B80CCF1040CBCF1C1
:10891000020F18BF00F8012BA8BF20F8022BA1EB13
:108920000C0100F00DB85FEAC17C24BF00F8012BF8
:1089300000F8012B48BF00F8012B70474FF00002F0
:1089400000B5134694469646203922BFA0E80C5045
:10895000A0E80C50B1F12001BFF4F7AF090728BF20
:10896000A0E80C5048BF0CC05DF804EB890028BF9C
:1089700040F8042B08BF704748BF20F8022B11F0C5
:10898000804F18BF00F8012B704710B5044610F057
:10899000030F08BF11F0030F40F015804FF0013EA8
:1089A000121FC0F20E8051F8043BA3EB0E0C2CEA10
:1089B000030C1CEACE1C08BF40F8043BF0D0A1F128
:1089C000040102F10402521E08DB11F8013B002BE6
:1089D00000F8013BF7D11146FFF78EFF204610BD8E
:1089E000704770477047704700487047106C002010
:1089F00010B5FFF7F9FF006810BD10B50446FFF78A
:108A0000F3FF046010BD2DE9F0470D4699469246EC
:108A1000044600F124080168880604D5E06921F0C5
:108A20001001216000E00120A84201DD471B00E0A9
:108A30000027A1697A1902EB0900081AA0612078C1
:108A4000C00602D42046FFF731FC002608E0D4E936
:108A500001211AF806009047206A401C761C20620B
:108A60004E45F4DB2078C0060AD52046FFF71EFCF1
:108A700006E0D4E9012130209047206A401C2062A2
:108A8000381EA7F10107F4DC07E0D4E9012118F84A
:108A900005009047206A401C2062281EA5F10105B0
:108AA000F3DC2046FFF718FC2078000602D50220F0
:108AB000BDE8F0870120FBE701694A1C02610878E4
:108AC000704700B58FB0CDE901310021059105490E
:108AD0007944CDE9031011466846FFF779FD0FB0E0
:108AE00000BD0000E5FFFFFF0A6802F8010B0A6005
:108AF0007047D1E900239A4202D2531C0B601070D8
:108B0000704710B5436913B1AFF3008001E0FFF780
:108B100006FC012010BD127800F124010A70002229
:108B20004A700122EDE711684FF0FF32E9E70000DB
:108B3000074B70B50D467B44FFF7C3FF044628463C
:108B400000F013FD10B14FF0FF3070BD204670BD36
:108B500075B1FFFF10B5436913B1AFF3008001E0B9
:108B6000FFF756FC012010BD128800F12401828419
:108B70000022C2840122EDE711684FF0FF32E9E7DD
:108B80002DE9F0418046D21D22F007020025D2E9EE
:108B90000002F52915A614D0011E72F1000106DAB3
:108BA0000023D0EB030063EB020211A608E0D8F823
:108BB00000108B0701D50FA602E0490701D50EA6CC
:108BC00001251146002408F1240704E000F0ACF868
:108BD00030323A55641C50EA0102F7D12B46324636
:108BE00021464046BDE8F041FFF70DBF0000000000
:108BF0002D0000002B000000200000002DE9F047B0
:108C000091460F4680460446002614F8015B2DB1BC
:108C100000F082F80068405DC007F6D12B2D02D02D
:108C20002D2D18D0641E4A463946204600F04EFCD1
:108C300027B13968A14201D1C7F800804FF0020482
:108C400071050BD54042002803DDFFF7CDFE04601F
:108C5000A007BDE8F08746F48066E4E70028F8DA6C
:108C6000FFF7C2FE04606FF00040F2E770B51646F1
:108C70000C46054600F050F8036893F801010128FE
:108C800006D0FF2C0FD8185D68B101202C7070BD84
:108C9000D3F807013246214603F20713034428465E
:108CA000BDE8704018474FF0FF3070BD10B5203A56
:108CB000C0F00B80B1E81850203AA0E81850B1E895
:108CC0001850A0E81850BFF4F5AF5FEA027C24BF4B
:108CD000B1E81850A0E8185044BF18C918C0BDE842
:108CE00010405FEA827C24BF51F8043B40F8043B0B
:108CF00008BF7047D20728BF31F8023B48BF11F8C0
:108D0000012B28BF20F8023B48BF00F8012B704719
:108D100000487047106C002010B500F04FFC001D9B
:108D200010BD00BFA516000030B5B0F10A024FEA31
:108D3000900E71F100034EEA817EB0EB0E0061EB04
:108D400091014FEA101E4EEA017E10EB0E0041EB3E
:108D500011114FEA102E4EEA016E10EB0E0041EB9E
:108D600011214FEA104E4EEA014E10EB0E0041EB7E
:108D70001141401841F100014FEAD00040EA417032
:108D80004FEAD10110EB80054FEA810444EA907468
:108D900044EB01046D1944EB0404521BA3414FF052
:108DA000000348BF0A3200D530BD401C41F100012C
:108DB00030BD70472DE9FF4F0C461E464FF0FF3780
:108DC0008BB0D2E90001DDF860800A908A46C1F3D9
:108DD0000A5505B93D46002108464FF00000BAF19A
:108DE000000F00F4400005DA00EB80004FF4400172
:108DF00001EA50004FEA9059B9F1010F00DDB94680
:108E00000A9850EA4A000ED044F61050A5F2FF35F9
:108E100045432F14B8F1000F1ED07542291E1EDDE8
:108E2000C9F100021CE0B8F1010F4FF0000001D0C1
:108E3000302103E0F24305E02154401CB042FBDB4B
:108E400030460022002121540B99C1F80880C1E965
:108E500000200FB0BDE8F08FBD1B6D1CDEE74A4659
:108E600000DA694206A800F0FBFB06AB93E80700B6
:108E700003AB83E8070050460A9900F0ADFC8DE88B
:108E80000700A0F500501F3800900398002D0ADD60
:108E900042F21F014A460844002303A90390684692
:108EA00000F016FF09E0A0F500504A461F380023E5
:108EB00003A90390684600F020FF8DE80700000436
:108EC000000C03D04FF0FF30410800E01046B8F12D
:108ED000000F03D00022009215461EE0751E05D437
:108EE000FFF722FF303262556D1EF9D5B3460122DD
:108EF000084302D000227F1C04E02078302801D1F2
:108F000000227F1E002A099784D01DE0112D07DA68
:108F1000FFF70AFF303262556D1C50EA0102F5D1AD
:108F2000084302D00098C8B10EE00021681E05E099
:108F3000235C625C63542254401E491C8142F7DB6F
:108F4000AB46A81B401E0990002004F80B000B98AC
:108F5000099AC0F80880C0E9002B7AE711264FF083
:108F6000000857E72DE9F04F88460446D21D22F04D
:108F7000070191B0D1E90001CDE90A0100F0F4FF49
:108F800002460B98C00F01D02D2007E02068810712
:108F900001D52B2002E0202101EAC000032A09901C
:108FA00001D0072A05DB03464146204600F00AFBB4
:108FB0000BE12078800601D5E06900E00620B8F1D9
:108FC000650F814606D0B8F1660F18D0B8F1670F6B
:108FD00070D131E00020B9F1110F009001DB1123B5
:108FE00001E009F101030AAA01A90CA8FFF7E2FEBA
:108FF000DDE90C70002609F10105834647E00120F8
:109000004B4600904FF000470AAA01A90CA8FFF7B1
:10901000D1FEDDE90DB00C995D46002610B909F1CD
:1090200001000D18B9EB050003D4C0F1FF3609F1BA
:109030000105A5EB09002BE0B9F1010F01DA4FF0B2
:1090400001090020B9F1110F0090484601DD1123FC
:1090500000E003460AAA01A90CA8FFF7ABFEDDE970
:109060000C704D4600268346207800070AD4AB4595
:1090700000DA5D4601A8012D04DD411911F8011C3B
:10908000302907D04F4502DA17F1040F04DA012026
:1090900082460FE06D1EEEE7002F02DCED1B3E4422
:1090A00003E0781CA84200DD7D1CB81B00F1010A1A
:1090B0004FF000472078000703D4AA4501DB4FF0AA
:1090C000FF3A0021B7F1004F0DF143088DF843102E
:1090D00024D002202B23002F01DA7F422D230A21E6
:1090E000021EA0F1010000DC5FB197FBF1FC97FBD1
:1090F000F1F201FB1C7C17460CF1300C08F801CD95
:10910000EEE7A8F1010003702188090501D545218A
:1091100000E06521A0F1010800F8011C09980FA9E1
:10912000A1EB0807FF1D00B10120411901EBEA7016
:10913000A1693844081A401EA0612078C00602D4F4
:109140002046FFF7B3F8099828B1D4E901219047E8
:10915000206A401C20622078C00622D52046FFF7F6
:10916000A5F81EE0002E04DBB34502DD01A8805DFA
:1091700000E03020D4E901219047206A401C2062A1
:10918000761CAAF101005FEA000A0AD100F016FA83
:10919000C0680168405CD4E901219047206A401C06
:1091A0002062281EA5F10105DCDC07E0D4E90121DD
:1091B00018F8010B9047206A401C2062381EA7F166
:1091C0000107F3DC2046FFF787F8032011B041E6E2
:1091D0002DE9F04F04460D46D21D22F0070089B05C
:1091E000D0E900974846394600F0BEFE0246F80F27
:1091F00001D02D2307E02068810701D52B2302E051
:10920000202101EAC0038DF820300BB1012000E0DD
:109210000020032A824601D0072A04DB2946204683
:1092200000F0D0F93FE12078800601D40D2500E060
:10923000E569C7F30A560D2D49DA00214FEA175B9D
:1092400008464FF00000002F00F4400007DA00EB62
:1092500080004FF4400100EBD07001EA60008115FE
:10926000012901DD4FF0FF3100224FEA850CBCF1EE
:10927000180F06D31346ACF118004FF08052C240CD
:1092800003E04FF4801323FA0CF30CF10C0CBCF147
:10929000200F04D3ACF1200C09FA0CF001E007FA1E
:1092A0000CF000294FF0004801DD18B90FE00ED195
:1092B00040450CD319EB02095F4121B9404502D169
:1092C0009F4329EA0209BBEB175F00D0761C208878
:1092D000000502D57B48784402E07A487844193882
:1092E00008AA302302F80A30037C0AF10101002E9B
:1092F0000AF1020A53546A4602DC4FF0300101E0E1
:109300004FF031014FF001088DF8001002D0A6F2A5
:10931000FF3603E059EA470100D06B4E002D02DC16
:109320002178090704D54FF002082E218DF801108D
:10933000C44600210BE0C7F303433F01C35C491C53
:109340006D1E02F80830052908F1010801DA002D28
:10935000F1DC00210CE000EB1973491C1B786D1E39
:10936000082902F808304FEA091908F1010801DA62
:10937000002DF0DC21688B0602D516E0A8F101086B
:10938000E04505DD02EB080313F8013C302BF5D076
:10939000B8F1000F09DD02EB080313F8013C2E2B96
:1093A00003D1090701D4A8F10108002D05DD3E21F4
:1093B00002F808106D1E08F10108407C002E02F82A
:1093C000080008F1010804DA2D20764202F80800AE
:1093D00002E02B2002F808000A214FF47A7086423E
:1093E00008F101080BDB96FBF0F3303302F808308C
:1093F00096FBF0F308F1010800FB136601E0642E10
:109400000CDB642096FBF0F3303302F8083096FB57
:10941000F0F308F1010800FB136601E00A2E06DBF9
:1094200096FBF1F0303002F8080008F1010896FBD5
:10943000F1F001FB1060303002F80800A16908F17A
:10944000010808EB050202EB0A00081AA061207867
:10945000C00602D42046FEF729FF216A08AE01EBC0
:109460000A00206204E0D4E9012116F8010B9047BC
:10947000BAF1010AF7D22078C00602D52046FEF7DD
:1094800015FF6E4609E016F8010B3E280FD0D4E90F
:1094900001219047206A401C2062B8F10108F2D2F5
:1094A0002046FEF719FF09B00320BDE8F08F206ABF
:1094B0002844206203E0D4E90121302090476D1E4A
:1094C000EBD3F8E78134000002FCFFFF2DE9F05FE9
:1094D000824615468B4600270AF10104B9460078FA
:1094E000302801D09DB113E014F8010B0127782832
:1094F00003D0582801D045B10AE00DB1102D07D195
:10950000002714F8010B102502E0082500E00A25C9
:109510000026B0460EE005FB080005FB06F101271A
:109520001FFA80F801EB1046B6F5803F00D3B9462C
:1095300014F8010B294600F085F80028EBDABBF19E
:10954000000F05D00FB1641E00E05446CBF8004078
:10955000B9F1000F06D0FFF747FA02210160C81EDB
:10956000BDE8F09F48EA0640FAE7007B00F0800083
:1095700070477546FFF7CCFBAE460500694653467B
:1095800020F00700854618B020B5F6F7A7FEBDE825
:1095900020404FF000064FF000074FF000084FF05A
:1095A000000B21F00701AC46ACE8C009ACE8C009EB
:1095B000ACE8C009ACE8C0098D4670470048704768
:1095C000306C00202DE9F0411F4604460326016857
:1095D000072A01F4006004DB08B116A505E016A512
:1095E00003E008B115A500E015A521F010002060EA
:1095F000A069C01EA0610FB1401EA0612046FEF709
:1096000055FE4FB1D4E9012138469047206A401CED
:109610002062C01C206206E0206AFAE7D4E901213A
:1096200015F8010B9047761EF8D22046FEF754FE3F
:10963000BDE8F0814E414E006E616E00494E46001D
:10964000696E66003A2800D2303820F02002412AA4
:1096500001D3A2F13700884201D34FF0FF307047A9
:109660002DE9F047814616468AB0354878440DC842
:109670008DE80D0032487844801C03AC0DC884E8A6
:109680000D0041F69B300844372190FBF1F290FB2E
:10969000F1F5A5F1800501FB12041B3C02D56442E3
:1096A000012000E00020DFF898A080460027FA445F
:1096B000AAF1BE0A0EE0E0070AD03246684607EB80
:1096C000470101230AEB810100F017FB8DE8070039
:1096D00064107F1C002CEED1194F7F44AE3F19E07F
:1096E000E80715D007EB04100DF1180A90E80E00FA
:1096F0008AE80E00C068F04201D1981908903246FD
:10970000012306A903A800F0F8FA03AB83E80700D9
:109710006D10641C002DE3D14FF001033246694601
:10972000B8F1000F03A802D000F0D2FA01E000F077
:10973000E4FAC9E90001C9F808200AB0BDE8F087D9
:109740007C31000010B50446AFF300802046BDE830
:109750001040F6F7AABD00004FF0013C50F8042B72
:1097600051F8043B9A4221D1A2EB0C03934313EA34
:10977000CC1317D150F8042B51F8043B9A4215D161
:10978000A2EB0C03934313EACC130BD150F8042B38
:1097900051F8043B9A4209D1A2EB0C03934313EA1C
:1097A000CC13DBD04FF00000704700BFD01A01BAD5
:1097B000B1FA81F101F0180122FA01F0CB40C1F1B8
:1097C0002001DBB2C0B2C01A2CFA01F3D11A9143C6
:1097D00011EAC311E6D170475FEA400C08BF91F06F
:1097E000000F4FEA8C234FEAC12243EA51514FEA5E
:1097F0001C5018BF00F5F0404FEA300018BF41F090
:1098000000415FEA6C5C00F02980BCF1FF3F08BFBB
:1098100040F080407047130C06BF12044FF0100C4C
:109820004FF0000C130E04BF12020CF1080C130FC2
:1098300004BF12010CF1040C930F04BF92000CF151
:10984000020CD30F04BF52000CF1010C11464FF073
:109850000002A0F11F00A0EB0C00704711F0004FB8
:1098600008BF704731F000413FF4D5AF0B0C06BF85
:1098700009044FF0100C4FF0000C0B0E04BF09024E
:109880000CF1080C0B0F04BF09010CF1040C8B0F39
:1098900004BF89000CF1020CCB0F04BF49000CF18E
:1098A000010CCCF12003A0EB0C0022FA03F302FA26
:1098B0000CF241EA030100F10100704720F07F4CF7
:1098C00080EA030023F07F47ACEB070303F57C53EA
:1098D00000F0004003F1FF032DE980494FEA154BEA
:1098E00009B44FEA144325EA0B4E24EA03480FF269
:1098F000042606EB132749083E785FEA320203FB91
:109900000667C7F5000707FB06F64FEA54374FEA2C
:10991000D64606F1020607FB066CCCF1005C4FEA66
:109920001C472CEA074C07FB06F40CFB06F504EB7E
:1099300015464FEA961634BF00204FF000404FEA1C
:10994000D13706FB07FC4FEA1C4C0CFB0BF7D21B74
:1099500003FB0CF761EB07010CFB0EF7B0EB0740C4
:1099600072EB17420CFB08F734BFA2EB0742B2EBD5
:10997000074261EB17414FEA0C444FEA910706FB9F
:1099800007FC4FEA1C4C0CFB0BF7B0EBC74072EB2B
:10999000573203FB0CF734BFA2EBC742B2EBC7420E
:1099A00061EB57310CFB0EF7B0EBC70072EB57724F
:1099B0000CFB08F734BFA2EBC702B2EBC70261EBA6
:1099C0005771039F4FEA816141EA921104EBCC0485
:1099D0004FEAD1374FEA826206FB07FC42EA901257
:1099E0004FEA80604FEA1C4C0CFB0BF7D21B03FBC9
:1099F0000CF761EB07010CFB0EF7B0EB074072EBC5
:109A000017420CFB08F734BFA2EB0742B2EB074248
:109A100061EB17414FEA8C554FEA910704EB9C2408
:109A200006FB07FC4FEA1C4C0CFB0BF7B0EBC740E6
:109A300072EB573203FB0CF734BFA2EBC742B2EB19
:109A4000C74261EB57310CFB0EF7B0EBC70072EB6E
:109A500057720CFB08F734BFA2EBC702B2EBC70288
:109A600061EB577115EB4C254FEA816141EA921188
:109A70004FEA82624FEAD13742EA901206FB07FCB6
:109A800044F100044FEA80604FEA1C4C0CFB0BF7DA
:109A9000D21B03FB0CF761EB07010CFB0EF7B0EBDD
:109AA000074072EB17420CFB08F734BFA2EB0742EA
:109AB000B2EB074261EB174115EB1C154FEA813100
:109AC00041EA92414FEA823242EA90424FEA8030C4
:109AD0004FEA0C7644F1000448EA03434EEA0B488F
:109AE0004FF0000EB2EB080C71EB030724BF624687
:109AF00039464EEB0E0E4FF0000B00185241494113
:109B00004BEB0B0BB2EB080C71EB03077BF1000B7B
:109B100024BF624639464EEB0E0E4FF0000B001884
:109B2000524149414BEB0B0BB2EB080C71EB0307B5
:109B30007BF1000B24BF624639464EEB0E0E51EA14
:109B4000020718BF46F0010616EB0E7655F100022B
:109B500054F1000103D5BDE88901BDE80088BDE8E6
:109B60008901BDE80048B619524141EB0101A3F15A
:109B70000103704780807F7E7D7C7B7A7978777661
:109B800076757473727171706F6E6E6D6C6C6B6ADA
:109B90006A69686867666665646463636261616078
:109BA000605F5F5E5E5D5D5C5C5B5B5A5A595958F5
:109BB000585757565655555554545353525252515F
:109BC000515050504F4F4F4E4E4D4D4D4C4C4C4BB5
:109BD0004B4B4A4A4A4949494848484747474746FC
:109BE0004646454545444444444343434342424238
:109BF00042414141002B9C4630D477002BD01CB50C
:109C00004FEA370703B44FF010004FF01001BAF1DC
:109C1000000F06D0BCF1000FDCBF40F0080040F0A0
:109C200008014FF000000FBCBDE810400BF1010B24
:109C3000BBF1010F08BF5FEA170722BF12F1010253
:109C400011F101014FF0004143F1000300F0004029
:109C500043EA00007047F9D35708D0E746EA0646C2
:109C600013F1400F4FEA16461FDD13F1200FDFBF3F
:109C700016430A46002120335B42BED0C3F12007C1
:109C800046EA064602FA07F74FEA164646EA07068C
:109C9000C3F1200722FA03F201FA07F721FA03F1D0
:109CA0004FF0000342EA0702A7E746EA020646EA47
:109CB00006464FEA164646EA0106BCBF46EA064695
:109CC000360C4FF000034FF000024FF0000194E714
:109CD0002DE9804C9A46934670B491E8380007C845
:109CE00031EA400C48BF34EA430C03D5FFF7E6FDE8
:109CF000FFF780FFF0BCBDE8008C2DE9804C9A4650
:109D0000934670B491E8380007C810F0804F08BF40
:109D100013F0804F03D100F005F8FFF76BFFF0BCA4
:109D2000BDE8008C20F07F4780EA030023F07F4CE1
:109D300007EB0C03A3F57C5300F00040A3F1FE03F6
:109D400092F0000F00F0B38095F0000F00F07780E4
:109D50002DE901494FEA11404FEA144621EA004833
:109D600000FB06FC24EA064708FB06F607FB08F89A
:109D700000FB07F718EB06484CEB164C4FEA124B6A
:109D800018EB07484FEA15464CEB174022EA0B4EFA
:109D90000BFB06FC25EA06470EFB06F607FB0EFE4C
:109DA0000BFB07F71EEB064E4CEB164C4FF0000674
:109DB0001EEB074E4CEB174B18EB0B0840F1000065
:109DC00018EB0E0B58EB000840F100008F1A4FF013
:109DD00000013CBFC943661B14BFB5EB040C002156
:109DE0003CBFC943F61B4FEA17444EEA8E0E27EAE2
:109DF00004454FEA1C4704FB07622CEA074C05FBAD
:109E000007F70CFB05F604FB0CFC16EB074642EBD0
:109E1000174216EB0C4642EB1C421BEB060658EBB6
:109E20000202414146EA9E0601D5BDE80189B61904
:109E3000524141EB0101A3F10103BDE801894FEA61
:109E400014454FEA114724EA054621EA074C05FB71
:109E500007F406FB07F70CFB06F105FB0CFC11EB06
:109E6000074144EB17444FEA124711EB0C4144EB16
:109E70001C4422EA074C05FB07F206FB07F70CFB24
:109E800006F605FB0CFC16EB074642EB174216EBF9
:109E90000C4642EB1C456A1854F1000148BF70475C
:109EA000B619524141EB0101A3F10103704795F04E
:109EB000000F37D04FEA11424FEA144721EA024619
:109EC00024EA074C02FB07F106FB07F70CFB06F43C
:109ED00002FB0CFC14EB074441EB17414FEA15471A
:109EE00014EB0C4441EB1C4125EA074C02FB07F53F
:109EF00006FB07F70CFB06F602FB0CFC16EB07460D
:109F000045EB174516EB0C4645EB1C42121951F177
:109F1000000148BF7047B619524141EB0101A3F15E
:109F2000010370474FEA14454FEA114724EA0546FA
:109F300021EA074C05FB07F106FB07F70CFB06F2CD
:109F40004FF0000605FB0CFC12EB074241EB1741FA
:109F500012EB0C4251EB1C4148BF7047921841EB89
:109F60000101A3F101037047490050EAC12018BF65
:109F700004204A0D18BF40F0010040F2FF72B2EB1E
:109F8000515F08BF40F00200012808BF052070475C
:109F90002DE9F0414F1E00EBC7010446D1E9000155
:109FA00015461E4637F006020DD02A46334600F00D
:109FB0000FFD7F1E04EBC703D3E9002300F030FA46
:109FC00037F00602F1D1022F25D0042F13D0062F2F
:109FD00018BFBDE8F0812A46334600F0F9FCD4E909
:109FE0000A2300F01DFA2A46334600F0F1FCD4E9BA
:109FF000082300F015FA2A46334600F0E9FCD4E9BC
:10A00000062300F00DFA2A46334600F0E1FCD4E9BD
:10A01000042300F005FA2A46334600F0D9FCD4E9BF
:10A02000022300F0FDF92A46334600F0D1FCD4E9C2
:10A030000023BDE8F04100F0F3B900000022134610
:10A040001046014900F0A8BA0000F03F012200F0DC
:10A05000E9BE002213461046114600F09DBA303882
:10A060000A2801D201207047002070472DE9F04DE9
:10A07000C84A002490B0914205DA21F0004393428F
:10A0800001D805D120B110B0BDE8F04DFFF7DEBF1B
:10A09000B1F5801F1BDA53EA000209D0002911DA5A
:10A0A0000120FEF7AAFC10B0BDE8F04DFFF7D1BFCC
:10A0B0000220FEF7A2FCFFF7C1FF10B081F00041C3
:10A0C000BDE8F08D6FF03504362200F0ABFE04EBF6
:10A0D0002152C1F31308B049A2F2FF33414401F405
:10A0E000801282F07F6103EB225281F04051009296
:10A0F00041EA08010022A94B00F074FD044608F172
:10A100000200A74EC0F313000D467E44032867D219
:10A11000D6E90023204600F097FB1ED100980028C6
:10A1200002BFD6E9000110B0BDE8F08D00F025FCBB
:10A1300007460C469B4A9C4B00F04AFC06460D46DF
:10A140009A4A9B4B3846214600F042FC10B03246FA
:10A150002B46BDE8F04D00F063B94FF05532954BFA
:10A160002046294600F034FC0022934B00F02EFDDF
:10A1700006460F4622462B461046194600F028FC9C
:10A1800032463B4600F024FC064600980F46F0B1EC
:10A1900000F0F3FB80468A46824A834B00F018FCAD
:10A1A00032463B4600F012FD22462B4600F01AFDD7
:10A1B00005460C467D4A7E4B4046514600F008FC61
:10A1C00010B02A462346BDE8F04D00F00BBD0B460B
:10A1D00010B0324620462946BDE8F04D00F002BDE1
:10A1E00000224FF08043204600F01AF902460B4649
:10A1F0002046294600F0D0F906460F46009800F0A8
:10A20000BCFBCDE9040132463B461046394600F01E
:10A21000DFFB0C9069480C9A4044019009910B4671
:10A22000104600F0D5FB8246024665488B46C8F1D1
:10A2300051080B4608F5D72803217844FFF7A8FEFC
:10A2400052465B4600F0C4FB0A905E480D915246B0
:10A250005B4604217844FFF79BFE099B0C9A00F0B3
:10A26000B7FB844601980D9B40EA080860460A9AAD
:10A2700000F0D6F883460891B8F1000F4EDD4FF09C
:10A28000FF322046294600F0CDFD22462B4600F045
:10A290009FFB804600988A4660B3DDE90401414A8D
:10A2A000414B00F095FB099100905A4640465146BB
:10A2B000089B00F0B5F832463B4600F089FB099B4D
:10A2C000009A00F0ADF84246534600F07FFC22466B
:10A2D0002B4600F087FC04460D46DDE90401334AB5
:10A2E000334B00F075FB10B022462B46BDE8F04D15
:10A2F00000F078BC5A464046089B00F091F8324680
:10A300003B4600F065FB4246534600F05FFC10B050
:10A3100022462B46BDE8F04D00F058BC009840B3F3
:10A32000DDE904011F4A204B00F052FB80468A46BB
:10A330005A4620462946089B00F054FC32463B46CC
:10A3400000F046FB4246534600F04CFC22462B46AA
:10A3500000F048FC04460D46DDE90401134A144BA5
:10A3600000F036FB10B022462B46BDE8F04D00F061
:10A3700039BC0B465A462046294600F033FC32468B
:10A380003B4600F025FB10B022462B46BDE8F04DC1
:10A3900000F01CBC0000F07F645F09000000F03F8B
:10A3A00032260000763C7935EF39EA3D0000E0FEC8
:10A3B000422EE63F5555D53F0000E03F86EBF9FFC2
:10A3C000CA240000C824000010B500290AD008786B
:10A3D000002807D005487844FFF7BEF9002801D0CF
:10A3E000002010BD0248784410BD00009E280000E7
:10A3F0009628000010B500290AD00878002807D058
:10A4000005487844FFF7A8F9002801D0002010BDC6
:10A410000248784410BD0000822900007A2900001B
:10A4200010B591EA030F48BF83F0004300F1E283C7
:10A43000841A71EB030C05D2121943EB0C03001BB9
:10A4400061EB0C01DFF824E14FEA1154A4EB135C3B
:10A450001EEA430F18BF9EEA445F73D023EA0E033F
:10A46000DCF1200E21EA045143F4801332D322FAA6
:10A470000CFE10EB0E0023FA0CFE41EB0E01CCF1AA
:10A48000200E03FA0EFE10EB0E0051F10001B1F5A3
:10A49000801FCCF1200E32D201EB045112FA0EF2E1
:10A4A000BDE8104058BF7047401C38BF5FEA420209
:10A4B00018BF7047002814BF20F0010041F10001CF
:10A4C0004FEA410313F5001F38BF7047A1F1C041A7
:10A4D00000F076BB012A43EB0302ACF1200CDCF167
:10A4E0001F0E32BF4FF0000E23FA0CF310EB0300E7
:10A4F00041EB0451B4EB115FD0D0A1EB045101F555
:10A50000801149085FEA300001EB04510ED350F18D
:10A51000000038BF12FA0EFE08D1BDE81040C9E7AE
:10A52000401C38BF5FEA4202CAD1C3E7BDE8104011
:10A530004FEA410313F5001F38BF7047A1F1C04136
:10A5400000F03EBB9EEA445F08D011EA5E0FBDE812
:10A55000104004BF01F0004100207047BDE81040EA
:10A5600070B500F0DFFA00BF64FBBE3E0000E0FF04
:10A5700002494FF0000000F023BC00BF0000F87F4C
:10A58000491058BFC1F140415B1058BFC3F140436F
:10A590008B42EFF3008070472DE9C04130B4DFF803
:10A5A000A0C23CEA111418BF3CEA131400F0EC807E
:10A5B00081EA03051CEA111444EAD57418BF1CEAA9
:10A5C000131500F0C780A4EB05044FF0004545EAE1
:10A5D000C12145EAC32341EA505143EA525304F1F1
:10A5E0007F74994204F500344FEAC0204FEAC2223A
:10A5F00008BF904200F09C804FEA13650FF24016AE
:10A60000765D4FEA134506FB05F7C7F1807706FB39
:10A6100007F74FEAD737A7FB03687642C8F58038BB
:10A62000A7FB06CE38BFA8F1010807FB08E64FF0EC
:10A63000000EA6FB028CE6FB03CEDCF1000CCEF193
:10A64000004E38BFAEF1010EA6FB0C584FF00007CC
:10A650004FF00005E6FB0E87A1FB08C6A0FB07CE66
:10A6600016EB0E0645F10005E1FB076515F1E04E1E
:10A670007EBFA4F580345FEA46066D4116F180077F
:10A6800045F100054FEA17274FEA066647EA0567D6
:10A69000A6F1DE46B6F1805F4FEA15251FD9384690
:10A6A00024F0010C05EBC471BCF1FE6F01EB0C1141
:10A6B00002D8F0BCBDE8008124425CBF01F5801ED9
:10A6C0009EEAC47F02D4F0BCBDE80081244238D4A5
:10A6D000F0BCA1F1C041BDE8004100F071BA4FEA01
:10A6E000D22242EA43524FEAD323A7FB02864FEA23
:10A6F000D02040EA415007FB03661EEA0E0F4FEAE6
:10A70000D12105FB026658BFA6EB0056B6EB0056FA
:10A710004FEA520E4EEAC37E18EB0E0E56EB530E66
:10A72000BDD518EB02085E417F1C55F10005B6E768
:10A730004FF480154FF000074FF000064FF000086F
:10A74000ADE7F0BC4FF0000001F1C04101F0004165
:10A75000BDE8008111EA0C1F0CEA131500D00CE0D3
:10A7600013EA0C1F00F025804FF00000F0BC81EAD6
:10A77000030101F00041BDE80081F0BCBDE80041EB
:10A7800081EA030100F01CBAF0BCBDE8004170B5DD
:10A7900000F0C8F9097EFC3E00F007B881EA030129
:10A7A0004FF0000001F00041704781EA030100F022
:10A7B00007BAF0BCBDE800414FF0000021497047E6
:10A7C000FFFDFBF9F7F5F4F2F0EEEDEBE9E8E6E476
:10A7D000E3E1E0DEDDDBDAD8D7D5D4D3D1D0CFCDFD
:10A7E000CCCBCAC8C7C6C5C4C2C1C0BFBEBDBCBB36
:10A7F000BAB9B8B7B6B5B4B3B2B1B0AFAEADACAB31
:10A80000AAA9A8A8A7A6A5A4A3A3A2A1A09F9F9E0A
:10A810009D9C9C9B9A9999989797969595949393BC
:10A82000929191908F8F8E8E8D8C8C8B8B8A898953
:10A8300088888787868585848483838282818180D6
:10A840000000FF070000F87F51EA030C17D41CF545
:10A85000801F58BFBCF5801F00F10680994218BFC9
:10A86000704708BF9042704707D711F5801F58BF47
:10A8700013F5801F19D499427047894270471CF51F
:10A88000801F08D5BCF5801FF7D58B4218BF7047D5
:10A8900008BF824270474FF4001C1CEB410F38BFC9
:10A8A0001CEB430F01D28B42704770B500F03AF9B0
:10A8B000922449004FF000514FF08053FFF760BEE3
:10A8C0004FEA41034FEA5353A3F58063D3F11E03CC
:10A8D000C8BFD3F1210C0CDD4FF0004242EAC12287
:10A8E00042EA505232FA03FC8CEAE17CACEBE170B4
:10A8F0007047102BC4BF0020704703F5787CBCF173
:10A90000FF3F04D06FF0004282EA2100704770B52B
:10A9100000F008F94992248000207047F2E7000017
:10A920004FEA1153A3F58063D3F11E03A8BFD3F1FF
:10A93000200C08DB4FF0004242EAC12252EA50529A
:10A9400032FA03F0704709420BD4102BC4BF002029
:10A95000704703F5787CBCF1FF3F05D04FF0FF3026
:10A9600070474FF00000704770B500F0DBF800BF93
:10A970004992248000207047F0E710F0004248BF61
:10A980004042B0FA80F310FA03F10AD0C3F11D037C
:10A9900003F580634FEA415002EB035202EBD121F1
:10A9A00070474FF000007047B0FA80F310FA03F1DF
:10A9B0000AD0C3F11D0303F580634FEA41504FEA0B
:10A9C000035202EBD12170474FF0000070470000A6
:10A9D000DFF848C170B51CEA111E1EBF1CEA131532
:10A9E0009EEA0C0F95EA0C0F00F06F8081EA0304D9
:10A9F00023EA4C134EEAD47E21EA4C1141F4801133
:10AA000043F48013AE44A1FB024CA0FB0365AEF1FE
:10AA10007F7E361955EB0C05A1FB034C4CF100036E
:10AA2000A0FB021C16EB0C06654153F10003094222
:10AA300018BF46F0010613F4007F0BD14FEA033133
:10AA40004FEA0530340341EA155140EA16506FF0E1
:10AA500003020AE04FEAC3214FEAC520F40241EAAB
:10AA6000555140EA56506FF0020202EB2E4201EBC4
:10AA7000025585EACE710AD05FEA440C18BF24F073
:10AA8000004450F1000041F1000120EAD47040F28E
:10AA9000FE7C624500D270BDA84214BF4FF08044D6
:10AAA0004FF04044002E08BF0024BEF1806FA8BFC5
:10AAB000A1F1C041BDE8704080F282804FF00000FB
:10AAC00001F1C04101F0004170479EEA0C0F0CEA11
:10AAD000131518BF95EA0C0F06D04FF0000081EA5D
:10AAE000030E0EF0004170BD00F01CF88900013E1D
:10AAF00000F007B800F009B84FEA430C5FEA5C5C6D
:10AB000008D081EA030100F05BB84FEA410C5FEA2C
:10AB10005C5CF6D14FF00000014970470000FF0770
:10AB20000000F87F0EF1020E2EF0030E5EF8046BAB
:10AB3000364205D4012A43EB030515F5001F12D850
:10AB4000012841EB010C1CF5001F0CD80ED14FEA77
:10AB5000D17C15F5001F0CEB4C0C0CF1020C08BF5E
:10AB60004CEBD37C04E04FF0080C01E04FEAD37CBF
:10AB70000CEB4C0526FA05F606F00706B6F1040CB8
:10AB800006D20EEB860CBDE870404CF0010C60471D
:10AB9000DFE80CF0090B02024FF000414FF000001B
:10ABA000A1F5002170BD19461046012851EB0104A2
:10ABB00018BFD4F5001484BF002001F0004170BD1F
:10ABC0000808A0F500114FEA3101704791EA030F20
:10ABD00010B581F000413FF52BAC83F0004300F04D
:10ABE00009B8000010B591EA030F48BF83F0004395
:10ABF0003FF51EAC841A71EB030C07D212198CF0CE
:10AC0000004C43EB0C03001B61EB0C01DFF8A4E1EB
:10AC10004FEA1154A4EB135C1EEA430F18BF9EEADF
:10AC2000445F00F0B08023EA6E03524221EA0451EF
:10AC3000C3EB6E0338BF5B1EDCF1200E25D322FA76
:10AC40000CFE10EB0E0043FA0CFE41EB0E01CCF1B2
:10AC5000200E03FA0EFE10EB0E0051F10001CCF1B4
:10AC6000200E29D412FA0EF201EB0451BDE8104077
:10AC700058BF7047401C1CBFB2F1004F70470028FE
:10AC80000CBF491C20F00100704712EB020E43EB91
:10AC9000030218BF4FF0010E4EEA4202ACF1200C45
:10ACA000DCF11E0E54D943FA0CFE10EB0E0051F1EC
:10ACB000FF31CCF11E0ED5D50EF1010E12FA0EFEAB
:10ACC000404141EB010101EB445C5FEA5C5C10D95F
:10ACD00010EBDE7001EB045138BFBEF1004FBDE850
:10ACE000104018BF704700280CBF491C20F001001D
:10ACF000704730D24FEAD42C11F5001124F40064CF
:10AD00001BD0B1FA81F20B3AA41AA41ED2F120038F
:10AD1000914030FA03F31943904001EBCC71002CC1
:10AD200001EB0451BDE81040A8BF704701F1C041DC
:10AD30004FF0000001F000417047B0FA80F310FAC4
:10AD400003F100D110BDE41A173C4805C90AE4E735
:10AD500001EB045110BD491001EB0451BDE8104056
:10AD60004FEA300002E04FF0000170474A0008BF90
:10AD70000042F8D0B2F5001F28BF704701F0004133
:10AD80004FF0000070479EEA445F07D011EA5E0F63
:10AD9000BDE8104004BF002100207047BDE810400E
:10ADA00070B5FFF7BFFE00BF40DFF63E83F0004105
:10ADB000104670470000E0FFFEF7D4B8FEF708BA6F
:10ADC0000CF00F03092B08BF082000F059800A2B54
:10ADD0000BD0082B18BF704708BF1CF0400F0AD0DB
:10ADE0004FF000004FF0000170471CF0400F18BFFB
:10ADF0004FF0004070471CF0100F08D020F0704357
:10AE000000F07F4242EAD3014FEA4370704700F0FE
:10AE1000604021F07F4242EA000201F07F4040EAB8
:10AE2000727070474FF0FF0C4CF4E06C1CEA115349
:10AE30001CBF9CEA030C9445C2BFDA4201EB0251ED
:10AE40007047002B0DD0BCF1000F0FD0002A01F08D
:10AE50000041A4BF41F0E04141F07F614FF00000AC
:10AE6000704701F000414FF00000704750EA013395
:10AE70004FF09B0C18BF4CF0806C7FF479AB70479F
:10AE80001CF4801F11D01CF4E02F03D06FEACC31EA
:10AE9000490070474FF04050EFF3008222F07042BB
:10AEA00042EA000282F3008870474FF000007047CA
:10AEB0000103070F1FFFFF1F0F0703010000000022
:10AEC00000E0E00000FCFC000000000000000000CA
:10AED00000000000003F3F0000383800003F3F0006
:10AEE000003F3F00003F3F00000000000000000066
:10AEF0000000F808E8E8E8E80808E8E8E8E80808F2
:10AF0000E8E8E8E80808F820E00000000000000099
:10AF100000001F101717171710101717171710100A
:10AF20001717171710101F0407000000000000007B
:10AF3000C05F5555D5755555555FC0000809090BBB
:10AF40000505050B09090000EACC0011F200FC24FC
:10AF500024E41FE485660000070A0700020B0403CF
:10AF6000040E00B3CF0012D2FE5190122400FF80D5
:10AF7000800001000F00000101010F000000BFC6AA
:10AF8000008888FF4824E4243F24E4040000080FDC
:10AF9000000808050205080800BCBC00000000000D
:10AFA0000000000000000000000000000000363635
:10AFB000000000000000000000000000A3BA000034
:10AFC0000000000000000000000000000000000081
:10AFD000005838000000000000000000000000A33E
:10AFE000AC000000000000000000000000000000B5
:10AFF00000000000182424180000000000000000D9
:10B000000000A1A300000000FE00000000000000FE
:10B0100000000000000000003300000000000000FD
:10B020000000000000A3A100000038340282C27CAE
:10B03000380000000000000000000000003737006A
:10B040000000000000000000A3BF00008080BEAA36
:10B05000AAAAEAAAAAAABE80800000048584945CF9
:10B0600054272424544C4484050400EACC00404274
:10B07000CC0000F888888808FF0809CA080000008A
:10B080003F90681F10209F4027182641F000B3CF43
:10B09000002424A4FEA3220022CC0000FF00000014
:10B0A00000080601FF00010404040404FF02020278
:10B0B00000BFC600101010FF109008888888FF8815
:10B0C000888808000444827F01808040432C102837
:10B0D00046818000BCBC001010FF109000FE525250
:10B0E000D25252525E000042827F8140308F929352
:10B0F00092FE9293968000CED50000002424242452
:10B1000024FC222222232200000002020202024228
:10B11000827F0202020202020200CAD6000000F090
:10B1200010101010FF10101010F000000000000FA1
:10B1300004040404FF040404040F000000D6D0003B
:10B14000000000000001E21CE00000000000000020
:10B15000804020100C03000000030C304080800071
:10B16000C8EB0000FE022242827202224282720278
:10B17000FE000000FF100806010E100806014E80B8
:10B180007F0000CDF800404042CC000444645C479E
:10B19000F444444404000040201F204444444444F8
:10B1A0007F4444444400C1AC00101010FF105044D0
:10B1B0005465C64464544440000444827F01828242
:10B1C0004A562322524E820200BDD3000000FE22C6
:10B1D0002222FE00FE828292A29E000080601F0258
:10B1E00042827F00FF402F102C438000B7FE0000FA
:10B1F0000090884C57A42454548C84000000000113
:10B20000018042221A07024282423E01010100CE21
:10B21000F10080809E9292929EE0809EB2D2929E99
:10B2200080000808F4949292F10001F2929494F84C
:10B230000800C6F7001060028C0008080809FA0828
:10B24000080808000004047E0140404141417F415C
:10B250004141414000D7A200808080FE8282FE8072
:10B2600080FE8282FE8080000080403F00407F8020
:10B27000601F40807F000000B2E1000000F8888875
:10B2800088880808FF08090AC8080080601F0010A5
:10B29000201F80402116182641F800B3C900080875
:10B2A00008F80808081010FF101010F00000103007
:10B2B000101F088848300E014080403F0000B9A6AA
:10B2C000000040301E101010FF1010101010000071
:10B2D0000081814121110D0301030D112141818163
:10B2E00000CAA70000FE02FA02FE4020D817101084
:10B2F000F01010008047300F1067804021160816AC
:10B3000021408000B0DC00080889EA1888000404A5
:10B31000FC040404FC0000020100FF018640201828
:10B32000074080403F0000B3F5001010F01F10F000
:10B330000040E05847405060C000402215081621E8
:10B340000000FE42424242FE0000CABC0000806093
:10B35000F807000000FF4020100804000001000072
:10B36000FF000402013F40404040407800BBAF0076
:10B37000040444C44F4444C424242FB424040400CB
:10B3800040442424150C04FE040C152424444000DD
:10B39000B2CB000000F8494A4C48F8484C4A49F8FA
:10B3A00000000010101312121212FF1212121213C8
:10B3B000101000B5A500404042CC0000FC24A4249D
:10B3C0002222A36200000040201F20584750484519
:10B3D000424548504000B7B5000000FE0202F2129C
:10B3E0001212F20202FE00000000007F202027243B
:10B3F00024242720207F000000BBD8000000223238
:10B400002AA6A26221110981010000000042221334
:10B410000B42827E02020A1223460000CFB50020B2
:10B4200030AC63300088C8A8998E88A8C8880022EC
:10B43000672212128040300F00003F40407100CD63
:10B44000B3008080848484FE82838280FF80808039
:10B45000800000804020180700000000FF0000006E
:10B460000000C9FD002030AC6330000202FE020281
:10B47000625AC60000226722121240308F80432C8D
:10B48000102C438000BCB60008C8B88FE8888840FC
:10B49000300FC8082818000008180808FF04844066
:10B4A000300E010E30408000C8ED00008060F807CB
:10B4B00080601C1010FF1010100000010000FF0041
:10B4C0000202020202FF0202020200BCFE00004071
:10B4D00042445840407F40405048C6000000004071
:10B4E00044444444444444444444FF000000B5B14F
:10B4F000000808E8292E28E80808C80C0BE8080806
:10B50000000000FF0949897F00000F40807F000094
:10B5100000C7B00000FE20203F2000FC24E42422CD
:10B5200023E20000807F0101FF80601F8041261818
:10B5300026418000B0E6000010101010D030FF301F
:10B54000D010101010000010080402090808FF08AD
:10B5500008090204081000B1BE00808080BEA2A2CB
:10B56000A2A2A2A2A2BE8080800000000006050464
:10B5700004044484443C00000000BAC5004040423A
:10B58000CC0040A09E8282829EA02020000000006D
:10B590003F908840432C10284641808000C9E80035
:10B5A000809090484C57242424544C448080800040
:10B5B000000000FF4949497F494949FF0000000058
:10B5C000B1B800008060F807000424242526242454
:10B5D000240400010000FF000000F94949494949DD
:10B5E000F90000D0C500000000FC545456555454D6
:10B5F00054FC0000000040300003394141455941EE
:10B60000417300083000CFA2000000007F49494983
:10B61000494949497F000000008141211D214181A4
:10B62000FF8989898989818100CAC70000028282D5
:10B63000422212FA0622224242820000010100FC4C
:10B6400044444445444444FC00000100B7F1000078
:10B6500010109010101116101010D0101000004093
:10B66000404040435C4040504C434040404000C15B
:10B67000A20000FE92929292FE0000FE020202FEE2
:10B680000000003F20100A04180000FF0004080713
:10B690000000BCB400003E22E2223E001088572485
:10B6A000548C000000407E403F22220001FE4242B6
:10B6B00042FE010100C2B700001088C433808242FC
:10B6C00022121A2622408000020100FF004042425E
:10B6D000427E424242424000BEB600404424A4940E
:10B6E0008C84FF848C94A4244440004040405F4AF2
:10B6F0004A4A4A4A4A4A5F40404000B2E9001010B4
:10B7000010FF10902020FF2010119610000004441C
:10B71000827F01004020130C142241F80000D5D292
:10B720000040445465C664544400FC4444C4424050
:10B730000020124A827F020A92601F0000FF000070
:10B7400000D0C20000FE0212929292FE92929212D9
:10B7500002FE000000FF40405F48484848485F4004
:10B7600040FF0000B9CC00008060F80780601C102A
:10B7700010FF1010100000010000FF000202020282
:10B7800002FF0202020200BCFE000414A444AF1433
:10B79000040404F40F2444040400124984423F8149
:10B7A00041310D030D3141818100BBF1000202FEE8
:10B7B000929292FE0206FC040404FC000008180F9A
:10B7C000080804FF048440271827408000C8A1000F
:10B7D000008060F807000424242526242424040083
:10B7E000010000FF000000F94949494949F90000FA
:10B7F000D0C500000000FC54545655545454FC006D
:10B800000000004030000339414145594141730077
:10B81000083000CFA2000040301E101010FF1010A2
:10B8200010101000000081814121110D0301030D52
:10B83000112141818100CAA70000FE02FA02FE40E8
:10B8400020D8171010F01010008047300F106780BC
:10B85000402116081621408000B0DC001010D0FFF7
:10B860009010804828090E0828488800040300FF2B
:10B8700000018080432C102C43808000D0A3000264
:10B88000FA8282FE804020504C434C5020400008F9
:10B89000184884443F404458414E6058474000D1C6
:10B8A000E900000202C2020202FE82828282820259
:10B8B00000004040407F4040407F4040404040408A
:10B8C0004000D5FD00080888C8380C0B0808E808B7
:10B8D0000808080800020100FF40414141417F4142
:10B8E0004141414000D4DA00020202020202FE029B
:10B8F0000242820202020200000000000000FF007B
:10B900000000000106000000CFC200909494F49F54
:10B910009494941010FF1012D4100020262524FEB9
:10B92000141414804027182641F000D4D800404257
:10B93000CC0000445454547F5454544440000000FC
:10B940007F201000FF15151555957F000000C7EBEF
:10B9500000804020180F88780808F8080808F800C8
:10B9600000001008844221100806014080403F007A
:10B9700000CEF00000FC2024A8FFA82400FC4444D2
:10B98000C4424000003F2221202F20A3601F00005E
:10B99000FF000000B6CF000000F888888888FF8884
:10B9A000888888F800000000001F080808087F88C1
:10B9B0008888889F80F000B5E700000000F112142D
:10B9C0001010101412F10000000040300003394143
:10B9D00041455941417300083000D7DC0040201038
:10B9E000EC27242424E40404FC00000000000000F0
:10B9F0003F424242424344484740700000B0FC008E
:10BA000090523410FF10345280708F0808F80800EC
:10BA1000829A566322528E008040330C334080005D
:10BA2000CAFD0080828282828282E2A2928A86821B
:10BA3000808000000000000040807F0000000000C7
:10BA4000000000D7D30000FE92929292FE0000FE0A
:10BA5000020202FE0000003F20100A04180000FF4E
:10BA6000000408070000BCB40000083000FF008894
:10BA700084532212CA0600000004040201FF0002DF
:10BA80000A1242827F02020200BDAB00404042CC5B
:10BA900000202222A2622222222000000040201F39
:10BAA00020444E4544444445464C4000D4CB00001D
:10BAB0001088C4330040424242C242424240000227
:10BAC0000100FF0000000040807F0000000000D067
:10BAD000D000101010FF1090001010FF1010F00098
:10BAE00000000444827F018040211A0718003F4073
:10BAF000F000D6B400001088C4330040424242C275
:10BB00004242424000020100FF0000000040807FEE
:10BB10000000000000D0D0000000FC044484042594
:10BB2000C604040404E4040040300F4040414E4089
:10BB30004063504C43404000D3A60000100894934B
:10BB4000929292929A9690F0000000403004748491
:10BB5000848CB4848484E407106000BCB100242485
:10BB6000A4FE2322003E22222222223E00000806BA
:10BB700001FF0106404949497F4949494100B3CC89
:10BB8000000000FC040404141556945434140404F6
:10BB90000040300F0001010141817F0101010503D7
:10BBA00000D0F20000E000FF10200888780F08E8BD
:10BBB00008088800010000FF00100C8344231807C8
:10BBC00018628100BBD600201008F7545454545416
:10BBD0005454F404040000809090494D57252525C5
:10BBE000554D4580808000B8B4001010D0FF9014EF
:10BBF000E4AFA4A4A4AFE4040000040300FF0089A0
:10BC00004B2A1A0E1A2A4B888000C4A300101090E9
:10BC1000909090901010FF101011161000002060EE
:10BC2000203F10101000030C102040F800CABD0087
:10BC300000080808080809FA0808080808080000A9
:10BC4000404041414141417F4141414141404000EB
:10BC5000D6F7004044C4444444401010FF10101074
:10BC6000F00000103C131014B840300E014080402A
:10BC70003F0000B6AF00101010FF10105020D81772
:10BC80001010F0101000007F2121217F804021162C
:10BC9000081621408000B9CA0000FE0222DA061010
:10BCA000D2565A535A56D2100000FF0810080710F7
:10BCB000171515FD1515171000D5CF0002FE92922D
:10BCC000FE0200101116F01413100000101F0808D7
:10BCD000FF048141310D030D31418100C1AA0000F3
:10BCE0000022322AA6A2622111098101000000006F
:10BCF0004222130B42827E02020A1223460000CF28
:10BD0000B5000000FE02020202020202020202026A
:10BD1000020080601F000000000000000000000022
:10BD20000000B3A700102C2424A4A465A624242476
:10BD300024A4340C0040494929241452897F040A60
:10BD40001110202000BCD200000000000000000004
:10BD5000002F000000000700070000147F147F146C
:10BD600000242A7F2A1200626408132300364955F2
:10BD7000225000000503000000001C2241000000CA
:10BD800041221C000014083E08140008083E080860
:10BD9000000000A0600000080808080800006060BB
:10BDA0000000002010080402003E5149453E0000FA
:10BDB000427F4000004261514946002141454B31DC
:10BDC000001814127F10002745454539003C4A49A8
:10BDD000493000017109050300364949493600061A
:10BDE0004949291E00003636000000005636000082
:10BDF00000081422410000141414141400004122FD
:10BE0000140800020151090600324959513E007CD4
:10BE10001211127C007F49494936003E41414122BE
:10BE2000007F4141221C007F49494941007F0909A7
:10BE30000901003E4149497A007F0808087F000057
:10BE4000417F4100002040413F01007F0814224112
:10BE5000007F40404040007F020C027F007F0408CA
:10BE6000107F003E4141413E007F09090906003E26
:10BE70004151215E007F091929460046494949314F
:10BE80000001017F0101003F4040403F001F204072
:10BE9000201F003F4038403F006314081463000730
:10BEA0000870080700615149454300007F41410087
:10BEB00000552A552A55000041417F000004020127
:10BEC0000204004040404040000001020400002005
:10BED00054545478007F4844443800384444442043
:10BEE00000384444487F00385454541800087E09F0
:10BEF00001020018A4A4A47C007F080404780000B8
:10BF0000447D4000004080847D00007F1028440074
:10BF10000000417F4000007C04180478007C080485
:10BF2000047800384444443800FC242424180018C1
:10BF3000242418FC007C08040408004854545420AD
:10BF400000043F444020003C4040207C001C204036
:10BF5000201C003C4030403C004428102844001C79
:10BF6000A0A0A07C004464544C4414141414141471
:10BF700000000000000000000000000000000000C1
:10BF8000000000F800000000000000333000000056
:10BF900000100C06100C060000000000000000005D
:10BFA00040C07840C0784000043F04043F040400CF
:10BFB000007088FC08300000001820FF211E0000DF
:10BFC000F008F000E018000000211C031E211E00F4
:10BFD00000F00888700000001E212324192721107A
:10BFE00010160E000000000000000000000000001D
:10BFF000000000E0180402000000000718204000C4
:10C0000000020418E00000000040201807000000B3
:10C01000404080F0804040000202010F0102020017
:10C02000000000F0000000000101011F01010100FB
:10C03000000000000000000080B070000000000060
:10C0400000000000000000000001010101010101E9
:10C050000000000000000000003030000000000080
:10C060000000000080601804006018060100000055
:10C0700000E010080810E000000F102020100F0052
:10C08000001010F8000000000020203F20200000D9
:10C090000070080808887000003028242221300031
:10C0A00000300888884830000018202020110E0039
:10C0B0000000C02010F8000000070424243F2400E2
:10C0C00000F80888880808000019212020110E00B7
:10C0D00000E0108888180000000F112020110E00C9
:10C0E00000380808C83808000000003F00000000C1
:10C0F0000070880808887000001C222121221C0082
:10C1000000E010080810E0000000312222110F00AA
:10C11000000000C0C000000000000030300000003F
:10C1200000000080000000000000806000000000AF
:10C1300000008040201008000001020408102000C8
:10C140004040404040404000040404040404040013
:10C1500000081020408000000020100804020100A8
:10C16000007048080808F0000000003036010000A8
:10C17000C030C828E810E0000718272423140B005B
:10C180000000C038E0000000203C230202273820D5
:10C1900008F8888888700000203F202020110E00B9
:10C1A000C0300808080838000718202020100800B0
:10C1B00008F808080810E000203F202020100F0099
:10C1C00008F88888E8081000203F20202320180065
:10C1D00008F88888E8081000203F200003000000CD
:10C1E000C03008080838000007182020221E02006E
:10C1F00008F808000008F808203F210101213F202D
:10C20000000808F8080800000020203F2020000057
:10C2100000000808F8080800C08080807F00000047
:10C2200008F888C028180800203F20012638200080
:10C2300008F8080000000000203F202020203000E7
:10C2400008F8F800F8F80800203F003F003F200001
:10C2500008F830C00008F808203F200007183F0009
:10C26000E01008080810E0000F10202020100F0038
:10C2700008F808080808F000203F2101010100002B
:10C28000E01008080810E0000F18242438504F0070
:10C2900008F8888888887000203F2000030C302030
:10C2A00000708808080838000038202121221C006E
:10C2B000180808F8080818000000203F20000000B7
:10C2C00008F808000008F808001F202020201F00A0
:10C2D0000878880000C83808000007380E01000000
:10C2E000F80800F80008F800033C0700073C0300CA
:10C2F000081868808068180820302C03032C302030
:10C300000838C800C83808000000203F200000009E
:10C3100010080808C83808002038262120201800F6
:10C32000000000FE020202000000007F40404000CA
:10C33000000C30C000000000000000010638C00002
:10C3400000020202FE000000004040407F000000AA
:10C3500000000402020204000000000000000000CF
:10C3600000000000000000008080808080808080CD
:10C3700000020204000000000000000000000000B5
:10C3800000008080808000000019242222223F20AB
:10C3900008F8008080000000003F112020110E00EE
:10C3A0000000008080800000000E1120202011007D
:10C3B000000000808088F800000E112020103F202F
:10C3C0000000808080800000001F222222221300B3
:10C3D000008080F0888888180020203F20200000FE
:10C3E0000000808080808000006B949494936000B3
:10C3F00008F8008080800000203F210000203F20BE
:10C4000000809898000000000020203F20200000BD
:10C41000000000809898000000C08080807F0000AD
:10C4200008F8000080808000203F24022D3020008A
:10C43000000808F8000000000020203F2020000035
:10C440008080808080808000203F20003F20003F4F
:10C450008080008080800000203F210000203F205D
:10C460000000808080800000001F202020201F000E
:10C47000808000808000000080FFA12020110E003D
:10C480000000008080808000000E112020A0FF802E
:10C49000808080008080800020203F2120000100DB
:10C4A0000000808080808000003324242424190030
:10C4B000008080E0808000000000001F202000003D
:10C4C0008080000000808000001F202020103F207E
:10C4D000808080000080808000010E30080601000E
:10C4E00080800080008080800F300C030C300F00B3
:10C4F00000808000808080000020312E0E312000DE
:10C50000808080000080808080818E70180601000D
:10C5100000808080808080000021302C222130002B
:10C5200000000000807C020200000000003F40404C
:10C5300000000000FF00000000000000FF000000FD
:10C540000002027C800000000040403F000000002C
:10C5500000060101020204040000000000000000C7
:10C560006001000001000000200000002000000029
:10C57000002C0000200000000306010B0405020946
:10C5800025262734350000010001000C00010000C1
:10C59000004000000000020000000400000008004D
:10C5A00000001000445B0020445C0020445D00203B
:10C5B000446900200B0000000C0000000D0000008A
:10C5C0000E0000000F00000010000000110000002D
:10C5D00038000000390000003A0000003B00000075
:10C5E0003B000000000102030405060004000000F7
:10C5F00008000000100000002000000040000000C3
:10C60000800000000001000001000200040008009A
:10C61000100020004000800000010002000400081B
:10C6200000100020004000800001020304050607FE
:10C6300008090A0B0C0D0E0F01000000020000009B
:10C6400004000000080000001000000020000000AE
:10C650004000000080000000000100000002000017
:10C66000000400000008000000100000002000008E
:10C670000040000000800000060708090A1717178D
:10C680001717282828282828000303060104060273
:10C69000050003051F1C1F1E1F1E1F1F1E1F1E1F20
:10C6A0001C1D1E3236370000010000000200000091
:10C6B000040000000800000010000000200000003E
:10C6C00000000000000000003031323334353637CE
:10C6D00038394142434445464030580030313233C6
:10C6E00034353637383961626364656640307800C6
:10C6F000040000080000000000000002000100002B
:10C70000100000000000000004FA97999999D93FA1
:10C71000AF788E1DC571CC3F9FC678D0099AC33FB4
:10C72000935555555555E53F599322942449D23F89
:10C73000DE03CB966446C73F44523EDF12F1C23F50
:10C74000000000000000000030313233343536374D
:10C750003839616263646566787000303132333431
:10C760003536373839414243444546585000000079
:10C7700002400000000000A0000000000540000092
:10C78000000000C8000000000C4000000000409CB9
:10C7900000000000194000000020BCBE00000000A6
:10C7A00034400000BFC91B8E00000004B5400000EB
:10C7B000504BCFD06607E2CF010000006C41000073
:10C7C0003E8251AADFEEA73401000000D9420000EA
:10C7D000DCB5A0E23A301F97FFFFFFFFB445000031
:10C7E000FD25A0C8E9A3C14FFFFFFFFFFF3F0000E9
:10C7F0000000008000000000FF3F000000000080FB
:10C80000000000000D0A2A2A2A2A2A2A2A2A2A2A6D
:10C810002A2A2A2A2A2A2A2A2A2A2A2A2A2A2A2A78
:10C820002A2A2A2A2A2A2A2A2A2A2A2A2A2A2A2A68
:10C830002A2A2A2A2A2A2A2A2A2A2A2A2A2A2A2A58
:10C840002A2A2A2A000000000D0AB0E6C8A8B9E981
:10C85000CAF4203A20EACCB3CFBFC6BCBC203230E9
:10C8600031372F382D323032372F38202E09090931
:10C870000909090D0ABCBCCAF5D6A7B3D6203A20CF
:10C880004D722E2057616E67202031333633353597
:10C890003133363138202E00415445300D0A000026
:10C8A00041542B4342430D0A0000000041542B51D8
:10C8B000504F57440D0A000041542B474D520D0A6A
:10C8C0000000000041540D0A0000000041542656AB
:10C8D0000D0A0000415426570D0A0000453A203148
:10C8E000000000002B434243000000004F4B0000BB
:10C8F000504F574552454420444F574E00000000CA
:10C900004552524F5200000041542B514943534766
:10C91000503D25642C312C222573222C22222C22DE
:10C92000222C310D0A00000041542B435245473D53
:10C93000320D0A0041542B43475245473D320D0A00
:10C940000000000041542B435245473F0D0A0000B0
:10C9500041542B43475245473F0D0A0041542B5148
:10C96000494143543F0D0A0041542B51434349442C
:10C970000D0A000041542B514E57494E464F0D0AA7
:10C980000000000041542B4353510D0A00000000E9
:10C9900041542B514944454143543D25640D0A00FF
:10C9A00041542B51494143543D25640D0A00000078
:10C9B0002B435245473A00002B43475245473A0024
:10C9C0002B514E57494E464F3A0000002B435351CE
:10C9D0003A0000002B51494143543A002B51434344
:10C9E0004944000041542B5149434C4F53453D2588
:10C9F000642C31300D0A000041542B51494F5045F1
:10CA00004E3D312C25642C22544350222C22257378
:10CA1000222C25642C25642C310D0A0041542B5105
:10CA20004953544154453D312C25640D0A00000002
:10CA300041542B514953454E443D25642C25640DEA
:10CA40000A0000002B514953544154453A0000005C
:10CA50002B51494F50454E3A000000003E00000067
:10CA600053454E44204F4B002573000041542B5139
:10CA70004654504346473D226163636F756E74228E
:10CA80002C222573222C222573220D0A000000007F
:10CA900041542B5146545052454E414D453D22255F
:10CAA00073222C222573220D0A00000041542B51C1
:10CAB0004654504357443D222573220D0A0000007E
:10CAC00041542B5146545053495A453D2225732217
:10CAD0000D0A000041542B514654504E4C53543DC6
:10CAE000222573220D0A000041542B514654505008
:10CAF00057440D0A0000000041542B514654504346
:10CB00004C4F53450D0A000041542B514654504C94
:10CB1000454E0D0A0000000041542B51465450531D
:10CB20005441540D0A00000041542B5146545043C7
:10CB300046473D22636F6E746578746964222C25C4
:10CB4000640D0A0041542B514654504346473D2240
:10CB50007472616E736D6F6465222C25640D0A001A
:10CB600041542B514654504346473D2266696C65FB
:10CB700074797065222C25640D0A000041542B51F4
:10CB80004654504F50454E3D222573222C25640DAE
:10CB90000A00000041542B514654504346473D2261
:10CBA00072737074696D656F7574222C25640D0A3B
:10CBB0000000000041542B514654504745543D223B
:10CBC0002573222C22434F4D3A222C25642C2564B8
:10CBD0000D0A00002B514654505057443A20300063
:10CBE0002B5146545052454E414D453A203000009D
:10CBF0002B5146545053495A453A2030000000000A
:10CC00002B51465450535441543A203000000000F8
:10CC10000D0A4F4B0D0A0D0A2B51465450474554EF
:10CC20003A2030002B514654504E4C53543A203049
:10CC3000000000002B514654504357443A20302CFA
:10CC4000300000002B51465450434C4F53450000D8
:10CC50002B4F4B00A0CD000800000020F406000080
:10CC60006C010008F4CF0008F40600207C95000059
:10CC7000C80100081001000043000000F8FFFFFF9A
:10CC800000404040404040404040414141414140DF
:10CC90004040404040404040404040404040404094
:10CCA0004005020202020202020202020202020223
:10CCB0000220202020202020202020020202020228
:10CCC0000202909090909090101010101010101080
:10CCD000101010101010101010101010020202028C
:10CCE00002028888888888880808080808080808D0
:10CCF00008080808080808080808080802020202CC
:10CD000040000000000000000000000000000000E3
:10CD10000000000000000000000000000000000013
:10CD20000000000000000000000000000000000003
:10CD300000000000000000000000000000000000F3
:10CD400000000000000000000000000000000000E3
:10CD500000000000000000000000000000000000D3
:10CD600000000000000000000000000000000000C3
:10CD700000000000000000000000000000000000B3
:10CD8000000000001C00000043000000F8FFFFFF4F
:10CD90000C0000000E0000000F0000002E0000003C
:10CDA00021057D0341424D000E7453686F7033348A
:10CDB00034373934373439400F015A3132312E3457
:10CDC000312E37392E38371215057C2F41424D222E
:10CDD00030E995110510581B701713ACC824088A48
:10CDE000021AF0081AFF011112C91B0804103201BF
:10CDF0001AC414320AAAEC1C2203191F111ACC14EB
:10CE0000190B114BF8CB1C1ADC101A043529145AD3
:10CE1000981CB938193532040A15D41C32050A1584
:10CE2000B81C32065AA08CDAE41C411A680C29405E
:10CE30001ADC08A9A829C41A280C091254293B5A3B
:10CE4000441CAAB038191929140A15343829C45AAF
:10CE5000501CDAB83829845A741CAAC01C198929B4
:10CE6000C45A841CDACC3832070A1508702A08FC28
:10CE7000190C1ADC5DB91C195432091A900C1A905D
:10CE80000CE91C320A5A5C54DAD470411AF80C2AA4
:10CE9000C8CCCACA381903111AE40C0A11648C29C7
:10CEA0003B1A1C3029E8AA4438191929681A301489
:10CEB0002A1478D95432045A681CDA601C411328A9
:10CEC000CB2A08B0E970291F1A6C3009121C298C72
:10CED0000A156038298C0A15441C298C0A15941CE3
:10CEE00029D81A7C1C0A11C81C32065A183811CAD3
:10CEF000CC1C32075AACA8DA341C32085AE81C1A87
:10CF0000D440A91C2A0914591CDA243829145AC0FF
:10CF10001CDAF038320B1AB4143228AA1038220165
:10CF2000320C5A08A8DA5054320D1A90543214DADE
:10CF3000E054320E5AF81CDA443813AD3A1B08DFBD
:10CF40000413402C3220146840581A2009E2681853
:10CF50000801020209020A0A8110090102030A03F8
:10CF60000B0B0214380140124412401A48041A4CA8
:10CF70000412501B4004141A04141A04141A041442
:10CF80001351431B085B041A65041A6F044112080D
:10CF90001C02401C041A30041A44041A58041A6C67
:10CFA000041A800419911B401C041A30041A44040A
:10CFB0001A5804111A08681A0C041A10041A1404D6
:10CFC0001A18041A1C041A2004011612401A040428
:10CFD0001A08041A0C041A100412143D4002040624
:10CFE0008019C02A040415060708098CA24A04E225
:04CFF00049140000E0
:0400000508000131BD
:020000040801F1
:10C00000B08E0020B9C20108D9790208DB79020894
:10C01000ED790208EF790208F179020800000000CA
:10C02000000000000000000000000000CBC201087A
:10C03000F379020800000000CFC20108A14D0208F8
:10C04000D3C2010843560208D3C201085F46020862
:10C05000D3C20108D3C201081144020831440208C6
:10C060005344020873440208954402080B3E020838
:10C070004D3E02088F3E0208DB3E0208F13F0208F7
:10C080004140020891400208D3C20108D3C201080E
:10C09000D3C20108D3C20108D3C20108B5440208C3
:10C0A000D3C20108D3C20108D3C20108D3C2010818
:10C0B000A94F0208CB4F0208ED4F0208D3C2010876
:10C0C000D3C20108D3C20108D3C20108D3C20108F8
:10C0D000D3C20108CB3802083B390208AB39020849
:10C0E000F744020897460208D3C20108D3C20108E8
:10C0F000D3C20108D3C20108D3C20108D3C20108C8
:10C10000D3C20108D3C201080F500208D3C20108EC
:10C110001B3A02088F3A02083150020853500208B5
:10C12000E14002082F4102087F410208CB4102088A
:10C1300000F002F800F0B0F80AA090E8000C824489
:10C140008344AAF10107DA4501D100F0A5F8AFF266
:10C15000090EBAE80F0013F0010F18BFFB1A43F0E5
:10C160000103184770170100901701000A444FF0AF
:10C17000000C10F8013B13F0070408BF10F8014B46
:10C180001D1108BF10F8015B641E05D010F8016B8B
:10C19000641E01F8016BF9D113F0080F1EBF10F8EF
:10C1A000014BAD1C0C1B09D16D1E58BF01F801CB12
:10C1B000FAD505E014F8016B01F8016B6D1EF9D595
:10C1C0009142D6D3704700000023002400250026AA
:10C1D000103A28BF78C1FBD8520728BF30C148BFEA
:10C1E0000B6070476E290BF0B98770290CF09F80A7
:10C1F00066290FF0CA8465290FF0C78467290FF0FC
:10C20000C48461290FF0C38403681B0A28BF41F06E
:10C21000800169290BF0668764290BF06387752913
:10C220000BF060876F290CF02C8078290CF06B8064
:10C23000E9290CF02786E4290CF02486F5290CF076
:10C240002186EF290CF02980F8290CF06A80036818
:10C25000DB0928BF41F0800163290CF0DE857329DA
:10C260000CF0E385E3290CF00186F3290CF0068637
:10C27000002070471FB50CF0C1FE04000020002113
:10C280000EF0AEFD401C6060002000210EF0BEFDEF
:10C29000E0601FBD10B510BD0DF09CF91146FFF711
:10C2A000E9FF00F02EFC0DF0C8F903B4FFF7F2FF30
:10C2B00003BC07F0DAF80000094880470948004746
:10C2C000FEE7FEE7FEE7FEE7FEE7FEE7FEE7FEE746
:10C2D000FEE7FEE704480549054A064B70470000A3
:10C2E000FF7A020831C10108B05E0020B08E002044
:10C2F000B06E0020B06E002010B508F0F9FEF548D1
:10C300000078C0074CD0F44806F07AFB032804D02C
:10C31000BDE81040F1A006F0DFBCEF49F3A03231D8
:10C3200006F0DAFCEC49F5A006F0D6FCF648EA4C3B
:10C330004178E1B994F832103039092917D894F8C6
:10C3400035103039092912D894F8371030390929B5
:10C350000DD821783039092909D8E17830390929EF
:10C3600005D861793039092901D801214170DA49AC
:10C37000E27D0B31E5A006F0AFFCD74994F825200B
:10C380001831E5A006F0A8FCD349E6A0263106F056
:10C39000A3FCD149BDE810402C31E5A006F09CBCBF
:10C3A00010BD38B508F0A4FE4FF4007006F056FC3E
:10C3B0000446002000906A462146E14806F0B8FD98
:10C3C000B0B920460CF00DF9217828290CD194F849
:10C3D0002510262908D1221812F8051C242903D17A
:10C3E00012F8031C292907D02146D6A006F074FCB8
:10C3F000204606F06DFC38BD6278412A15D0632ACC
:10C4000008D02146D7A006F067FCDEA1522002F03A
:10C410009AFCEDE782B22146E14806F03AFD002899
:10C42000E6D0E0A006F0B2FCE2E72146E2A006F08A
:10C4300053FCDDE738B508F05BFE4FF4007006F002
:10C440000DFC0446002000906A462146D44806F0C0
:10C450006FFD20B9BDF80010204601F0AAFC20466F
:10C4600006F036FC38BD10B508F042FEBDE81040BD
:10C4700001F080BD38B508F03BFE964C20784007AF
:10C4800029D54FF4806006F0E9FB054600200090B6
:10C490006A462946D04806F04BFDC8B9BDF80020D1
:10C4A0002946CE4805F027FE032811D0BDF800200C
:10C4B0002946CA4805F01FFE032809D0207820F03D
:10C4C00004002070C6A006F061FCC5A004F0A1FE27
:10C4D000284606F0FDFB38BD7CB508F009FE4FF498
:10C4E000806006F0BBFB06460020019001AA3146A1
:10C4F000C04806F01DFD002851D1BFA1304606F00E
:10C5000055FE0546002D46DB4FF4007006F0A6FBF5
:10C5100004464FF480700090711900230A222046CF
:10C5200006F075FD20460CF05CF8217828290CD126
:10C5300094F82510262908D1211811F8052C242A51
:10C5400003D111F8031C292907D02146AEA006F01B
:10C55000C3FB204606F0BCFB21E06178412915D0E1
:10C56000432908D02146AFA006F0B6FBB5A1522062
:10C5700002F0E9FBEDE782B22146894806F089FC2A
:10C580000028E6D087A006F001FCE2E72146B4A02F
:10C5900006F0A2FBDDE73146B9A006F0F7FB304616
:10C5A00006F096FB7CBD70B508F0A2FD4948007806
:10C5B00040072DD5B948044605F0FDFAB748401F9D
:10C5C000054604F0DFFF2B462246B5A1482002F0C5
:10C5D000BAFB102006F042FB06462B46B7A21021FC
:10C5E00030460BF001FD304602F09AFA1021304639
:10C5F0000CF0ECF82346B3A2102130460BF0F4FC0B
:10C60000304602F054FA3046BDE8704006F060BB98
:10C6100070BD38B508F06CFD4FF4807006F01EFB5D
:10C620000446002000906A462146A84806F080FC97
:10C6300090B9BDF80010204605F0D9FD254A78B123
:10C64000022823D0032828D0042814D0A0A006F064
:10C650009DFB9FA004F0DDFD204606F039FB38BDB0
:10C66000107820F0040010709EA006F08FFB9DA0B3
:10C6700004F0CFFDF0E7107820F0010010709EA0CC
:10C6800006F084FB9CA004F0C4FDE5E79EA006F044
:10C690007DFB9DA004F0BDFDDEE7A0A006F076FBCB
:10C6A0009EA004F0B6FDD7E704F022B838B508F034
:10C6B0001FFD4FF4806006F0D1FA04460020009080
:10C6C0006A462146994806F033FC08B921462FE115
:10C6D00031E10000350000202C280020BBF1C8A16A
:10C6E000475053CAFDBEDDCAA7B0DC00555443C84D
:10C6F000D5C6DAA3BA2573B6C8000000555443CA9C
:10C70000B1BCE4A3BA25730000000020CEB3B6C8C4
:10C71000A3BA257325630000BEADB6C8A3BA2573BE
:10C7200025630000CBD9B6C8A3BA2573BDDA0000D3
:10C73000BDC7B7BDCFF2A3BA2573B6C800000000CD
:10C7400040110020555342CAD5B5BDCFC2D0D02725
:10C75000B7C727B7A8CAFDBEDDD6A13A2573202EDC
:10C7600000000000555342CAD5B5BDCFC2D0D0CECF
:10C77000B4D6AAC0E0D0CDCAFDBEDDD6A13A25739D
:10C78000202E0000555342CAD5B5BDCFC2D0D0CE61
:10C79000B4D6AAC0E0D0CDCAFDBEDDD6A10000004F
:10C7A0003C0800207355736572636D64517565753F
:10C7B00065D2E7B3F6A3A100555342C9CFCEBBBBA8
:10C7C000FAC8B7C8CFCAD5B5BDCAFDBEDDD6A13A35
:10C7D0002573202E000000003A0D0020F2010020F9
:10C7E0005463702053656E644461746120457272B5
:10C7F00021000000202000202B51495552433A20AF
:10C800002272656376220000544350CAD5B5BDCF6D
:10C81000C2D0D027B7C727B7A8CAFDBEDDD6A13A78
:10C8200025732000544350CAD5B5BDCFC2D0D0CE59
:10C83000B4D6AAC0E0D0CDCAFDBEDDD6A13A2573DC
:10C8400020000000544350CAD5B5BDCFC2D0D0CED1
:10C85000B4D6AAC0E0D0CDCAFDBEDDD6A10000008E
:10C8600054637020736572766572C8B7C8CFCAD535
:10C87000B5BDCAFDBEDDD6A13A257320000000007B
:10C8800054435020CFC2D0D0CAFDBEDDBDE2CEF6AB
:10C89000CAA7B0DC3A25732000000000821D0020EA
:10C8A0004353513A25732C204543323020566F6C48
:10C8B000746167653A25736D5600000025736D56E7
:10C8C000000000004353512573000000262400207F
:10C8D00054637020756E6B6E6F776E207572632077
:10C8E0002E000000546370207365727665722063B9
:10C8F0006C6F736564202E00546370205044502088
:10C900006465616374202E0054637020696E636FE8
:10C910006D696E672066756C6C202E005463702004
:10C92000696E636F6D696E67202E00004C190020E0
:10C93000D7A006F0D1F9204606F0CAF938BD38B5BF
:10C9400008F0D6FB4FF4806006F088F9044600201A
:10C9500000906A462146D34806F0EAFA18B9214603
:10C96000D1A006F0B9F9204606F0B2F938BD2DE99C
:10C97000F04108F0BDFBD14ED14C4FF000053078AE
:10C98000C10708D0810706D5410704D5000702D5A5
:10C990002570BDE8F0812078401CC0B220700228CC
:10C9A00004D9C8A004F035FC0BF04AF83078C00771
:10C9B0000CD1CAA002F057F804F083FE03286AD015
:10C9C000C8A004F026FCCBA006F086F93078C10799
:10C9D0001DD080071BD4CAA002F045F81E2006F027
:10C9E0003DF907461E21384605F0FDF803285CD0C6
:10C9F000384604F00EFC307820F00100307004F06E
:10CA000081FE384606F068F9384606F061F930785C
:10CA1000C10714D0810712D5400710D4BAA002F084
:10CA200022F802F076F9032844D0307820F0040090
:10CA30003070B9A006F050F9BAA004F0EAFB3078E3
:10CA4000C10711D081070FD500070DD405F0A7FD50
:10CA500003283BD0307820F008003070B5A006F0F5
:10CA60003BF9B8A004F0D5FBBAA006F035F9307850
:10CA7000C1078ED081078CD541078AD5000788D59C
:10CA8000B84805F098F8B748401F04F07BFD02F065
:10CA900065F825707DE702F0CDFA307840F00100AE
:10CAA0003070B1A006F018F990E7307840F002003D
:10CAB0003070A6E7307840F004003070ADA14C2013
:10CAC00002F041F9B1A006F007F9B8E7307840F07C
:10CAD00008003070B0A001F0C6FF02F0F5F907467B
:10CAE000AFA14C2002F02FF9032F04D0B1A004F025
:10CAF00090FB0AF0A5FFB9A006F0EEF800F0E8FA06
:10CB0000B2E708B54FF4E0314FF0006008F0D5FD12
:10CB100008F0EEFA4FF4407008F09AFDB34800F0C8
:10CB200091FBB34800F01AFCB24800F0F0FAB248AA
:10CB300003F060FE08F0DCFA00F070FA01F09DFAF4
:10CB4000AE4C4FF47A7501230A222946207808F06A
:10CB5000B6F9AB49207808F097F908F0C9FAAFF2B6
:10CB6000F110009000236A100221A6A00BF08AF9B0
:10CB7000534C60600BF09EF9AFF23D200090012312
:10CB800064220221A1A00BF07DF9A0600BF092F9C4
:10CB9000AFF2E74002230090642219469EA00BF0FA
:10CBA00071F9E0600BF086F9AFF2035000900323B7
:10CBB000642202219BA00BF065F920610BF07AF949
:10CBC000AFF2B150009004233222022197A00BF063
:10CBD00059F960610BF06EF9AFF2356000900523F2
:10CBE000AA00022194A00BF04DF9A0610BF062F9AC
:10CBF000AFF21B70009006230A22022192A00BF0D4
:10CC000041F9E0610BF056F9AFF2977000900723FD
:10CC10000A2202218FA00BF035F920620BF04AF9AD
:10CC2000AFF2BD7000900823322201218CA00BF0DE
:10CC300029F960620BF03EF9AFF607000090092376
:10CC40003222012189A00BF01DF9A0620BF032F90C
:10CC5000AFF6B10000900A231422012186A00BF048
:10CC600011F9E0620BF026F9AFF6731000900B2378
:10CC70002A46022182A00BF005F920630BF01AF975
:10CC80008249834801F0D4FF01F0EBFFFEE77047D3
:10CC9000527334383520726563646174613A257368
:10CCA000202E000046150020527332333220726568
:10CCB00063646174613A2573202E00003500002002
:10CCC00000000020CFB5CDB3CDF8C2E7B1C0C0A3FE
:10CCD000A3ACD6D8C6F4CFB5CDB32100CED5CAD635
:10CCE000D6D03A00C4A3BFE9B0B2D7B0D2ECB3A358
:10CCF00021000000CED5CAD6CAA7B0DC00000000D3
:10CD0000C8EBCDF8D6D03A00C1ACBDD3544350B730
:10CD1000FECEF1C6F73A0000544350C1ACBDD3CAB1
:10CD2000A7B0DC00544350C1ACBDD3CAA7B0DC21CE
:10CD30000000000048545450B3F5CABCBBAFCAA7AA
:10CD4000B0DC000048545450B3F5CABCBBAFCAA70E
:10CD5000B0DC2100CACDB7C545433230D7CAD4B400
:10CD600021000000821D0020CED5CAD6B3C9B9A6C5
:10CD70002100000044657669636520746370206358
:10CD80006F6E6E657463656421000000544350C18A
:10CD9000ACBDD3B3C9B9A600D7A2B2E1D6D03A0090
:10CDA00044657669636520526567697374657221AD
:10CDB0000000000048747470B3F5CABCBBAF4F4BA1
:10CDC000A3ACD7A2B2E1C7EBC7F3CAA7B0DCA3AC50
:10CDD000D6D8C6F4CFB5CDB321000000D3B2BCFE87
:10CDE000D7A2B2E1B3C9B9A621000000420C0020CD
:10CDF00048000020FF0700202465030034000020C5
:10CE0000D1D001084E65745461736B005273323394
:10CE1000325461736B0000005273343835546173BF
:10CE20006B0000004C65645461736B005463705573
:10CE300072635461736B000054637048656172746F
:10CE40005461736B00000000546370446F776E543C
:10CE500061736B0054637055705461736B00000014
:10CE60004D656E755461736B0000000055636D6411
:10CE70005461736B000000005573625461736B0062
:10CE8000476E73735461736B00000000057F0208E6
:10CE9000C17E020800B585B01322A34968460BF095
:10CEA00016FC9DF80900401C8DF809009FA0008821
:10CEB000ADF80B00684607F0C5FE9B4804F0A9F9E1
:10CEC0009BA004F0A6F90AF0BBFD05B000BD70B54B
:10CED00005460C467B2008F095FD012804D122462A
:10CEE00098A128460BF0BBFC7C2008F08BFD0128A4
:10CEF00004D1224696A128460BF0B1FC7D2008F013
:10CF000081FD012804D1224694A128460BF0A7FCFC
:10CF10007E2008F077FD012804D1224693A12846FF
:10CF20000BF09DFC7C2008F06DFD88B97D2008F099
:10CF300069FD68B97E2008F065FD48B97A2008F0DF
:10CF400061FD012804D122468CA128460BF087FC04
:10CF5000BDE8704008F07DBE10B504460B2204F118
:10CF600019000BF07CFC002084F8250010BD10B5E2
:10CF700004460B2204F125000BF071FC002084F81C
:10CF8000310010BD30B5A1B07F480BF00BF87F48E1
:10CF90000BF008F87E4C7F48211DFFF7E8FF7D4B22
:10CFA0000B22253300217CA00AF0FCFF79481930C0
:10CFB000054607F0EBFA29467648FFF7CDFF2946EC
:10CFC0007AA00AF0EFFFA1787CA030390AF0EAFFDE
:10CFD0000121704807F0E3FA6E4A18217CA00AF09C
:10CFE000E1FF6C480B2131300446FFF770FF224609
:10CFF0000B217CA00AF0D6FF63480AF0D3FF802102
:10D0000001A80BF005FC23467BA2802101A80AF0B1
:10D01000EBFF01A804F0FDF821B030BD10B507F01A
:10D02000C0FE04F0D3F8002006F020F90D2007F030
:10D0300077FCFFF7A7FFAFF2A311022007F0D6FAA3
:10D0400000F070FF03F04FFB03F0B3FB08F0F6F9BC
:10D0500003F038FE4FF4E134204603F0FBFB20469A
:10D0600003F02AFCBDE8104008F0C3BA2DE9F041F6
:10D07000654D4FF48078404605F0F0FD0746634E5D
:10D080007068C0F30F240BE042463946284608F08A
:10D0900031F83A465EA14C2001F055FE05F5807549
:10D0A000641EA4B2F0D2414638460BF08FFB3279B1
:10D0B0003946284608F01EF83A4655A14C2001F0A2
:10D0C00042FE384605F004FEBDE8F04104F036B8F3
:10D0D00010B5524C207807F061FF5148007870B9C4
:10D0E0002C481022104913380BF020FA60B100F0E0
:10D0F0009DFF284814220C4913380BF0B0FB207810
:10D10000BDE8104007F03BBF01F0B6FCF7E7002197
:10D1100040F8191F41608160C160016141611938A7
:10D1200019210BF053BB0000245D002030310000BA
:10D130005274635F416C725F43616C6C6261636BDC
:10D1400021000000D6D8C9CFB5E7C6F4B6AF0000BD
:10D15000C8EDB8B4CEBBC6F4B6AF0000B6C0C1A22D
:10D16000BFB4C3C5B9B7C6F4B6AF0000B4B0BFDA38
:10D17000BFB4C3C5B9B7C6F4B6AF0000D3B2B8B434
:10D18000CEBBC6F4B6AF000054D3020898D3020851
:10D19000420C0020FF0700200D0A426F6F74B0E6BA
:10D1A000B1BE203A20252A2E2A7300000D0A4150D4
:10D1B0005020B0E6B1BE203A202573000D0A52750A
:10D1C0006E4170704E756D3A2041505025640000DC
:10D1D0000D0AC9E8B1B8B1E0BAC5203A20252E2A17
:10D1E000730000000D0AD6D8C6F4D4ADD2F2203AAE
:10D1F00020252E2A73000000D6D8C6F4D4ADD2F272
:10D200003A25732E0000000000F80708541D002086
:10D21000B1BEB5D86C6F673A2573000034000020AA
:10D220004C000020F8220146F94808F006B810B575
:10D23000F8210BF0CBFABDE81040F822F549F4488C
:10D2400007F058BF7CB50446F34805F019FE2046A8
:10D25000FFF7EDFF5B202070302060703120A07060
:10D26000E070207CFF2809D104F110004021054620
:10D270000BF0ACFAE9A128460BF084F994F85000C1
:10D28000FF2809D104F15000402105460BF09EFA19
:10D29000E4A128460BF076F994F89000FF2809D114
:10D2A00004F19000402105460BF090FADEA12846DB
:10D2B0000BF068F994F8D000FF2809D104F1D000F0
:10D2C000102105460BF082FADBA128460BF05AF933
:10D2D00094F8E000FF2816D0A8B1CE49DA48E03132
:10D2E00001F0FAFC94F8F000FF2817D0B0B1C9495A
:10D2F000D548F03101F0FDFC5D2084F8F7002046B0
:10D30000BDE87C408EE704F1E000102105460BF0FB
:10D310005DFAC9A128460BF035F9E3E70020C4F80F
:10D32000F000A4F8F400009001900A22694641F64A
:10D33000583005F0C4FE694604F1F0000BF022F904
:10D34000DAE701460322C14807F077BF00220280D6
:10D35000827001460322BD4807F0CCBE10B50446DA
:10D360002046FFF7F3FF2046BDE81040E9E72DE92E
:10D37000F04105460F46032640F2492005F06EFCB9
:10D3800004463B464FF40077B1A2394604F126002B
:10D390000AF02AFE002801DDB8420BDD40F29E2291
:10D3A000ACA1B1A005F0F2FC204605F091FC0220F2
:10D3B000BDE8F08128222270642190FBF1F2303226
:10D3C000A27090FBF1F201FB12020A2192FBF1F232
:10D3D0003032E27090FBF1F201FB1200303020712C
:10D3E000A84908786071401CC0B20870392801D97A
:10D3F000302008700422A4A1A01D0BF030FA0121F6
:10D4000004F10A0007F0CBF83B2184F82210B5F8AC
:10D410002310A4F82310262184F8251068784328C7
:10D4200014D072216170032299A120460BF06CF890
:10D4300020460BF0D6F8401C82B22146002006F0B0
:10D4400054F9204605F044FC3046B1E752216170A2
:10D4500003228FA120460BF057F820460BF0C1F8AD
:10D4600082B221468B4805F014FD0028E9D04FF424
:10D470002E7278A188A005F089FCE2E7532070475E
:10D480002DE9F04707463C46A0782179303800EB7B
:10D49000C00202EB001001EB8001E0786FF02F0278
:10D4A000303800EB800002EB40000D18DFF860A17F
:10D4B000F8225849504607F01DFE4FF4807630465A
:10D4C00005F0CCFB8046534B7BA2F03399463146A6
:10D4D00040460AF089FD064694F82300312804D11D
:10D4E000611991F82610242902D030281DD021E09E
:10D4F000102148460BF06AF92A4604F126014846F5
:10D500000BF0ADF9F8224349504607F096FEC6F5F8
:10D51000807108EB06004B466CA20AF065FD5324AF
:10D5200041463846FFF723FF05E0601990F82600D2
:10D53000242806D04924404605F0CAFB2046BDE811
:10D54000F087532441463846FFF711FFF3E72DE9F2
:10D55000F04707463C46A0782179303800EBC002FE
:10D5600002EB001001EB8001E0786FF02F02303801
:10D5700000EB800002EB40000D18DFF894A0F822C9
:10D580002449504607F0B6FD4FF48076304605F04A
:10D5900065FB80461F4B52A2E03399463146404618
:10D5A0000AF022FD064694F82300312804D16119BF
:10D5B00091F82610242902D030281DD021E0102116
:10D5C00048460BF003F92A4604F1260148460BF0C1
:10D5D00046F9F8220F49504607F02FFEC6F5807134
:10D5E00008EB06004B4643A20AF0FEFC53244146DA
:10D5F0003846FFF7BCFE05E0601990F826002428A5
:10D6000005D04924404605F063FB204697E77BE0C0
:10D6100000880108420C00203C0800202F41424DA8
:10D620000000000041424D0053686F7033343437BE
:10D6300039343734390000003132312E34312E374D
:10D64000392E383700000000F20100200090010858
:10D650002573000055534552434D445C7573657204
:10D66000636D642E6300000025732C25643A757089
:10D6700044617461427566207370696C6C6F766585
:10D6800072A3A100380000204D41433A0000000081
:10D69000245829003A0D002025732C25643A735430
:10D6A0006370305175657565207370696C6C6F7649
:10D6B0006572A3A1000000002A4745542A20546344
:10D6C00070506F72743A5B25735D21002A53455484
:10D6D0002A20546370506F72743A5B25735D210089
:10D6E0002A4745542A2054637049503A5B25735D9C
:10D6F000210000002A5345542A2054637049503AAF
:10D700005B25735D21000000532441463846FFF736
:10D710002EFE77E72DE9F04707463C46A0782179B1
:10D72000303800EBC00202EB001001EB8001E07822
:10D730006FF02F02303800EB800002EB40000D1834
:10D74000DFF8F4A3F822FB49504607F0D3FC4FF46E
:10D750008076304605F082FA8046F64BF7A2D03349
:10D760009946314640460AF03FFC064694F82300AD
:10D77000312804D1611991F82610242902D03028CB
:10D780001DD021E0102148460BF020F82A4604F174
:10D79000260148460BF063F8F822E649504607F0A8
:10D7A0004CFDC6F5807108EB06004B46E8A20AF076
:10D7B0001BFC532441463846FFF7D9FD05E06019AC
:10D7C00090F82600242805D04924404605F080FA28
:10D7D0002046B4E6532441463846FFF7C8FDF4E737
:10D7E0002DE9F04707463C46A0782179303800EB18
:10D7F000C00202EB001001EB8001E0786FF02F0215
:10D80000303800EB800002EB40000D18DFF828A351
:10D81000F822C849504607F06DFC4FF48076304638
:10D8200005F01CFA8046C34BCEA290339946314690
:10D8300040460AF0D9FB064694F82300312804D16B
:10D84000611991F82610242902D030281DD021E03A
:10D85000402148460AF0BAFF2A4604F1260148460C
:10D860000AF0FDFFF822B349504607F0E6FCC6F582
:10D87000807108EB06004B46C0A20AF0B5FB5324AA
:10D8800041463846FFF773FD05E0601990F8260021
:10D89000242805D04924404605F01AFA20464EE6D1
:10D8A000532441463846FFF762FDF4E72DE9F0477F
:10D8B00007463C46A0782179303800EBC00202EBE5
:10D8C000001001EB8001E0786FF02F02303800EBA0
:10D8D000800002EB40000D18DFF85CA2F8229549A9
:10D8E000504607F007FC4FF48076304605F0B6F955
:10D8F0008046904BA7A250339946314640460AF0E5
:10D9000073FB064694F82300312804D1611991F87D
:10D910002610242902D030281DD021E0402148467D
:10D920000AF054FF2A4604F1260148460AF097FF00
:10D93000F8228049504607F080FCC6F5807108EB5C
:10D9400006004B4699A20AF04FFB53244146384645
:10D95000FFF70DFD05E0601990F82600242805D09A
:10D960004924404605F0B4F92046E8E553244146F1
:10D970003846FFF7FCFCF4E72DE9F04707463C4644
:10D98000A0782179303800EBC00202EB001001EBE7
:10D990008001E0786FF02F02303800EB800002EB5E
:10D9A00040000D18DFF890A1F8226249504607F0B8
:10D9B000A1FB4FF48076304605F050F980465D4B70
:10D9C00080A210339946314640460AF00DFB0646C8
:10D9D00094F82300312804D1611991F826102429E4
:10D9E00002D030281DD021E0402148460AF0EEFE4A
:10D9F0002A4604F1260148460AF031FFF8224D4933
:10DA0000504607F01AFCC6F5807108EB06004B463D
:10DA100072A20AF0E9FA532441463846FFF7A7FC00
:10DA200005E0601990F82600242805D049244046D6
:10DA300005F04EF9204682E5532441463846FFF76B
:10DA400096FCF4E72DE9F84307463C46DFF8E890FA
:10DA5000F8223849484607F04DFB4FF480752846B8
:10DA600005F0FCF806466348804606F08FFDCDF8C9
:10DA70000080DFF8C08060A2294698F80230304666
:10DA80000AF0B2FA054694F82300312804D167A1C0
:10DA9000A01C05F08BFB20B194F82300302821D086
:10DAA00025E094F82600302807D0312805D0322808
:10DAB00003D0332801D050241AE088F80200F8225D
:10DAC0001C49484607F0B9FB98F80230C5F580714B
:10DAD000701957A20AF088FA532431463846FFF7E6
:10DAE00046FC05E051A1A01C05F060FB30B14924C3
:10DAF000304605F0EDF82046BDE8F8835324314662
:10DB00003846FFF734FCF3E72DE9F04707463C467B
:10DB1000DFF82490F8220749484607F0EBFA4FF463
:10DB20008075284605F09AF80646DFF8088098F8D0
:10DB300001308FE0420C0020008801082A4745543C
:10DB40002A2046747049503A5B25735D210000001D
:10DB50002A5345542A2046747049503A5B25735D18
:10DB6000210000002A4745542A20467470506173F2
:10DB700073776F72643A5B25735D21002A534554B5
:10DB80002A2046747050617373776F72643A5B2514
:10DB9000735D21002A4745542A20467470557365E9
:10DBA000726E616D653A5B25735D21002A534554A1
:10DBB0002A20467470557365726E616D653A5B25F7
:10DBC000735D21002A4745542A20467470466F6CC5
:10DBD0006465723A5B25735D210000002A53455449
:10DBE0002A20467470466F6C6465723A5B25735DDB
:10DBF00021000000180800202A4745542A205275A9
:10DC00006E4170704E756D3A5B41505025635D20DA
:10DC1000212020202A4745542A20417070566572E1
:10DC200073696F6E3A5B25735D20210030303100DF
:10DC30002A5345542A2052756E4170704E756D3AC4
:10DC40005B41505025635DD6D8C6F4BAF3C9FAD00B
:10DC5000A721000083A2294630460AF0C5F90546EF
:10DC600094F82300312805D1AFF24001A01C05F043
:10DC70009DFA20B194F8230030281DD022E094F8BA
:10DC80002600302803D0312801D050241BE088F82A
:10DC90000100F8227949484607F0CFFA98F8013098
:10DCA000C5F58071701976A20AF09EF953243146A9
:10DCB0003846FFF75CFB06E0AFF29001A01C05F0D0
:10DCC00075FA28B14924304605F002F8204636E4BA
:10DCD000532431463846FFF74AFBF4E7F0B58DB0E0
:10DCE0000446F82265496B4807F004FA6AA104F17A
:10DCF000260005F05BFA18B149240DB02046F0BDAE
:10DD00004FF40076304604F0A9FF07466448054604
:10DD100006F03CFC5948F030A0F12002A0F1E003ED
:10DD2000CDE90932A0F11001CDE90B105D4A603850
:10DD3000A2F10903CDE905329039CDE90710111F91
:10DD4000A0F18C029038C378CDE9022501930491AB
:10DD5000817800914378544A314638460AF044F9B4
:10DD600039462046FFF703FB5324384604F0B0FF42
:10DD7000C3E770B504464DA104F1260005F016FA7C
:10DD800010B15025284670BD53254AA12046FFF703
:10DD9000EEFA642007F049F800F0B2FF642007F0C3
:10DDA00044F803F0AFFC4CA003F033FA09F048FE4E
:10DDB000E8E710B5044694F824003038112835D22D
:10DDC000DFE800F0090D1115191D2125292D343426
:10DDD0003434343431002046FFF7CBFF27E02046AF
:10DDE000FFF77CFF23E02046FFF78EFE1FE0204672
:10DDF000FFF728FE1BE02046FFF7BEFD17E0204698
:10DE0000FFF754FD13E02046FFF7EAFC0FE0204641
:10DE1000FFF780FC0BE02046FFF799FB07E0204668
:10DE2000FFF72EFB03E0FFF729FB00E04E202E4911
:10DE3000502809D049280DD04E2811D149682046D4
:10DE4000BDE81040FFF793BA89682046BDE810404E
:10DE5000FFF78DBAC9682046BDE81040FFF787BAC2
:10DE600010BD00002A4745542A20496170466C6164
:10DE7000673A5B25635D212000000000420C002012
:10DE80002A5345542A20496170466C61673A5B25E4
:10DE9000635D2100008801084745545F49415000F7
:10DEA00018080020861D0020E8D30208434D445F77
:10DEB000525354002A5345542A20557365722063E7
:10DEC0006F6E74726F6C206465766963652072652D
:10DED0007374617274210000D6D8C6F4C3FCC1EE1D
:10DEE000C8EDD6D8C6F421003800002049490620E4
:10DEF00048707047474907204870704745490520DA
:10DF000048707047434909204870704741490320D1
:10DF1000487070473F490C20487070473D490B20BE
:10DF20004870704710B502F0F1FBAFF20F010C2002
:10DF300006F03DFAAFF223010B2006F038FAAFF2FB
:10DF40003301092006F033FAAFF247010D2006F045
:10DF50002EFAAFF25701072006F029FAAFF26B0153
:10DF60000F2006F024FAAFF27B01BDE81040062036
:10DF700006F01DBA27484278011D0D2A48D2DFE875
:10DF800002F0474747174727372F471F47070F001C
:10DF9000027802EB420201EB8202527802702EE01C
:10DFA000027802EB420201EB82029278027026E0D4
:10DFB000027802EB420201EB8202D27802701EE08C
:10DFC000027802EB420201EB82021279027016E043
:10DFD000027802EB420201EB8202527902700EE0FB
:10DFE000027802EB420201EB82029279027006E0B3
:10DFF000027802EB420201EB8202D2790270002227
:10E000004270007800EB400001EB80008068004720
:10E01000704700004C00002008B5F8A000230090D5
:10E0200003220C21184602F042FD08BD38B51E201F
:10E0300004F014FE04460522F64920460AF00FFCBF
:10E040000122002310211046009402F030FD1E2111
:10E0500020460AF0BBFBEF490A220B3920460AF0A2
:10E06000FEFB002302220C210120009402F01FFD80
:10E070002046BDE8384004F02BBE10B5FFF7D6FFB0
:10E08000BDE81040C8E708B5E3A0012300901A4698
:10E090001021002002F00BFDE2A0002300900222DC
:10E0A0001021184602F003FDE1A000230090032296
:10E0B0001021184602F0FBFC08BD08B5D6A00023CD
:10E0C000009001221021184602F0F1FCD5A000902A
:10E0D000012302221021002002F0E9FCD4A0002339
:10E0E000009003221021184602F0E1FC08BD08B59B
:10E0F000C9A00023009001221021184602F0D7FC8D
:10E10000C8A00023009002221021184602F0CFFC84
:10E11000C7A00090012303221021002002F0C7FCB9
:10E1200008BD08B5BFA000230090012210211846A9
:10E1300002F0BDFCBEA00023009002221021184670
:10E1400002F0B5FCBDA000900123032210210020A5
:10E1500002F0ADFC08BD08B5B5A000230090012277
:10E160001021184602F0A3FCB4A000230090022264
:10E170001021184602F09BFCB3A00090012303225B
:10E180001021002002F093FC08BD08B5B1A00123C6
:10E1900000901A461021002002F089FCB0A0002354
:10E1A000009002221021184602F081FCAFA000234B
:10E1B000009003221021184602F079FC08BD08B532
:10E1C000A4A00023009001221021184602F06FFC49
:10E1D000A3A00090012302221021002002F067FC7E
:10E1E000A2A00023009003221021184602F05FFC39
:10E1F00008BD08B597A00023009001221021184601
:10E2000002F055FC96A0002300900222102118462F
:10E2100002F04DFC95A00090012303221021002064
:10E2200002F045FC08BD08B58DA000230090012236
:10E230001021184602F03BFC8CA000230090022223
:10E240001021184602F033FC8BA00090012303221A
:10E250001021002002F02BFC08BD08B589A0012385
:10E2600000901A461021002002F021FC88A0002313
:10E27000009002221021184602F019FC87A000230A
:10E28000009003221021184602F011FC08BD08B5C9
:10E290007CA00023009001221021184602F007FC08
:10E2A0007BA00090012302221021002002F0FFFB3E
:10E2B0007AA00023009003221021184602F0F7FBF9
:10E2C00008BD08B576A0012300901A461021002051
:10E2D00002F0EDFB75A000230090022210211846E9
:10E2E00002F0E5FB6DA000230090032210211846E8
:10E2F00002F0DDFB08BD08B569A0002300900122F3
:10E300001021184602F0D3FB68A0009001230222DE
:10E310001021002002F0CBFB60A00023009003221C
:10E320001021184602F0C3FB08BD08B562A0012306
:10E3300000901A461021002002F0B9FB61A00023D2
:10E34000009002221021184602F0B1FB61A00023C8
:10E35000009003221021184602F0A9FB08BD08B561
:10E3600055A00023009001221021184602F09FFBC7
:10E3700054A00090012302221021002002F097FBFC
:10E3800054A00023009003221021184602F08FFBB6
:10E3900008BD08B548A000230090012210211846AE
:10E3A00002F085FB47A000230090022210211846AE
:10E3B00002F07DFB47A000900123032210210020E2
:10E3C00002F075FB08BD08B546A0012300901A466F
:10E3D0001021002002F06BFB44A0002300900222D9
:10E3E0001021184602F063FB42A000230090032294
:10E3F0001021184602F05BFB08BD00004D454E554C
:10E4000020202020202020202020202020424143A6
:10E410004B0000002F5D002046545020D0C5CFA2F5
:10E420000000000054435020D0C5CFA200000000DF
:10E43000C9E8B1B8C9FDBCB600000000C9E8B1B870
:10E44000D0C5CFA20000000047505320D0C5CFA2B6
:10E4500000000000B2E9D1AF465450D5CBBAC50098
:10E46000B2E9D1AF465450C3DCC2EB00B2E9D1AF40
:10E470004654502020495000B2E9D1AF465450C212
:10E48000B7BEB600B2E9D1AF544350202049500086
:10E49000B2E9D1AF544350B6CBBFDA002000000040
:10E4A000B2E9D1AFB5B1C7B041505000C1A2BCB4C0
:10E4B000C9FDBCB641505000B2E9D1AF4D4143490E
:10E4C00044000000B2E9D1AF41505020B0E6B1BEE7
:10E4D00000000000B2E9D1AF424F4F54B0E6B1BEE8
:10E4E00000000000BEADCEB3B6C80000BDC7B7BDCA
:10E4F000CFF20000CBD9B6C8D6B5000008B5AFF250
:10E500001C000023009001221021184602F0CFFACF
:10E51000AFF228000090012302221021002002F017
:10E52000C6FAAFF2300000230090032210211846F3
:10E5300002F0BDFA60E708B5AFF258000023009082
:10E5400001221021184602F0B2FAAFF26000002357
:10E55000009002221021184602F0A9FAAFF26C00D6
:10E560000090012303221021002002F0A0FA43E7CB
:10E5700008B5F9A0012300901A461021002002F0EE
:10E5800096FAF8480023009002221021184602F063
:10E590008EFAAFF2F80000230090032210211846F3
:10E5A00002F085FA28E708B5EFA0012300901A468B
:10E5B0001021002002F07BFAEA480023403000904E
:10E5C00002221021184602F072FAE64840380AF09A
:10E5D00008F8102809D9E3480023303800900322B6
:10E5E0001021184602F063FA06E7AFF2501000233C
:10E5F000009003221021184602F059FAFCE608B5F3
:10E60000DCA0012300901A461021002002F04FFAEE
:10E61000D44800238030009002221021184602F0D6
:10E6200046FAD048403809F0DCFF102809D9CD4817
:10E6300000233038009003221021184602F037FAE8
:10E64000DAE6AFF2A810002300900322102118464A
:10E6500002F02DFAD0E638B5C8A0012300901A4682
:10E660001021002002F023FABE4C0023403C02227D
:10E6700010211846009402F01AFA204609F0B1FF62
:10E68000102809D904F11000002300900322102162
:10E69000184602F00CFA38BDAFF2002000230090BB
:10E6A00003221021184602F002FA38BD08B5B6A0C0
:10E6B000012300901A461021002002F0F8F9A94821
:10E6C00000239030009002221021184602F0EFF94A
:10E6D000A448403809F085FF102809D9A148002333
:10E6E0003038009003221021184602F0E0F983E64A
:10E6F000AFF258200023009003221021184602F0A8
:10E70000D6F979E608B5A2A0012300901A46102197
:10E71000002002F0CCF993480023A03000900222A0
:10E720001021184602F0C3F98E48403809F059FF0D
:10E73000102809D98B48002330380090032210217B
:10E74000184602F0B4F957E6AFF2B020002300906B
:10E7500003221021184602F0AAF94DE638B58FA021
:10E76000012300901A461021002002F0A0F9102089
:10E7700004F074FA04467B488CA250381021837848
:10E78000204609F031FC0023022210211846009493
:10E7900002F08DF9AFF2FC2000230090032210213B
:10E7A000184602F084F92046BDE8384004F090BADB
:10E7B00010B56C49312050394870F822804806F075
:10E7C0003CFD80A004F088FA022006F02EFBBDE894
:10E7D000104009F035B938B57FA0012300901A46E2
:10E7E0001021002002F063F9192004F037FA0446E2
:10E7F0000121204605F0D3FE002302220C211846F9
:10E80000009402F054F904F1150000230090032253
:10E810000C21184602F04BF92046BDE8384004F0C0
:10E8200057BA38B56EA0012300901A461021002077
:10E8300002F03DF90C2004F011FA0446204605F0E0
:10E84000A5FE0023022210211846009402F02FF9A1
:10E85000AFF2B8300023009003221021184602F0D6
:10E8600026F92046BDE8384004F032BA08B55FA06A
:10E87000012300901A461021002002F018F93948AF
:10E8800000234C38009002221021184602F00FF9A4
:10E89000AFF2F8300023009003221021184602F056
:10E8A00006F9A9E53EB554A0012300901A461021AF
:10E8B000002002F0FCF8524C207E08B9E07AD8B172
:10E8C00094F825004E494FA21831CDE900210023CC
:10E8D000029003221021184602F0E9F8E07D484931
:10E8E00048A20B31CDE90021002302900222102121
:10E8F000184602F0DCF83EBD44A00023009002223E
:10E900001021184602F0D3F8AFF2704000230090B7
:10E9100003221021184602F0CAF83EBD1CB53FA0E4
:10E92000012300901A461021002002F0C0F834485C
:10E930003CA12C30CDE90010002302221021184602
:10E9400002F0B5F8AFF2AC40002300900322102192
:10E95000184602F0ACF81CBD465450D5CBBAC53AA7
:10E9600000000000920C0020465450C3DCC2EB3A79
:10E97000000000004654502049503A00465450C20E
:10E98000B7BEB63A000000005443502049503A0048
:10E99000544350B6CBBFDA3A00000000B5B1C7B05F
:10E9A000D4CBD0D0415050BAC53A000052756E4118
:10E9B00070704E756D3A5B25635DA1A30000000089
:10E9C00000880108C9FDBCB6C9E8B1B8A3ACBCB4A5
:10E9D000BDABD6D8C6F400004D414349443A0000CF
:10E9E00041505020B0E6B1BEBAC53A00424F4F5434
:10E9F000B0E6B1BEBAC53A00BEADCEB3B6C83A00B5
:10EA00002C2800202573256300000000475053D0B8
:10EA1000C5BAC5C8F52E2E2E00000000BDC7B7BD73
:10EA2000CFF23A00257320B6C80000001CB570A0D4
:10EA3000012300901A461021002002F038F86E4899
:10EA40006EA1CDE90010002302221021184602F029
:10EA50002EF8AFF2B8500023009003221021184680
:10EA600002F025F877E708B5002300901A46102138
:10EA7000184602F01CF8BFE438B5624C2078C10794
:10EA80004FF010000AD000905FA30022022138202E
:10EA900001F0E2FF2068401C206038BDAFF2046343
:10EAA000009000220221382001F0D6FFF2E71CB5C9
:10EAB000044610200022009054A31146104601F095
:10EAC000CBFF554809F002FD00211C2808DB534804
:10EAD0001023CDE900102022084602F0B1FA16E01A
:10EAE00017280ADA4D4810238030CDE900100021A4
:10EAF0002022084602F0A4FA09E0484810234030DA
:10EB0000CDE9001000212022084602F099FA0C20DD
:10EB100000220090234611461A2001F09DFF1AE7BB
:10EB20001CB5044610210022009138A31146402054
:10EB300001F092FF39490022C031CDE900211023B4
:10EB400020220021402002F07BFA0C2100220091BB
:10EB5000234611465A2001F07FFFFCE610B5102035
:10EB600004F07CF804462C4B2DA25B1F102120469C
:10EB700009F03AFA2046FFF7D3FF1021204609F0AA
:10EB800025FE254B28A21021204609F02DFA20460B
:10EB9000FFF78DFF2046BDE8104004F099B870479C
:10EBA00008B50023009001221021184601F07FFFD4
:10EBB000BDE80840022001F06FBF08B500230090B7
:10EBC00002221021012001F072FF15E438B50C4635
:10EBD0000023009001221021184601F068FF002355
:10EBE000022210211846009401F061FF38BD000098
:10EBF000CBD9B6C8D6B53A0052280020257320BD1F
:10EC0000DA000000E80100203A0000002020202067
:10EC10002020202000000000821D002082BC02086D
:10EC200025736D560000000043535125730000000A
:10EC300070B505460C4600230F220A21032006F07A
:10EC40003EF92946032006F01FF900230E220A216F
:10EC5000022006F034F92146BDE87040022006F09B
:10EC600013B910B5032006F08AF9BDE81040022060
:10EC700006F085B910B5032006F090F9BDE8104004
:10EC8000022006F08BB913480168491C0160016835
:10EC9000491C00D10160704710B500230C2264218B
:10ECA000052006F00CF9AFF22101BDE81040052067
:10ECB00006F0EAB810B5052006F061F90549002014
:10ECC000086010BD10B5052006F068F9014800681D
:10ECD00010BD0000EC01002070B504460D46102167
:10ECE000601C09F073FD2946601CBDE8704009F006
:10ECF00049BC10B50446084609F0E8FB608210BD27
:10ED000010B5002003F0DEF9BDE81040012002F04C
:10ED100078BE10B503F000F903280CD1434803F086
:10ED2000D5F904464149032C06D04A8A491C40A023
:10ED300004F02CF8204610BD4A8A491C43A003F079
:10ED4000CBFF204610BD0FB4F8B50646032540F2B0
:10ED5000492003F083FF044608AB00934FF400778B
:10ED6000394604F12600079A09F002F9002801DD6E
:10ED7000B8420BDD82223CA140A004F007F82046F7
:10ED800003F0A6FF0220F8BC5DF814FB28222270D5
:10ED90006670642290FBF2F13031A17090FBF2F1C9
:10EDA00002FB11010A2291FBF2F13031E17090FB7C
:10EDB000F2F102FB1100303020711C49891E0878E5
:10EDC0006071401CC0B20870392801D93020087029
:10EDD000042231A1A01D09F042FD012104F10A0025
:10EDE00005F0DDFB3B2184F822103022022104F1E2
:10EDF000230009F0E3FC262184F82510032228A132
:10EE0000204609F081FB204609F0EBFB82B2214647
:10EE1000244804F03EF820B1A12213A122A003F05F
:10EE2000B5FF204603F054FF2846ACE7F20100206E
:10EE300054435020536572766572C1ACBDD3CAA7E6
:10EE4000B0DC3A25733A256420A3A1005443502036
:10EE5000536572766572C1ACBDD3B3C9B9A63A2504
:10EE6000733A256420A3A100555345525F54435083
:10EE70005C757365725F7463702E630025732C2557
:10EE8000643A757044617461427566207370696C90
:10EE90006C6F766572A3A1004D41433A00000000FB
:10EEA000245829003A0D002025732C25643A735408
:10EEB0006370305175657565207370696C6C6F7621
:10EEC0006572A3A100000000F0B585B001213748AC
:10EED00005F065FB01F0EAFA0746344801F0D0FA84
:10EEE000024633A1384601F0B7F9384601F054F92B
:10EEF000044621462FA003F01DFF2146324803F0AF
:10EF000059FB0446032C0DD03048017821F008014C
:10EF100001702FA002F07DF9384600F0E1F805B04D
:10EF20002046F0BD03F093FB0446032CF4D17B2173
:10EF30002B4809F04BFB00F0ECFD064630000FD0EB
:10EF400028A101F054F9054615B1E86804280FD04E
:10EF5000022427A003F01AFF304600F0C1F8DBE7D7
:10EF600000F072F8014627A003F0B6FE0224F3E792
:10EF700013222848296909F072FC264805F0C2FDD1
:10EF800013222449684609F0A2FB9DF80900401CA1
:10EF90008DF8090020A00088ADF80B00684605F048
:10EFA00051FE1EA0296903F0C5FED5E7FF0700202A
:10EFB0006D616300D3B2BCFED7A2B2E14A534F4E9B
:10EFC000A3BA2573000000000802002035000020CD
:10EFD0004874747020706F7374206572722E000014
:10EFE000E01E002073797354696D653200000000E3
:10EFF0004E6F20226A736F6E5F74696D6522202EDA
:10F0000000000000636A736F6E206572723A2573A8
:10F0100000000000245D0020303100002573CEAADE
:10F02000BBF1C8A1B5BDB5C4B7FECEF1C6F7CAB134
:10F03000BCE42E0010B503F0D7FC03F0D8FC044666
:10F0400003F0D8FC204610BDFE480068704770B53C
:10F0500004460D46002C01D02DB10AE00DB101206F
:10F0600070BD002070BD012070BD207898B1641C77
:10F070006D1C207808F06FFF0646287808F06BFFBB
:10F080008642F2D0207808F066FF0446287808F01F
:10F0900062FF201A70BD002070BD70B50646304674
:10F0A00009F09FFA451C284603F0D8FD041E06D03F
:10F0B0002A463146204609F00AFB204670BD20460C
:10F0C00003F006FE002070BD10B5282003F0C6FD39
:10F0D00004461CB12821204609F09AFB204610BDA9
:10F0E00070B5044619E02568A089C00503D4A0685E
:10F0F00008B1FFF7F5FFA089C00503D4206908B166
:10F1000003F0E6FDA089800503D4206A08B103F06E
:10F11000DFFD204603F0DCFD2C46002CE3D170BD62
:10F120002DE9F34F85B08A4600242546C6490020C4
:10F13000CDE90201002637468346012001909AF866
:10F1400000002D2805D1C1490020CDE902010AF1B6
:10F15000010A9AF80000302801D10AF1010A9AF850
:10F1600000003138082817D89AF8000030380CF021
:10F1700010F9804689460022B54B204629460CF0FE
:10F180006FF942464B460BF057FE04460D461AF8FF
:10F19000010F30380928E7D99AF800002E2827D126
:10F1A0009AF80100302823D3392821D80AF1010A1E
:10F1B0009AF8000030380CF0ECF8804689460022BE
:10F1C000A34B204629460CF04BF942464B460BF028
:10F1D00033FE04460D4600229B4B304639460CF068
:10F1E00065FB06460F461AF8010F30380928DFD9AB
:10F1F0009AF80000652801D045281DD11AF8010FA2
:10F200002B2802D02D2803D010E00AF1010A0DE0CE
:10F210004FF0FF3001900AF1010A07E00BEB8B0180
:10F2200000EB410B0AF1010AABF1300B9AF8000038
:10F23000A0F130010929F1D901980BFB00F00CF085
:10F24000A8F832463B460BF0F7FD02460B4600207D
:10F250007F490BF0B3F806460F46DDE9020122466E
:10F260002B460CF0FDF832463B460CF0F9F804460C
:10F270000D460598C0E90645204629460CF02CF8B5
:10F280000599486105980321C16007B05046BDE863
:10F29000F08F401E40EA600040EAA00040EA2010E3
:10F2A00040EA202040EA2040401C704770B50446E8
:10F2B000002C08D0236833B1A268501861688142DD
:10F2C00003DB981870BD002070BDFFF7E2FF064613
:10F2D000304603F0C3FC054665B1D4E90012284668
:10F2E00009F0F5F9206803F0F3FC66602560A0687A
:10F2F000284470BD206803F0EBFC002060602060B3
:10F3000070BD10B50446002C08D0206830B1A1684B
:10F31000084409F066F9A168084410BD002010BD3A
:10F320002DE9F04707460E46DFF82881D7E9064564
:10F3300000221346204629460BF092FF12D12EB12F
:10F3400002213046FFF7B2FF814603E0022003F0BE
:10F3500085FC8146B9F1000F03D03FA00088A9F8D1
:10F3600000009CE078690CF014F822462B460CF063
:10F370009DFA21F00041002243460CF035F821D8D7
:10F38000364A374B204629460CF02EF81AD8002270
:10F39000344B204629460CF061F913D82EB11521C3
:10F3A0003046FFF783FF814603E0152003F056FC4B
:10F3B0008146B9F1000F72D02BA148467A6908F056
:10F3C000FDFD6CE02EB140213046FFF76FFF814616
:10F3D00003E0402003F042FC8146B9F1000F5ED00B
:10F3E000204629460AF0CEFD22462B460CF05EFA56
:10F3F00021F00041002243460BF0F6FF0ED825F025
:10F4000000412046194A1A4B0BF0EEFF06D2224665
:10F410002B4618A1484608F0D1FD40E0204625F0D3
:10F42000004106460F46154A154B0BF0DDFF06D38B
:10F43000304639460022134B0CF010F929D22246EF
:10F440002B4621E0180200200000F03F0000F0BF32
:10F45000000024400000B03C300000000000C0FF6D
:10F46000FFFFDF410000E0C12564000044F3C2E477
:10F47000E4E9634C252E3066000000008DEDB5A058
:10F48000F7C6B03E65CDCD41F6A1484608F096FDE1
:10F4900005E022462B46F4A1484608F08FFD484679
:10F4A000BDE8F0870178A1F13002092A01D81146A0
:10F4B0000AE0A1F14102052A01D8373904E0A1F19F
:10F4C0006102052A0AD857390A01401C0178A1F1C6
:10F4D0003003092B04D8303A11440EE00020704765
:10F4E000A1F14103052B02D8373A114405E0A1F1FF
:10F4F0006103052B0BD8573A11440A01401C0178CF
:10F50000A1F13003092B04D8303A11440EE0002059
:10F510007047A1F14103052B02D8373A114405E0A9
:10F52000A1F16103052B0AD8573A1144090140782B
:10F53000A0F13002092A04D830390844704700206D
:10F540007047A0F14102052A02D8373908447047B4
:10F55000A0F16102052A02D85739084470470020FB
:10F5600070472DE9F04780460D466C1C0020297835
:10F57000222907D0BD480560002091E7641C5C2A61
:10F5800000D1641C2278222A02D00AB1401CF5D195
:10F59000401C03F063FB0746380004D0681C3C465F
:10F5A0004FF480691AE000207AE75C2903D004F860
:10F5B000011B401C12E0461C3078722825D006DC66
:10F5C000622816D0662818D06E2804D119E0742855
:10F5D0001FD0752821D004F8010B701C0178222956
:10F5E00001D00029E1D100212170017822296AD0BF
:10F5F0006AE0082004F8010BEFE70C2004F8010B87
:10F60000EBE70A2004F8010BE7E70D2004F8010BF3
:10F61000E3E7092004F8010BDFE7701CFFF742FF66
:10F620000546361DA5F55C404845D6D3002DD4D0FF
:10F63000A5F55840484513D270785C28CDD1B078F4
:10F640007528CAD1F01CFFF72DFFB61DA0F55C414F
:10F650004945C2D2C5F3090161F39F2000F5803509
:10F660000421802D01D2012108E0B5F5006F01D2FF
:10F67000022103E0B5F5803F00D203216018012983
:10F680001AD0022911D0032908D0042919D105F074
:10F69000BF0242F0800200F8012DAD0905F0BF0263
:10F6A00042F0800200F8012DAD0905F0BF0242F0E2
:10F6B000800200F8012DAD096D4A525C2A4300F822
:10F6C000012D441889E7401CC8F810700421C8F8BF
:10F6D0000C10E5E62DE9F04705468A460024002196
:10F6E000A9460AE0421E1F2A11D322280FD05C2807
:10F6F0000DD00020014309F1010999F8000000280C
:10F70000F0D18046222721B125B32E4644E00120C6
:10F71000F0E7A9EB0506BAF1000F05D0F11C504641
:10F72000FFF7C4FD044603E0F01C03F097FA04461B
:10F7300074B1277004F101092946484608F022FFF8
:10F7400009F8067009EB060080F801802046A7E65C
:10F750000020A5E6BAF1000F05D003215046FFF7BF
:10F76000A5FD044603E0032003F078FA04462CB11B
:10F7700040A1204608F006FF204691E600208FE6D3
:10F7800049463DA008F0B6FE08B1641C03E0B9F19B
:10F79000200F00D2641D761C96F80090B9F1000F7E
:10F7A00001D0641CECD1BAF1000F05D0E11C504629
:10F7B000FFF77CFD064603E0E01C03F04FFA064627
:10F7C0002EB1304600F8017B4FF05C0925E00020A7
:10F7D00066E61F2907D9222905D05C2903D000F845
:10F7E000011B6D1C19E000F8019B044615F8012B64
:10F7F0000C2A25D006DC082A1ED0092A2CD00A2A79
:10F8000006D121E00D2A23D0222A12D05C2A0CD066
:10F810001BA1204608F0D2FB601D29780029D8D111
:10F82000077080F8018030463AE684F80090601C4A
:10F83000F3E72770601CF0E762202070601CECE7A3
:10F8400066202070601CE8E76E202070601CE4E7F2
:10F8500072202070601CE0E774202070601CDCE7E0
:10F86000006937E7256500002566000018020020C2
:10F8700082BD020822220000225C080C0A0D090049
:10F88000752530347800000000E0401C002804D0CA
:10F890000178002901D02029F7D970472DE9F041DE
:10F8A00007460878FE4E7B2803D031600020BDE873
:10F8B000F0810620F860481CFFF7E6FF054628782F
:10F8C0007D2818D0FFF700FC0446B860A8B1284690
:10F8D000FFF7DAFF01462046FFF743FEFFF7D4FFAC
:10F8E00068B1216921620027276101783A2908D08F
:10F8F00030600020DBE7681CD9E70020D7E7002054
:10F90000D5E7401CFFF7C0FF0146204600F086F80F
:10F91000FFF7BAFF0546280028D1C8E7FFF7D4FB58
:10F92000A8B1206044600446681CFFF7ADFF0146A3
:10F930002046FFF716FEFFF7A7FF50B121692162AD
:10F94000276101783A2906D030600020AFE7002017
:10F95000ADE70020ABE7401CFFF796FF01462046CD
:10F9600000F05CF8FFF790FF054645B128782C2899
:10F97000D4D028787D2804D03560002097E7002077
:10F9800095E7681C93E72DE9F04107460878C44ED7
:10F990005B2802D03160002089E70520F860481C10
:10F9A000FFF772FF044620785D2811D0FFF78CFB2B
:10F9B0000546B86070B12046FFF766FF014628464D
:10F9C00000F02CF8FFF760FF0446200004D016E09A
:10F9D000601C6CE700206AE7002068E7FFF774FB13
:10F9E000B0B1286045600546601CFFF74DFF014639
:10F9F000284600F013F8FFF747FF044654B120787B
:10FA00002C28EBD020785D2806D0346000204EE70B
:10FA100000204CE700204AE7601C48E770B5054627
:10FA20000C46002C20D004229EA1204608F0F8FDB0
:10FA3000E0B105229DA1204608F0F2FDD0B10422DC
:10FA40009CA1204608F0ECFDC0B1207822281AD0F5
:10FA50002D2803D0A0F13001092919D821462846C4
:10FA6000BDE87040FFF75CBB002070BD0220E8607D
:10FA7000201D70BD0020E860601D70BD0120E860A1
:10FA80006861201D70BD21462846BDE8704068E5CC
:10FA90005B2805D07B2808D081480460002070BD19
:10FAA00021462846BDE870406DE721462846BDE85E
:10FAB0007040F3E62DE9F04104460D469046FFF70D
:10FAC00003FB0646764F00203860BEB12046FFF7A4
:10FAD000DBFE01463046FFF7A1FF044684B1B8F1D2
:10FAE000000F12D02046FFF7CFFE0446207860B109
:10FAF0003046FFF7F5FA3C600020D8E60020D6E655
:10FB00003046FFF7EDFA0020D1E605B12C60304613
:10FB1000CDE600221146CDE72DE9F04F85B006462F
:10FB2000894615461C4600200490072002904FF09D
:10FB3000000BB06800270021019101E07F1C0068E4
:10FB40000028FBD137B1002C70D0A76895B34FF0D7
:10FB5000020A32E04CB115B109F1040100E00321C1
:10FB60002046FFF7A3FB024607E015B109F10400A8
:10FB700000E0032003F072F8024662B110467B21D8
:10FB800000F8011B85B10A2100F8011B002109239F
:10FB9000A9F1010906E0002005B0BDE8F08F00F8EA
:10FBA000013B491C4945FADB7D2101700021417070
:10FBB0001046F1E7FFE74FF0010A0AF10101204684
:10FBC000FFF774FB88B17B2100F8011B15B10A21F6
:10FBD00000F8011B4FF0000880F80080A068504436
:10FBE000A060B66809F101096CE00020D4E78DB18E
:10FBF00049462046FFF75AFB10B10021092204E0D4
:10FC00000020C9E700F8012B491C4945FADBA06830
:10FC10004844A0602146306AFFF75CFD2046FFF7AC
:10FC200070FBA0601DB14FF0020A02E06CE04FF0E3
:10FC3000010A51462046FFF739FBA8B13A2100F8E6
:10FC4000011B0DB109210170A0685044A06023463A
:10FC50002A464946304600F026FA2046FFF751FB77
:10FC6000A0601DB1012002E0002095E7002031686E
:10FC700009B1012100E0002100EB010A0AF10101B4
:10FC80002046FFF713FB18B3316811B12C2100F89F
:10FC9000011B15B10A2100F8011B80F800800DE05E
:10FCA000180200206E756C6C0000000066616C73B9
:10FCB000650000007472756500000000A068504483
:10FCC000A0603668002E92D125B109F1010102E051
:10FCD000002061E702212046FFF7E8FA28B15DB174
:10FCE00000270921A9F1010904E0002054E700F8E8
:10FCF000011B7F1C4F45FADB7D21017080F80180DC
:10FD0000206838440490D7E0BC00204602F0A6FFEB
:10FD100080465FEA080016D0204602F09FFF824628
:10FD20005FEA0A0011D02146404608F071FD2146E5
:10FD3000504608F06DFDB46809F101098DB30298D1
:10FD40004844029031E0002026E7404602F0C0FF20
:10FD5000002021E70021206AFFF7BCFC03904AF84D
:10FD60002B0000232A464946204600F09CF95946BC
:10FD70000BF1010B48F82100039999B190B108F0FB
:10FD800030FC0646039808F02CFC311815B109F137
:10FD9000020000E00020014402980844801C029008
:10FDA00002E002E0012001902468002CD2D10198E9
:10FDB00018B9029802F052FF0490049808B9012083
:10FDC00001900198B0B100240AE05AF8240008B16B
:10FDD00002F07EFF58F8240008B102F079FF641C9D
:10FDE000BC42F2DB504602F073FF404602F070FF67
:10FDF0000020D1E604997B200870049C641C15B196
:10FE00000A2004F8010B4FF0000B84F800B0002624
:10FE10003BE03DB10020092102E004F8011B401C39
:10FE20004845FADB5AF8260008F0DBFB00905AF848
:10FE300026102046009A08F04AFC009804443A2014
:10FE400004F8010B15B1092004F8010B58F826102D
:10FE5000204608F097FB58F8260008F0C2FB04443F
:10FE6000781E864202D02C2004F8010B15B10A201E
:10FE700004F8010B84F800B05AF8260002F028FFBD
:10FE800058F8260002F024FF761CBE42C1DB504623
:10FE900002F01EFF404602F01BFF4DB10020092179
:10FEA000A9F1010902E004F8011B401C4845FADBF6
:10FEB0007D20207084F801B004986DE62DE9FF4F95
:10FEC00081B0834690461F464FF000094FF0050A67
:10FED000DBF8080000260025002401E0761C0068FD
:10FEE0000028FBD17EB1002F5FD0BE6801213846CB
:10FEF000FFF7DCF9C8B15B210170B868401CB8603D
:10FF0000DBF808503DE02FB103213846FFF7CEF96A
:10FF1000044603E0032002F0A1FE04461CB1FCA14C
:10FF2000204608F02FFB204636E6002034E60299F2
:10FF30003B464246491C284600F0B5F83846FFF7D4
:10FF4000E0F9B8602868D8B1B8F1000F02D04FF0DE
:10FF5000020901E04FF0010909F101013846FFF7FC
:10FF6000A5F9F0B12C2100F8011BB8F1000F02D067
:10FF7000202100F8011B00210170B8684844B860D6
:10FF80002D680DB1002CD2D002213846FFF78EF932
:10FF900048B15D21017000214170386800EB06090D
:10FFA0007FE00020F8E50020F6E5B000009002F0C8
:10FFB00055FE0746380005D0009908F029FCDBF80B
:10FFC00008B01EE00020E7E5029900234246491CE4
:10FFD000584600F068F829466D1C47F8210068B1C2
:10FFE00008F0FFFA0146B8F1000F01D0012000E04F
:10FFF0000020084482440AF1020A00E00124DBF8F0
:020000040802F0
:1000000000B0BBF1000F01D0002CDDD01CB9504670
:1000100002F024FE8146B9F1000F00D1012474B131
:10002000002405E057F8240008B102F051FE641CDA
:10003000B442F7DB384602F04BFE0020ACE55B2013
:1000400089F800004C464FF0000A04F801AF002583
:100050001EE057F8250008F0C4FA834657F825102B
:100060005A46204608F033FB5C44701E85420AD095
:100070002C2004F8010BB8F1000F02D0202004F866
:10008000010B84F800A057F8250002F021FE6D1C3A
:10009000B542DEDB384602F01BFE5D20207084F89E
:1000A00001A0484678E570B50024002809D083B344
:1000B000057B072D6ED2DFE805F01320062D3237C1
:1000C0003B00002070BD05211846FFF7EFF80446FD
:1000D000002C5FD0AFF23441204608F053FA59E0CB
:1000E00006211846FFF7E2F80446002C52D0AFF282
:1000F0004441204608F046FA4CE005211846FFF737
:10010000D5F8044634B3AFF25441204608F03AFA29
:1001100040E011E01946FFF703F904463AE01946BA
:10012000FFF79EFB044635E0FFF7C8FE044631E0CA
:10013000FFF7F2FC04462DE0037B072B2AD2DFE811
:1001400003F00A1004161B202500AFF2A840FEF7AA
:10015000A4FF04461EE0AFF2AC40FEF79EFF04464B
:1001600018E0AFF2B040FEF798FF044612E000211D
:10017000FFF7D6F804460DE00021FFF771FB0446B7
:1001800008E00023FFF79AFE044603E00023FFF790
:10019000C3FC0446204670BD00230122194682E7B5
:1001A00000231A4619467EE7FEB505460C4616465C
:1001B000204602F053FD00900194002002906B460F
:1001C000324600212846FFF76EFFFEBD8168002001
:1001D00001E0401C09680029FBD17047806801E0FC
:1001E000491E0068002801D00029F9DC704770B56D
:1001F0000D46846800E024682CB12946206AFEF789
:1002000026FF0028F7D1204670BD01604860704786
:1002100070B50546FEF758FF044674B128222946FA
:10022000204608F099FA00202062E16841F48071CC
:10023000E16060602060204670BD002070BD024615
:100240009068002901D010B991607047104610B134
:100250000268002AFAD1D8E770B505460E46144662
:10026000002C0CD0206A08B102F032FD3046FEF7B7
:1002700014FF206221462846BDE87040DFE770BDCC
:1002800070B506460D461446002C10D0A089800596
:1002900003D4206A08B102F01BFD2562E06840F437
:1002A0000070E06021463046BDE87040C7E770BD91
:1002B00010B504460846FFF7ABFF01462046BDE8EF
:1002C0001040BCE770B504460D461046FFF7A0FF8E
:1002D000024629462046BDE87040BDE702469068C8
:1002E00001E00068491E08B10029FADC90B14168BC
:1002F00009B103680B60016809B143684B609168FC
:10030000814201D101689160002101604160704724
:100310005B5D00000020FAE710B5FFF7DFFFBDE8E6
:100320001040FEF7DDBE2DE9F04106460F460025E0
:10033000B46801E06D1C24682CB13946206AFEF7D0
:1003400086FE0028F6D124B129463046BDE8F041AA
:10035000C4E70020BDE8F08110B5FFF7E4FFBDE879
:100360001040FEF7BDBE30B40C461146836801E074
:100370001B68641E0BB1002CFADC4BB10B605A6891
:100380004A60596082689A4204D1816030BC7047EB
:1003900030BC54E748680160F8E730B40346986819
:1003A00001E00068491E08B10029FADC0028EDD000
:1003B000016811604468546001B14A6099688142E3
:1003C00001D19A6001E051680A600021416001603A
:1003D00030BCFEF785BED9E72DE9F04106468846D8
:1003E00017460025B46801E06D1C24682CB1414615
:1003F000206AFEF72CFE0028F6D1002CAAD0404639
:10040000FEF74BFE38623A4629463046BDE8F041D9
:10041000C3E79FE710B5FEF757FE002801D0022181
:10042000C16010BD10B5FEF74FFE002801D00121BC
:10043000C16010BD10B5FEF747FE002801D00021B5
:10044000C16010BD10B50446FEF73EFE002804D082
:100450000CB1012100E00021C16010BD70B504465F
:100460000D46FEF731FE064646B10320F060C6E9B0
:100470000645204629460AF02FFF7061304670BDC0
:1004800070B50546FEF720FE04462CB10420E0605E
:100490002846FEF702FE2061204670BD10B5FEF72B
:1004A00013FE002801D00521C16010BD10B5FEF774
:1004B0000BFE002801D00621C16010BD2DE9F047D8
:1004C000804689460027FFF7E9FF064600240DE035
:1004D00058F824000AF05DFFFFF7C0FF05465CB145
:1004E00029463846FFF791FE2F46641C0EB14C4555
:1004F000EEDB3046BDE8F087B560F5E72DE9F04763
:10050000804689460027FFF7C9FF064600240DE014
:1005100058F824000BF0B4FAFFF7A0FF054654B1D9
:1005200029463846FFF771FE2F46641C0EB14C4534
:10053000EEDB3046DEE7B560F6E72DE9F0478046B2
:1005400089460027FFF7AAFF064600240CE008EBC7
:10055000C40103C9FFF782FF054654B12946384656
:10056000FFF753FE2F46641C0EB14C45EFDB3046BF
:10057000C0E7B560F6E72DE9F047074688464FF03B
:100580000009FFF78BFF064600240BE057F8240014
:10059000FFF776FF054654B129464846FFF735FE7A
:1005A000A946641C0EB14445F0DB3046A2E7B560B5
:1005B000F6E72DE9F04106460F460024002E1DD037
:1005C000FEF782FD054628001AD0F06820F48070FE
:1005D000E86070696861D6E90601C5E9060130691D
:1005E00018B1FEF75AFD286160B1306A18B1FEF704
:1005F00054FD286258B17FB1B66821E00020A9E619
:100600000020A7E62846FEF76BFD0020A2E628465C
:10061000FEF766FD00209DE628469BE60121304658
:10062000FFF7C7FF20B144B120604460044606E0F4
:100630002846FEF755FD00208CE6A8600446366883
:10064000002EEBD1284685E6014626E0202A08D078
:10065000092A08D00D2A08D00A2A08D02F2A08D043
:100660000AE0401C19E0401C17E0401C15E0401C4B
:1006700013E043782F2B03D02F2A06D008E0401C2C
:10068000027852B10A2A08D0F9E743782A2B0BD016
:10069000222A12D001F8012B401C0278002AD5D161
:1006A0000020087033E6401C027822B12A2AFAD1D1
:1006B00042782F2AF7D1801CEFE701F8012B401C6C
:1006C00008E05C2A02D101F8012B401C10F8012B34
:1006D00001F8012B02780AB1222AF2D110F8012B7D
:1006E00001F8012BD9E710220921042003F0EEBD07
:1006F0000921042003F050BE10B5FFF7F9FF4FF4B5
:10070000C87004F092FBBDE81040F1E738B506244C
:100710000C23482219460020009403F0F3FD08231F
:1007200048220B210020009403F0ECFD082348220E
:1007300009210220009403F0E5FD08234822072147
:100740000220009403F0DEFD082348220621022047
:10075000009403F0D7FD082348220F2103200094C2
:1007600003F0D0FD082348220D210320009403F05C
:10077000C9FD48220B21032003F0A8FD48220821CF
:10078000002003F0A3FD48220921022003F09EFD72
:1007900048220821022003F099FD48220E2103205F
:1007A00003F094FDBDE8384048220C21032003F0FB
:1007B0008DBD10220A21042003F088BD0A210420E7
:1007C00003F0EABD10B5FFF7F9FF4FF4C87004F06D
:1007D0002CFBBDE81040F1E710B50A460146114870
:1007E00002F057FB002804D0BDE810400EA002F034
:1007F000CDBA10BD10B504460A4802F041FB0123F2
:100800000C222146002002F03BFEAFF23301BDE88E
:100810001040002002F008BE0A460146002002F007
:1008200064BF0000401100207355736251756575F7
:1008300065D2E7B3F6A3A10010B50A4601461148F8
:1008400002F027FB002804D0BDE810400EA002F003
:100850009DBA10BD10B504460A4802F011FB0523ED
:100860000C222146042002F00BFEAFF23301BDE85A
:100870001040042002F0D8BD0A460146042002F0D0
:1008800034BF000046150020735253323332517585
:10089000657565D2E7B3F6A3A100000010B50A465E
:1008A0000146184802F0F5FA002804D0BDE81040CF
:1008B00015A002F06BBA10BD10B50446102200213D
:1008C000032003F003FD154B00221A600D4802F0CF
:1008D000D7FA05230C222146032002F0D1FDAFF206
:1008E0004301BDE81040032002F09EBD10B50A464A
:1008F0000A4C012121600146032002F0F6FE00208F
:10090000206010BD4C190020735253343835517596
:10091000657565D2E7B3F6A3A1000000808122428D
:100920000320401EC0B2FCD27047F0B5034600253C
:1009300000260127FE4C01290CD00022C4F8986142
:10094000C4F89061C4F894613AB118060DD5C4F8A2
:100950009C610CE0C4F89871F2E7180602D5C4F85F
:100960009C7104E0C4F89C6101E0C4F89C71C4F877
:100970009471FFF7D5FF5806030E6D1CEDB2082DDC
:10098000E0D3C4F89071C4F89871F0BD10B5044676
:10099000B031C8B200221146FFF7C7FFA41CC4F350
:1009A0000310002240F010001146FFF7BEFF04F0D4
:1009B0000F000022BDE810401146B6E72DE9F041D6
:1009C000804606980E461F4600242038C5B2B8F16E
:1009D0007F0F02D9A046B61CF6B20C2A06D0102A08
:1009E00019D0BDE8F041D3A002F0D0B9761CF1B225
:1009F0004046FFF7CBFFD44905EB450001EB40052E
:100A00003A46285D0121FFF790FF641CE4B2062CF2
:100A1000F6D3BDE8F08131464046FFF7B7FFCB483B
:100A200000EB05153A46285D0121FFF77EFF641CA7
:100A3000E4B2082CF6D3761CF1B24046FFF7A6FFCD
:100A4000002428193A46007A0121FFF76EFF641C42
:100A5000E4B2082CF5D3DCE72DE9F8430446DDF8D1
:100A600020800E4691461F46002510E000904B4620
:100A7000424631462046FFF7A1FF04EB5800C4B2BE
:100A8000782C02D90024761CF6B26D1CEDB2785D8C
:100A90000028EBD1BDE8F88308B51021400600918D
:100AA000010E0022AAA31046FFF7D6FF08BD0FB41F
:100AB0002DE9FE4F0C46934600254FEA540880204E
:100AC000B0FBF8F64FEA4B07102C1BD00420029025
:100AD0000DF14409CDF80490701C02F0BFF8824675
:100AE0004B46711C5046109A07F042FA8146B145B8
:100AF0000BD90AEB060010F8010C7F2805D9A6F1E6
:100B0000010905E04A200290E2E7B14500D9B1466B
:100B10000C98012802D002280AD105E0A6EB0900B2
:100B2000400808FB00F503E0A6EB090008FB00F510
:100B3000B9F1000F7CDD5846FFF7AEFF00268BE0D1
:100B40001AF806107F2909D80091F9B2E8B22246B6
:100B50000F9BFFF733FF05EB54057CE0002077E0A7
:100B6000102C02D00C2C38D071E0C0EBC00202EB8C
:100B700082037C4A03EB020898F82020914266D158
:100B80000AEB060298F8213052789A425FD1F9B206
:100B9000E8B2FFF7FBFE4FF0000B07E018F80B0080
:100BA00001210F9AFFF7C1FE0BF1010BA345F5D30D
:100BB000781CC1B2E8B2FFF7E9FEA34607E018F8D7
:100BC0000B0001210F9AFFF7B0FE0BF1010BBBEBFD
:100BD000440FF4D32544761C3DE000EBC00202EB49
:100BE0004203604A6C3A03EB020898F818209142DD
:100BF0002DD10AEB060298F8193052789A4226D184
